 jaccessinspector

 Timestamp is fd691ca9 (reproducible build file hash)

 Preferred load address is 0000000140000000

 Start         Length     Name                   Class
 0001:00000000 00000030H .text$di                CODE
 0001:00000030 0000f1d0H .text$mn                CODE
 0001:0000f200 00000040H .text$mn$00             CODE
 0001:0000f240 00000090H .text$x                 CODE
 0001:0000f2d0 00000015H .text$yd                CODE
 0002:00000000 00000440H .idata$5                DATA
 0002:00000440 00000038H .00cfg                  DATA
 0002:00000478 00000008H .CRT$XCA                DATA
 0002:00000480 00000008H .CRT$XCAA               DATA
 0002:00000488 00000008H .CRT$XCU                DATA
 0002:00000490 00000008H .CRT$XCZ                DATA
 0002:00000498 00000008H .CRT$XIA                DATA
 0002:000004a0 00000008H .CRT$XIAA               DATA
 0002:000004a8 00000008H .CRT$XIAC               DATA
 0002:000004b0 00000008H .CRT$XIZ                DATA
 0002:000004b8 00000008H .CRT$XLA                DATA
 0002:000004c0 00000008H .CRT$XLZ                DATA
 0002:000004c8 00000008H .CRT$XPA                DATA
 0002:000004d0 00000008H .CRT$XPZ                DATA
 0002:000004d8 00000008H .CRT$XTA                DATA
 0002:000004e0 00000010H .CRT$XTZ                DATA
 0002:000004e8 00000000H .gehcont$y              DATA
 0002:000004e8 00000000H .gfids$y                DATA
 0002:000004f0 00002410H .rdata                  DATA
 0002:00002900 00000000H .rdata$CastGuardVftablesA DATA
 0002:00002900 00000000H .rdata$CastGuardVftablesC DATA
 0002:00002900 00000028H .rdata$T                DATA
 0002:00002928 000001f4H .rdata$r                DATA
 0002:00002b1c 00000118H .rdata$voltmd           DATA
 0002:00002c34 000003e4H .rdata$zzzdbg           DATA
 0002:00003018 00000008H .rtc$IAA                DATA
 0002:00003020 00000008H .rtc$IZZ                DATA
 0002:00003028 00000008H .rtc$TAA                DATA
 0002:00003030 00000008H .rtc$TZZ                DATA
 0002:00003038 00000004H .tls                    DATA
 0002:0000303c 00000004H .tls$                   DATA
 0002:00003040 00000008H .tls$ZZZ                DATA
 0002:00003048 000008c0H .xdata                  DATA
 0002:00003908 000000ecH .xdata$x                DATA
 0002:000039f4 00000000H .edata                  DATA
 0002:000039f4 00000118H .idata$2                DATA
 0002:00003b0c 00000014H .idata$3                DATA
 0002:00003b20 00000440H .idata$4                DATA
 0002:00003f60 00000a28H .idata$6                DATA
 0003:00000000 00000b98H .data                   DATA
 0003:00000b98 00000080H .data$r                 DATA
 0003:00000c18 00000028H .data$rs                DATA
 0003:00000c40 00000b80H .bss                    DATA
 0004:00000000 00000f6cH .pdata                  DATA
 0005:00000000 000001c0H .rsrc$01                DATA
 0005:000001c0 00000ed0H .rsrc$02                DATA

  Address         Publics by Value              Rva+Base               Lib:Object

 0000:00000000       __AbsoluteZero             0000000000000000     <absolute>
 0000:00000000       ___safe_se_handler_count   0000000000000000     <absolute>
 0000:00000000       ___safe_se_handler_table   0000000000000000     <absolute>
 0000:00000000       __arm64x_extra_rfe_table   0000000000000000     <absolute>
 0000:00000000       __arm64x_extra_rfe_table_size 0000000000000000     <absolute>
 0000:00000000       __arm64x_native_entrypoint 0000000000000000     <absolute>
 0000:00000000       __arm64x_redirection_metadata 0000000000000000     <absolute>
 0000:00000000       __arm64x_redirection_metadata_count 0000000000000000     <absolute>
 0000:00000000       __dynamic_value_reloc_table 0000000000000000     <absolute>
 0000:00000000       __enclave_config           0000000000000000     <absolute>
 0000:00000000       __guard_check_icall_a64n_fptr 0000000000000000     <absolute>
 0000:00000000       __guard_eh_cont_count      0000000000000000     <absolute>
 0000:00000000       __guard_eh_cont_table      0000000000000000     <absolute>
 0000:00000000       __guard_fids_count         0000000000000000     <absolute>
 0000:00000000       __guard_fids_table         0000000000000000     <absolute>
 0000:00000000       __guard_iat_count          0000000000000000     <absolute>
 0000:00000000       __guard_iat_table          0000000000000000     <absolute>
 0000:00000000       __guard_longjmp_count      0000000000000000     <absolute>
 0000:00000000       __guard_longjmp_table      0000000000000000     <absolute>
 0000:00000000       __hybrid_auxiliary_delayload_iat 0000000000000000     <absolute>
 0000:00000000       __hybrid_auxiliary_delayload_iat_copy 0000000000000000     <absolute>
 0000:00000000       __hybrid_auxiliary_iat     0000000000000000     <absolute>
 0000:00000000       __hybrid_auxiliary_iat_copy 0000000000000000     <absolute>
 0000:00000000       __hybrid_code_map          0000000000000000     <absolute>
 0000:00000000       __hybrid_code_map_count    0000000000000000     <absolute>
 0000:00000000       __hybrid_image_info_bitfield 0000000000000000     <absolute>
 0000:00000000       __x64_code_ranges_to_entry_points 0000000000000000     <absolute>
 0000:00000000       __x64_code_ranges_to_entry_points_count 0000000000000000     <absolute>
 0000:00000100       __guard_flags              0000000000000100     <absolute>
 0000:00000000       __ImageBase                0000000140000000     <linker-defined>
 0001:00000030       initializeAccessBridge     0000000140001030 f   AccessBridgeCalls.obj
 0001:00001100       shutdownAccessBridge       0000000140002100 f   AccessBridgeCalls.obj
 0001:00001150       IsJavaWindow               0000000140002150 f   AccessBridgeCalls.obj
 0001:00001190       GetAccessibleContextFromHWND 0000000140002190 f   AccessBridgeCalls.obj
 0001:000011d0       getHWNDFromAccessibleContext 00000001400021d0 f   AccessBridgeCalls.obj
 0001:00001210       SetJavaShutdown            0000000140002210 f   AccessBridgeCalls.obj
 0001:00001240       SetFocusGained             0000000140002240 f   AccessBridgeCalls.obj
 0001:00001270       SetFocusLost               0000000140002270 f   AccessBridgeCalls.obj
 0001:000012a0       SetCaretUpdate             00000001400022a0 f   AccessBridgeCalls.obj
 0001:000012d0       SetMouseClicked            00000001400022d0 f   AccessBridgeCalls.obj
 0001:00001300       SetMouseEntered            0000000140002300 f   AccessBridgeCalls.obj
 0001:00001330       SetMouseExited             0000000140002330 f   AccessBridgeCalls.obj
 0001:00001360       SetMousePressed            0000000140002360 f   AccessBridgeCalls.obj
 0001:00001390       SetMouseReleased           0000000140002390 f   AccessBridgeCalls.obj
 0001:000013c0       SetMenuCanceled            00000001400023c0 f   AccessBridgeCalls.obj
 0001:000013f0       SetMenuDeselected          00000001400023f0 f   AccessBridgeCalls.obj
 0001:00001420       SetMenuSelected            0000000140002420 f   AccessBridgeCalls.obj
 0001:00001450       SetPopupMenuCanceled       0000000140002450 f   AccessBridgeCalls.obj
 0001:00001480       SetPopupMenuWillBecomeInvisible 0000000140002480 f   AccessBridgeCalls.obj
 0001:000014b0       SetPopupMenuWillBecomeVisible 00000001400024b0 f   AccessBridgeCalls.obj
 0001:000014e0       SetPropertyNameChange      00000001400024e0 f   AccessBridgeCalls.obj
 0001:00001510       SetPropertyDescriptionChange 0000000140002510 f   AccessBridgeCalls.obj
 0001:00001540       SetPropertyStateChange     0000000140002540 f   AccessBridgeCalls.obj
 0001:00001570       SetPropertyValueChange     0000000140002570 f   AccessBridgeCalls.obj
 0001:000015a0       SetPropertySelectionChange 00000001400025a0 f   AccessBridgeCalls.obj
 0001:000015d0       SetPropertyTextChange      00000001400025d0 f   AccessBridgeCalls.obj
 0001:00001600       SetPropertyCaretChange     0000000140002600 f   AccessBridgeCalls.obj
 0001:00001630       SetPropertyVisibleDataChange 0000000140002630 f   AccessBridgeCalls.obj
 0001:00001660       SetPropertyChildChange     0000000140002660 f   AccessBridgeCalls.obj
 0001:00001690       SetPropertyActiveDescendentChange 0000000140002690 f   AccessBridgeCalls.obj
 0001:000016c0       SetPropertyTableModelChange 00000001400026c0 f   AccessBridgeCalls.obj
 0001:000016f0       ReleaseJavaObject          00000001400026f0 f   AccessBridgeCalls.obj
 0001:00001720       GetVersionInfo             0000000140002720 f   AccessBridgeCalls.obj
 0001:00001760       GetAccessibleContextAt     0000000140002760 f   AccessBridgeCalls.obj
 0001:000017c0       GetAccessibleContextWithFocus 00000001400027c0 f   AccessBridgeCalls.obj
 0001:00001800       GetAccessibleContextInfo   0000000140002800 f   AccessBridgeCalls.obj
 0001:00001840       GetAccessibleChildFromContext 0000000140002840 f   AccessBridgeCalls.obj
 0001:00001880       GetAccessibleParentFromContext 0000000140002880 f   AccessBridgeCalls.obj
 0001:000018c0       GetAccessibleTextInfo      00000001400028c0 f   AccessBridgeCalls.obj
 0001:00001910       GetAccessibleTextItems     0000000140002910 f   AccessBridgeCalls.obj
 0001:00001960       GetAccessibleTextSelectionInfo 0000000140002960 f   AccessBridgeCalls.obj
 0001:000019a0       GetAccessibleTextAttributes 00000001400029a0 f   AccessBridgeCalls.obj
 0001:000019f0       GetAccessibleTextRect      00000001400029f0 f   AccessBridgeCalls.obj
 0001:00001a40       GetAccessibleTextLineBounds 0000000140002a40 f   AccessBridgeCalls.obj
 0001:00001aa0       GetAccessibleTextRange     0000000140002aa0 f   AccessBridgeCalls.obj
 0001:00001b00       getAccessibleTableInfo     0000000140002b00 f   AccessBridgeCalls.obj
 0001:00001b40       getAccessibleTableCellInfo 0000000140002b40 f   AccessBridgeCalls.obj
 0001:00001ba0       getAccessibleTableRowHeader 0000000140002ba0 f   AccessBridgeCalls.obj
 0001:00001be0       getAccessibleTableColumnHeader 0000000140002be0 f   AccessBridgeCalls.obj
 0001:00001c20       getAccessibleTableRowDescription 0000000140002c20 f   AccessBridgeCalls.obj
 0001:00001c60       getAccessibleTableColumnDescription 0000000140002c60 f   AccessBridgeCalls.obj
 0001:00001ca0       getAccessibleTableRowSelectionCount 0000000140002ca0 f   AccessBridgeCalls.obj
 0001:00001ce0       isAccessibleTableRowSelected 0000000140002ce0 f   AccessBridgeCalls.obj
 0001:00001d20       getAccessibleTableRowSelections 0000000140002d20 f   AccessBridgeCalls.obj
 0001:00001d70       getAccessibleTableColumnSelectionCount 0000000140002d70 f   AccessBridgeCalls.obj
 0001:00001db0       isAccessibleTableColumnSelected 0000000140002db0 f   AccessBridgeCalls.obj
 0001:00001df0       getAccessibleTableColumnSelections 0000000140002df0 f   AccessBridgeCalls.obj
 0001:00001e40       getAccessibleTableRow      0000000140002e40 f   AccessBridgeCalls.obj
 0001:00001e90       getAccessibleTableColumn   0000000140002e90 f   AccessBridgeCalls.obj
 0001:00001ee0       getAccessibleTableIndex    0000000140002ee0 f   AccessBridgeCalls.obj
 0001:00001f30       getAccessibleRelationSet   0000000140002f30 f   AccessBridgeCalls.obj
 0001:00001f70       getAccessibleHypertext     0000000140002f70 f   AccessBridgeCalls.obj
 0001:00001fb0       activateAccessibleHyperlink 0000000140002fb0 f   AccessBridgeCalls.obj
 0001:00001ff0       getAccessibleHyperlinkCount 0000000140002ff0 f   AccessBridgeCalls.obj
 0001:00002030       getAccessibleHypertextExt  0000000140003030 f   AccessBridgeCalls.obj
 0001:00002080       getAccessibleHypertextLinkIndex 0000000140003080 f   AccessBridgeCalls.obj
 0001:000020d0       getAccessibleHyperlink     00000001400030d0 f   AccessBridgeCalls.obj
 0001:00002120       getAccessibleKeyBindings   0000000140003120 f   AccessBridgeCalls.obj
 0001:00002160       getAccessibleIcons         0000000140003160 f   AccessBridgeCalls.obj
 0001:000021a0       getAccessibleActions       00000001400031a0 f   AccessBridgeCalls.obj
 0001:000021e0       doAccessibleActions        00000001400031e0 f   AccessBridgeCalls.obj
 0001:00002230       IsSameObject               0000000140003230 f   AccessBridgeCalls.obj
 0001:00002270       setTextContents            0000000140003270 f   AccessBridgeCalls.obj
 0001:000022b0       getParentWithRole          00000001400032b0 f   AccessBridgeCalls.obj
 0001:000022f0       getParentWithRoleElseRoot  00000001400032f0 f   AccessBridgeCalls.obj
 0001:00002330       getTopLevelObject          0000000140003330 f   AccessBridgeCalls.obj
 0001:00002370       getObjectDepth             0000000140003370 f   AccessBridgeCalls.obj
 0001:000023b0       getActiveDescendent        00000001400033b0 f   AccessBridgeCalls.obj
 0001:000023f0       GetCurrentAccessibleValueFromContext 00000001400033f0 f   AccessBridgeCalls.obj
 0001:00002440       GetMaximumAccessibleValueFromContext 0000000140003440 f   AccessBridgeCalls.obj
 0001:00002490       GetMinimumAccessibleValueFromContext 0000000140003490 f   AccessBridgeCalls.obj
 0001:000024e0       GetAccessibleSelectionFromContext 00000001400034e0 f   AccessBridgeCalls.obj
 0001:00002520       GetAccessibleSelectionCountFromContext 0000000140003520 f   AccessBridgeCalls.obj
 0001:00002560       IsAccessibleChildSelectedFromContext 0000000140003560 f   AccessBridgeCalls.obj
 0001:000025a0       RemoveAccessibleSelectionFromContext 00000001400035a0 f   AccessBridgeCalls.obj
 0001:000025e0       SelectAllAccessibleSelectionFromContext 00000001400035e0 f   AccessBridgeCalls.obj
 0001:00002610       getVirtualAccessibleName   0000000140003610 f   AccessBridgeCalls.obj
 0001:00002660       requestFocus               0000000140003660 f   AccessBridgeCalls.obj
 0001:000026a0       selectTextRange            00000001400036a0 f   AccessBridgeCalls.obj
 0001:000026f0       getTextAttributesInRange   00000001400036f0 f   AccessBridgeCalls.obj
 0001:00002750       getVisibleChildrenCount    0000000140003750 f   AccessBridgeCalls.obj
 0001:00002790       getVisibleChildren         0000000140003790 f   AccessBridgeCalls.obj
 0001:000027e0       setCaretPosition           00000001400037e0 f   AccessBridgeCalls.obj
 0001:00002820       getCaretLocation           0000000140003820 f   AccessBridgeCalls.obj
 0001:00002870       getEventsWaiting           0000000140003870 f   AccessBridgeCalls.obj
 0001:000028a0       addAccessibleSelectionFromContext 00000001400038a0 f   AccessBridgeCalls.obj
 0001:000028e0       clearAccessibleSelectionFromContext 00000001400038e0 f   AccessBridgeCalls.obj
 0001:00002910       printError                 0000000140003910 f   AccessBridgeDebug.obj
 0001:00002a60       PrintDebugString           0000000140003a60 f   AccessBridgeDebug.obj
 0001:00002af0       wPrintJavaDebugString      0000000140003af0 f   AccessBridgeDebug.obj
 0001:00002b80       wPrintDebugString          0000000140003b80 f   AccessBridgeDebug.obj
 0001:00002c10       initializeFileLogger       0000000140003c10 f   AccessBridgeDebug.obj
 0001:00002d90       finalizeFileLogger         0000000140003d90 f   AccessBridgeDebug.obj
 0001:00002dd0       getTimeStamp               0000000140003dd0 f   AccessBridgeDebug.obj
 0001:00002e20       PrintJavaDebugString2      0000000140003e20 f   AccessBridgeDebug.obj
 0001:00002ea0       __local_stdio_printf_options 0000000140003ea0 f i AccessBridgeDebug.obj
 0001:00002eb0       _vfprintf_l                0000000140003eb0 f i AccessBridgeDebug.obj
 0001:00002f00       _vfwprintf_l               0000000140003f00 f i AccessBridgeDebug.obj
 0001:00002f50       fprintf                    0000000140003f50 f i AccessBridgeDebug.obj
 0001:00002fa0       printf                     0000000140003fa0 f i AccessBridgeDebug.obj
 0001:00003000       vfprintf                   0000000140004000 f i AccessBridgeDebug.obj
 0001:00003030       vfwprintf                  0000000140004030 f i AccessBridgeDebug.obj
 0001:00003060       ?initBroadcastMessageIDs@@YAHXZ 0000000140004060 f   AccessBridgeMessages.obj
 0001:000030b0       ?getTimeAndDate@@YAPEADXZ  00000001400040b0 f   AccessInfo.obj
 0001:00003180       ?displayAndLog@@YAXPEAUHWND__@@HPEAU_iobuf@@PEADZZ 0000000140004180 f   AccessInfo.obj
 0001:000032a0       ?logString@@YAXPEAU_iobuf@@PEBDZZ 00000001400042a0 f   AccessInfo.obj
 0001:00003360       ?getAccessibleInfo@@YAPEADJ_JPEADH@Z 0000000140004360 f   AccessInfo.obj
 0001:000033b0       ?getAccessibleInfo@@YAPEADJ_JHHPEADH@Z 00000001400043b0 f   AccessInfo.obj
 0001:00005d90       ?appendToBuffer@@YAHPEAD_KPEBDZZ 0000000140006d90 f   AccessInfo.obj
 0001:00005ea0       snprintf                   0000000140006ea0 f i AccessInfo.obj
 0001:00005f00       vsnprintf                  0000000140006f00 f i AccessInfo.obj
 0001:00005f80       ?AddMessage@MessageHistory@@QEAAXPEBD@Z 0000000140006f80 f   MessageHistory.obj
 0001:00006070       ?GetFirstMessage@MessageHistory@@QEAAPEBDXZ 0000000140007070 f   MessageHistory.obj
 0001:000060e0       ?GetPreviousMessage@MessageHistory@@QEAAPEBDXZ 00000001400070e0 f   MessageHistory.obj
 0001:00006170       ?GetNextMessage@MessageHistory@@QEAAPEBDXZ 0000000140007170 f   MessageHistory.obj
 0001:00006210       ?GetLastMessage@MessageHistory@@QEAAPEBDXZ 0000000140007210 f   MessageHistory.obj
 0001:00006290       ?GetCurrentMessage@MessageHistory@@QEAAPEBDXZ 0000000140007290 f   MessageHistory.obj
 0001:000062e0       ?GetMessageA@MessageHistory@@QEAAPEBD_K@Z 00000001400072e0 f   MessageHistory.obj
 0001:00006380       ?GetCurrentMessageIndex@MessageHistory@@QEAA_KXZ 0000000140007380 f   MessageHistory.obj
 0001:000063f0       ?IsFirstMessage@MessageHistory@@QEAAHXZ 00000001400073f0 f   MessageHistory.obj
 0001:00006450       ?IsLastMessage@MessageHistory@@QEAAHXZ 0000000140007450 f   MessageHistory.obj
 0001:000064d0       ?GetMessageCount@MessageHistory@@QEAA_KXZ 00000001400074d0 f   MessageHistory.obj
 0001:00006500       ?clear@MessageHistory@@QEAAXXZ 0000000140007500 f   MessageHistory.obj
 0001:00006520       ??$?0$$V@?$_Compressed_pair@V?$allocator@D@std@@V?$_String_val@U?$_Simple_types@D@std@@@2@$00@std@@QEAA@U_Zero_then_variadic_args_t@1@@Z 0000000140007520 f i MessageHistory.obj
 0001:00006550       ??$?0V?$allocator@D@std@@$$V@?$_Compressed_pair@V?$allocator@D@std@@V?$_String_val@U?$_Simple_types@D@std@@@2@$00@std@@QEAA@U_One_then_variadic_args_t@1@$$QEAV?$allocator@D@1@@Z 0000000140007550 f i MessageHistory.obj
 0001:00006590       ??$?0V?$basic_string@DU?$char_traits@D@std@@V?$allocator@D@2@@std@@@?$_List_node_emplace_op2@V?$allocator@U?$_List_node@V?$basic_string@DU?$char_traits@D@std@@V?$allocator@D@2@@std@@PEAX@std@@@std@@@std@@QEAA@AEAV?$allocator@U?$_List_node@V?$basic_string@DU?$char_traits@D@std@@V?$allocator@D@2@@std@@PEAX@std@@@1@$$QEAV?$basic_string@DU?$char_traits@D@std@@V?$allocator@D@2@@1@@Z 0000000140007590 f i MessageHistory.obj
 0001:00006610       ??$_Adl_verify_range@V?$_List_const_iterator@V?$_List_val@U?$_List_simple_types@V?$basic_string@DU?$char_traits@D@std@@V?$allocator@D@2@@std@@@std@@@std@@@std@@V12@@std@@YAXAEBV?$_List_const_iterator@V?$_List_val@U?$_List_simple_types@V?$basic_string@DU?$char_traits@D@std@@V?$allocator@D@2@@std@@@std@@@std@@@0@0@Z 0000000140007610 f i MessageHistory.obj
 0001:00006610       ?_Adopt@_Iterator_base0@std@@QEAAXPEBX@Z 0000000140007610 f i MessageHistory.obj
 0001:00006610       ?_Alloc_proxy@_Container_base0@std@@QEAAXAEBU_Fake_allocator@2@@Z 0000000140007610 f i MessageHistory.obj
 0001:00006610       ?_Orphan_ptr2@?$_List_val@U?$_List_simple_types@V?$basic_string@DU?$char_traits@D@std@@V?$allocator@D@2@@std@@@std@@@std@@QEAAXPEAU?$_List_node@V?$basic_string@DU?$char_traits@D@std@@V?$allocator@D@2@@std@@PEAX@2@@Z 0000000140007610 f i MessageHistory.obj
 0001:00006610       ?_Start_element_lifetimes@?$basic_string@DU?$char_traits@D@std@@V?$allocator@D@2@@std@@CAXQEAD_K@Z 0000000140007610 f i MessageHistory.obj
 0001:00006610       ?_Swap_proxy_and_iterators@_Container_base0@std@@QEAAXAEAU12@@Z 0000000140007610 f i MessageHistory.obj
 0001:00006620       ??$_Allocate@$0BA@U_Default_allocate_traits@std@@$0A@@std@@YAPEAX_K@Z 0000000140007620 f i MessageHistory.obj
 0001:00006660       ??$_Allocate_manually_vector_aligned@U_Default_allocate_traits@std@@@std@@YAPEAX_K@Z 0000000140007660 f i MessageHistory.obj
 0001:000066f0       ??$_Construct@$00PEBD@?$basic_string@DU?$char_traits@D@std@@V?$allocator@D@2@@std@@AEAAXQEBD_K@Z 00000001400076f0 f i MessageHistory.obj
 0001:000068c0       ??$_Construct_in_place@PEADAEAPEAD@std@@YAXAEAPEAD0@Z 00000001400078c0 f i MessageHistory.obj
 0001:000068c0       ??$_Construct_in_place@PEADAEBQEAD@std@@YAXAEAPEADAEBQEAD@Z 00000001400078c0 f i MessageHistory.obj
 0001:000068c0       ??$_Construct_in_place@PEAU?$_List_node@V?$basic_string@DU?$char_traits@D@std@@V?$allocator@D@2@@std@@PEAX@std@@AEAPEAU12@@std@@YAXAEAPEAU?$_List_node@V?$basic_string@DU?$char_traits@D@std@@V?$allocator@D@2@@std@@PEAX@0@0@Z 00000001400078c0 f i jaccessinspector.obj
 0001:000068c0       ??$_Construct_in_place@PEAU?$_List_node@V?$basic_string@DU?$char_traits@D@std@@V?$allocator@D@2@@std@@PEAX@std@@AEBQEAU12@@std@@YAXAEAPEAU?$_List_node@V?$basic_string@DU?$char_traits@D@std@@V?$allocator@D@2@@std@@PEAX@0@AEBQEAU10@@Z 00000001400078c0 f i MessageHistory.obj
 0001:00006910       ??$_Convert_size@_K_K@std@@YA_K_K@Z 0000000140007910 f i MessageHistory.obj
 0001:00006910       ??$_Unfancy@D@std@@YAPEADPEAD@Z 0000000140007910 f i MessageHistory.obj
 0001:00006910       ??$addressof@$$CBV?$_String_val@U?$_Simple_types@D@std@@@std@@@std@@YAPEBV?$_String_val@U?$_Simple_types@D@std@@@0@AEBV10@@Z 0000000140007910 f i MessageHistory.obj
 0001:00006910       ??$addressof@PEAD@std@@YAPEAPEADAEAPEAD@Z 0000000140007910 f i MessageHistory.obj
 0001:00006910       ??$addressof@PEAU?$_List_node@V?$basic_string@DU?$char_traits@D@std@@V?$allocator@D@2@@std@@PEAX@std@@@std@@YAPEAPEAU?$_List_node@V?$basic_string@DU?$char_traits@D@std@@V?$allocator@D@2@@std@@PEAX@0@AEAPEAU10@@Z 0000000140007910 f i MessageHistory.obj
 0001:00006910       ??$addressof@V?$_List_val@U?$_List_simple_types@V?$basic_string@DU?$char_traits@D@std@@V?$allocator@D@2@@std@@@std@@@std@@@std@@YAPEAV?$_List_val@U?$_List_simple_types@V?$basic_string@DU?$char_traits@D@std@@V?$allocator@D@2@@std@@@std@@@0@AEAV10@@Z 0000000140007910 f i MessageHistory.obj
 0001:00006910       ??$addressof@V?$_String_val@U?$_Simple_types@D@std@@@std@@@std@@YAPEAV?$_String_val@U?$_Simple_types@D@std@@@0@AEAV10@@Z 0000000140007910 f i MessageHistory.obj
 0001:00006910       ??$addressof@V?$basic_string@DU?$char_traits@D@std@@V?$allocator@D@2@@std@@@std@@YAPEAV?$basic_string@DU?$char_traits@D@std@@V?$allocator@D@2@@0@AEAV10@@Z 0000000140007910 f i MessageHistory.obj
 0001:00006910       ??$forward@AEAPEAD@std@@YAAEAPEADAEAPEAD@Z 0000000140007910 f i MessageHistory.obj
 0001:00006910       ??$forward@AEAPEAU?$_List_node@V?$basic_string@DU?$char_traits@D@std@@V?$allocator@D@2@@std@@PEAX@std@@@std@@YAAEAPEAU?$_List_node@V?$basic_string@DU?$char_traits@D@std@@V?$allocator@D@2@@std@@PEAX@0@AEAPEAU10@@Z 0000000140007910 f i jaccessinspector.obj
 0001:00006910       ??$forward@AEBQEAD@std@@YAAEBQEADAEBQEAD@Z 0000000140007910 f i MessageHistory.obj
 0001:00006910       ??$forward@AEBQEAU?$_List_node@V?$basic_string@DU?$char_traits@D@std@@V?$allocator@D@2@@std@@PEAX@std@@@std@@YAAEBQEAU?$_List_node@V?$basic_string@DU?$char_traits@D@std@@V?$allocator@D@2@@std@@PEAX@0@AEBQEAU10@@Z 0000000140007910 f i MessageHistory.obj
 0001:00006910       ??$forward@V?$_List_unchecked_const_iterator@V?$_List_val@U?$_List_simple_types@V?$basic_string@DU?$char_traits@D@std@@V?$allocator@D@2@@std@@@std@@@std@@U_Iterator_base0@2@@std@@@std@@YA$$QEAV?$_List_unchecked_const_iterator@V?$_List_val@U?$_List_simple_types@V?$basic_string@DU?$char_traits@D@std@@V?$allocator@D@2@@std@@@std@@@std@@U_Iterator_base0@2@@0@AEAV10@@Z 0000000140007910 f i MessageHistory.obj
 0001:00006910       ??$forward@V?$allocator@D@std@@@std@@YA$$QEAV?$allocator@D@0@AEAV10@@Z 0000000140007910 f i MessageHistory.obj
 0001:00006910       ??$forward@V?$basic_string@DU?$char_traits@D@std@@V?$allocator@D@2@@std@@@std@@YA$$QEAV?$basic_string@DU?$char_traits@D@std@@V?$allocator@D@2@@0@AEAV10@@Z 0000000140007910 f i MessageHistory.obj
 0001:00006910       ??$move@AEAV?$_List_const_iterator@V?$_List_val@U?$_List_simple_types@V?$basic_string@DU?$char_traits@D@std@@V?$allocator@D@2@@std@@@std@@@std@@@std@@@std@@YA$$QEAV?$_List_const_iterator@V?$_List_val@U?$_List_simple_types@V?$basic_string@DU?$char_traits@D@std@@V?$allocator@D@2@@std@@@std@@@std@@@0@AEAV10@@Z 0000000140007910 f i MessageHistory.obj
 0001:00006910       ??$move@AEAV?$_List_unchecked_const_iterator@V?$_List_val@U?$_List_simple_types@V?$basic_string@DU?$char_traits@D@std@@V?$allocator@D@2@@std@@@std@@@std@@U_Iterator_base0@2@@std@@@std@@YA$$QEAV?$_List_unchecked_const_iterator@V?$_List_val@U?$_List_simple_types@V?$basic_string@DU?$char_traits@D@std@@V?$allocator@D@2@@std@@@std@@@std@@U_Iterator_base0@2@@0@AEAV10@@Z 0000000140007910 f i MessageHistory.obj
 0001:00006910       ??$move@AEAV?$allocator@D@std@@@std@@YA$$QEAV?$allocator@D@0@AEAV10@@Z 0000000140007910 f i MessageHistory.obj
 0001:00006910       ??$move@AEAV?$basic_string@DU?$char_traits@D@std@@V?$allocator@D@2@@std@@@std@@YA$$QEAV?$basic_string@DU?$char_traits@D@std@@V?$allocator@D@2@@0@AEAV10@@Z 0000000140007910 f i MessageHistory.obj
 0001:00006910       ??0?$allocator@D@std@@QEAA@XZ 0000000140007910 f i MessageHistory.obj
 0001:00006910       ??0?$allocator@U?$_List_node@V?$basic_string@DU?$char_traits@D@std@@V?$allocator@D@2@@std@@PEAX@std@@@std@@QEAA@XZ 0000000140007910 f i jaccessinspector.obj
 0001:00006910       ?_Get_first@?$_Compressed_pair@V?$allocator@D@std@@V?$_String_val@U?$_Simple_types@D@std@@@2@$00@std@@QEAAAEAV?$allocator@D@2@XZ 0000000140007910 f i MessageHistory.obj
 0001:00006910       ?_Get_first@?$_Compressed_pair@V?$allocator@D@std@@V?$_String_val@U?$_Simple_types@D@std@@@2@$00@std@@QEBAAEBV?$allocator@D@2@XZ 0000000140007910 f i MessageHistory.obj
 0001:00006910       ?_Get_first@?$_Compressed_pair@V?$allocator@U?$_List_node@V?$basic_string@DU?$char_traits@D@std@@V?$allocator@D@2@@std@@PEAX@std@@@std@@V?$_List_val@U?$_List_simple_types@V?$basic_string@DU?$char_traits@D@std@@V?$allocator@D@2@@std@@@std@@@2@$00@std@@QEAAAEAV?$allocator@U?$_List_node@V?$basic_string@DU?$char_traits@D@std@@V?$allocator@D@2@@std@@PEAX@std@@@2@XZ 0000000140007910 f i MessageHistory.obj
 0001:00006910       ?_Get_first@?$_Compressed_pair@V?$allocator@U?$_List_node@V?$basic_string@DU?$char_traits@D@std@@V?$allocator@D@2@@std@@PEAX@std@@@std@@V?$_List_val@U?$_List_simple_types@V?$basic_string@DU?$char_traits@D@std@@V?$allocator@D@2@@std@@@std@@@2@$00@std@@QEBAAEBV?$allocator@U?$_List_node@V?$basic_string@DU?$char_traits@D@std@@V?$allocator@D@2@@std@@PEAX@std@@@2@XZ 0000000140007910 f i MessageHistory.obj
 0001:00006920       ??$_Deallocate@$0BA@$0A@@std@@YAXPEAX_K@Z 0000000140007920 f i MessageHistory.obj
 0001:00006960       ??$_Destroy_in_place@PEAD@std@@YAXAEAPEAD@Z 0000000140007960 f i MessageHistory.obj
 0001:00006960       ??$_Destroy_in_place@PEAU?$_List_node@V?$basic_string@DU?$char_traits@D@std@@V?$allocator@D@2@@std@@PEAX@std@@@std@@YAXAEAPEAU?$_List_node@V?$basic_string@DU?$char_traits@D@std@@V?$allocator@D@2@@std@@PEAX@0@@Z 0000000140007960 f i MessageHistory.obj
 0001:00006960       ??1_Bxty@?$_String_val@U?$_Simple_types@D@std@@@std@@QEAA@XZ 0000000140007960 f i MessageHistory.obj
 0001:00006960       ?_Activate_SSO_buffer@?$_String_val@U?$_Simple_types@D@std@@@std@@QEAAXXZ 0000000140007960 f i MessageHistory.obj
 0001:00006960       ?_Orphan_all@_Container_base0@std@@QEAAXXZ 0000000140007960 f i MessageHistory.obj
 0001:00006960       ?_Orphan_non_end@?$_List_val@U?$_List_simple_types@V?$basic_string@DU?$char_traits@D@std@@V?$allocator@D@2@@std@@@std@@@std@@QEAAXXZ 0000000140007960 f i MessageHistory.obj
 0001:00006960       ?_Release@_Fake_proxy_ptr_impl@std@@QEAAXXZ 0000000140007960 f i MessageHistory.obj
 0001:00006970       ??$_Emplace@V?$basic_string@DU?$char_traits@D@std@@V?$allocator@D@2@@std@@@?$list@V?$basic_string@DU?$char_traits@D@std@@V?$allocator@D@2@@std@@V?$allocator@V?$basic_string@DU?$char_traits@D@std@@V?$allocator@D@2@@std@@@2@@std@@QEAAPEAU?$_List_node@V?$basic_string@DU?$char_traits@D@std@@V?$allocator@D@2@@std@@PEAX@1@QEAU21@$$QEAV?$basic_string@DU?$char_traits@D@std@@V?$allocator@D@2@@1@@Z 0000000140007970 f i MessageHistory.obj
 0001:00006a20       ??$_Free_non_head@V?$allocator@U?$_List_node@V?$basic_string@DU?$char_traits@D@std@@V?$allocator@D@2@@std@@PEAX@std@@@std@@@?$_List_node@V?$basic_string@DU?$char_traits@D@std@@V?$allocator@D@2@@std@@PEAX@std@@SAXAEAV?$allocator@U?$_List_node@V?$basic_string@DU?$char_traits@D@std@@V?$allocator@D@2@@std@@PEAX@std@@@1@PEAU01@@Z 0000000140007a20 f i MessageHistory.obj
 0001:00006a90       ??$_Freenode0@V?$allocator@U?$_List_node@V?$basic_string@DU?$char_traits@D@std@@V?$allocator@D@2@@std@@PEAX@std@@@std@@@?$_List_node@V?$basic_string@DU?$char_traits@D@std@@V?$allocator@D@2@@std@@PEAX@std@@SAXAEAV?$allocator@U?$_List_node@V?$basic_string@DU?$char_traits@D@std@@V?$allocator@D@2@@std@@PEAX@std@@@1@PEAU01@@Z 0000000140007a90 f i MessageHistory.obj
 0001:00006ae0       ??$_Freenode@V?$allocator@U?$_List_node@V?$basic_string@DU?$char_traits@D@std@@V?$allocator@D@2@@std@@PEAX@std@@@std@@@?$_List_node@V?$basic_string@DU?$char_traits@D@std@@V?$allocator@D@2@@std@@PEAX@std@@SAXAEAV?$allocator@U?$_List_node@V?$basic_string@DU?$char_traits@D@std@@V?$allocator@D@2@@std@@PEAX@std@@@1@PEAU01@@Z 0000000140007ae0 f i MessageHistory.obj
 0001:00006b30       ??$_Get_size_of_n@$00@std@@YA_K_K@Z 0000000140007b30 f i MessageHistory.obj
 0001:00006b50       ??$_Get_size_of_n@$0DA@@std@@YA_K_K@Z 0000000140007b50 f i MessageHistory.obj
 0001:00006b90       ??$_Get_unwrapped@AEAV?$_List_const_iterator@V?$_List_val@U?$_List_simple_types@V?$basic_string@DU?$char_traits@D@std@@V?$allocator@D@2@@std@@@std@@@std@@@std@@@std@@YA?A_TAEAV?$_List_const_iterator@V?$_List_val@U?$_List_simple_types@V?$basic_string@DU?$char_traits@D@std@@V?$allocator@D@2@@std@@@std@@@std@@@0@@Z 0000000140007b90 f i MessageHistory.obj
 0001:00006bc0       ??$_Get_unwrapped_n@V?$_List_const_iterator@V?$_List_val@U?$_List_simple_types@V?$basic_string@DU?$char_traits@D@std@@V?$allocator@D@2@@std@@@std@@@std@@@std@@_K@std@@YA?A_T$$QEAV?$_List_const_iterator@V?$_List_val@U?$_List_simple_types@V?$basic_string@DU?$char_traits@D@std@@V?$allocator@D@2@@std@@@std@@@std@@@0@_K@Z 0000000140007bc0 f i MessageHistory.obj
 0001:00006bf0       ??$_Seek_wrapped@V?$_List_const_iterator@V?$_List_val@U?$_List_simple_types@V?$basic_string@DU?$char_traits@D@std@@V?$allocator@D@2@@std@@@std@@@std@@@std@@V?$_List_unchecked_const_iterator@V?$_List_val@U?$_List_simple_types@V?$basic_string@DU?$char_traits@D@std@@V?$allocator@D@2@@std@@@std@@@std@@U_Iterator_base0@2@@2@@std@@YAXAEAV?$_List_const_iterator@V?$_List_val@U?$_List_simple_types@V?$basic_string@DU?$char_traits@D@std@@V?$allocator@D@2@@std@@@std@@@std@@@0@$$QEAV?$_List_unchecked_const_iterator@V?$_List_val@U?$_List_simple_types@V?$basic_string@DU?$char_traits@D@std@@V?$allocator@D@2@@std@@@std@@@std@@U_Iterator_base0@2@@0@@Z 0000000140007bf0 f i MessageHistory.obj
 0001:00006c20       ??$advance@V?$_List_const_iterator@V?$_List_val@U?$_List_simple_types@V?$basic_string@DU?$char_traits@D@std@@V?$allocator@D@2@@std@@@std@@@std@@@std@@_K@std@@YAXAEAV?$_List_const_iterator@V?$_List_val@U?$_List_simple_types@V?$basic_string@DU?$char_traits@D@std@@V?$allocator@D@2@@std@@@std@@@std@@@0@_K@Z 0000000140007c20 f i MessageHistory.obj
 0001:00006c90       ??$construct@V?$basic_string@DU?$char_traits@D@std@@V?$allocator@D@2@@std@@V12@@?$_Default_allocator_traits@V?$allocator@U?$_List_node@V?$basic_string@DU?$char_traits@D@std@@V?$allocator@D@2@@std@@PEAX@std@@@std@@@std@@SAXAEAV?$allocator@U?$_List_node@V?$basic_string@DU?$char_traits@D@std@@V?$allocator@D@2@@std@@PEAX@std@@@1@QEAV?$basic_string@DU?$char_traits@D@std@@V?$allocator@D@2@@1@$$QEAV31@@Z 0000000140007c90 f i MessageHistory.obj
 0001:00006ce0       ??$destroy@V?$basic_string@DU?$char_traits@D@std@@V?$allocator@D@2@@std@@@?$_Default_allocator_traits@V?$allocator@U?$_List_node@V?$basic_string@DU?$char_traits@D@std@@V?$allocator@D@2@@std@@PEAX@std@@@std@@@std@@SAXAEAV?$allocator@U?$_List_node@V?$basic_string@DU?$char_traits@D@std@@V?$allocator@D@2@@std@@PEAX@std@@@1@QEAV?$basic_string@DU?$char_traits@D@std@@V?$allocator@D@2@@1@@Z 0000000140007ce0 f i MessageHistory.obj
 0001:00006d00       ??$distance@V?$_List_const_iterator@V?$_List_val@U?$_List_simple_types@V?$basic_string@DU?$char_traits@D@std@@V?$allocator@D@2@@std@@@std@@@std@@@std@@@std@@YA_JV?$_List_const_iterator@V?$_List_val@U?$_List_simple_types@V?$basic_string@DU?$char_traits@D@std@@V?$allocator@D@2@@std@@@std@@@std@@@0@0@Z 0000000140007d00 f i MessageHistory.obj
 0001:00006d80       ??$max@_K@std@@YAAEB_KAEB_K0@Z 0000000140007d80 f i MessageHistory.obj
 0001:00006dd0       ??$min@_K@std@@YAAEB_KAEB_K0@Z 0000000140007dd0 f i MessageHistory.obj
 0001:00006e20       ??0?$_Alloc_construct_ptr@V?$allocator@U?$_List_node@V?$basic_string@DU?$char_traits@D@std@@V?$allocator@D@2@@std@@PEAX@std@@@std@@@std@@QEAA@AEAV?$allocator@U?$_List_node@V?$basic_string@DU?$char_traits@D@std@@V?$allocator@D@2@@std@@PEAX@std@@@1@@Z 0000000140007e20 f i MessageHistory.obj
 0001:00006e50       ??0?$_List_const_iterator@V?$_List_val@U?$_List_simple_types@V?$basic_string@DU?$char_traits@D@std@@V?$allocator@D@2@@std@@@std@@@std@@@std@@QEAA@PEAU?$_List_node@V?$basic_string@DU?$char_traits@D@std@@V?$allocator@D@2@@std@@PEAX@1@PEBV?$_List_val@U?$_List_simple_types@V?$basic_string@DU?$char_traits@D@std@@V?$allocator@D@2@@std@@@std@@@1@@Z 0000000140007e50 f i MessageHistory.obj
 0001:00006e90       ??0?$_List_iterator@V?$_List_val@U?$_List_simple_types@V?$basic_string@DU?$char_traits@D@std@@V?$allocator@D@2@@std@@@std@@@std@@@std@@QEAA@PEAU?$_List_node@V?$basic_string@DU?$char_traits@D@std@@V?$allocator@D@2@@std@@PEAX@1@PEBV?$_List_val@U?$_List_simple_types@V?$basic_string@DU?$char_traits@D@std@@V?$allocator@D@2@@std@@@std@@@1@@Z 0000000140007e90 f i MessageHistory.obj
 0001:00006ed0       ??0?$_List_unchecked_const_iterator@V?$_List_val@U?$_List_simple_types@V?$basic_string@DU?$char_traits@D@std@@V?$allocator@D@2@@std@@@std@@@std@@U_Iterator_base0@2@@std@@QEAA@PEAU?$_List_node@V?$basic_string@DU?$char_traits@D@std@@V?$allocator@D@2@@std@@PEAX@1@PEBV?$_List_val@U?$_List_simple_types@V?$basic_string@DU?$char_traits@D@std@@V?$allocator@D@2@@std@@@std@@@1@@Z 0000000140007ed0 f i MessageHistory.obj
 0001:00006f10       ??0?$_String_val@U?$_Simple_types@D@std@@@std@@QEAA@XZ 0000000140007f10 f i MessageHistory.obj
 0001:00006f50       ??0?$basic_string@DU?$char_traits@D@std@@V?$allocator@D@2@@std@@QEAA@$$QEAV01@@Z 0000000140007f50 f i MessageHistory.obj
 0001:00006fb0       ??0?$basic_string@DU?$char_traits@D@std@@V?$allocator@D@2@@std@@QEAA@QEBD@Z 0000000140007fb0 f i MessageHistory.obj
 0001:00007000       ??0_Bxty@?$_String_val@U?$_Simple_types@D@std@@@std@@QEAA@XZ 0000000140008000 f i MessageHistory.obj
 0001:00007020       ??0_Fake_proxy_ptr_impl@std@@QEAA@AEBU_Fake_allocator@1@AEBU_Container_base0@1@@Z 0000000140008020 f i MessageHistory.obj
 0001:00007040       ??0bad_alloc@std@@AEAA@QEBD@Z 0000000140008040 f i MessageHistory.obj
 0001:00007080       ??0bad_alloc@std@@QEAA@AEBV01@@Z 0000000140008080 f i MessageHistory.obj
 0001:000070c0       ??0bad_array_new_length@std@@QEAA@AEBV01@@Z 00000001400080c0 f i MessageHistory.obj
 0001:00007100       ??0bad_array_new_length@std@@QEAA@XZ 0000000140008100 f i MessageHistory.obj
 0001:00007140       ??0exception@std@@QEAA@AEBV01@@Z 0000000140008140 f i MessageHistory.obj
 0001:000071a0       ??0exception@std@@QEAA@QEBDH@Z 00000001400081a0 f i MessageHistory.obj
 0001:000071f0       ??1?$_Alloc_construct_ptr@V?$allocator@U?$_List_node@V?$basic_string@DU?$char_traits@D@std@@V?$allocator@D@2@@std@@PEAX@std@@@std@@@std@@QEAA@XZ 00000001400081f0 f i MessageHistory.obj
 0001:00007230       ??1?$_Compressed_pair@V?$allocator@D@std@@V?$_String_val@U?$_Simple_types@D@std@@@2@$00@std@@QEAA@XZ 0000000140008230 f i MessageHistory.obj
 0001:00007250       ??1?$_List_node_emplace_op2@V?$allocator@U?$_List_node@V?$basic_string@DU?$char_traits@D@std@@V?$allocator@D@2@@std@@PEAX@std@@@std@@@std@@QEAA@XZ 0000000140008250 f i MessageHistory.obj
 0001:000072a0       ??1?$_String_val@U?$_Simple_types@D@std@@@std@@QEAA@XZ 00000001400082a0 f i MessageHistory.obj
 0001:000072c0       ??1?$basic_string@DU?$char_traits@D@std@@V?$allocator@D@2@@std@@QEAA@XZ 00000001400082c0 f i MessageHistory.obj
 0001:000072f0       ??1bad_alloc@std@@UEAA@XZ  00000001400082f0 f i MessageHistory.obj
 0001:00007310       ??1bad_array_new_length@std@@UEAA@XZ 0000000140008310 f i MessageHistory.obj
 0001:00007330       ??1exception@std@@UEAA@XZ  0000000140008330 f i MessageHistory.obj
 0001:00007360       ??2@YAPEAX_KPEAX@Z         0000000140008360 f i MessageHistory.obj
 0001:00007370       ??8?$_List_const_iterator@V?$_List_val@U?$_List_simple_types@V?$basic_string@DU?$char_traits@D@std@@V?$allocator@D@2@@std@@@std@@@std@@@std@@QEBA_NAEBV01@@Z 0000000140008370 f i MessageHistory.obj
 0001:00007370       ??8?$_List_unchecked_const_iterator@V?$_List_val@U?$_List_simple_types@V?$basic_string@DU?$char_traits@D@std@@V?$allocator@D@2@@std@@@std@@@std@@U_Iterator_base0@2@@std@@QEBA_NAEBV01@@Z 0000000140008370 f i MessageHistory.obj
 0001:000073b0       ??9?$_List_const_iterator@V?$_List_val@U?$_List_simple_types@V?$basic_string@DU?$char_traits@D@std@@V?$allocator@D@2@@std@@@std@@@std@@@std@@QEBA_NAEBV01@@Z 00000001400083b0 f i MessageHistory.obj
 0001:000073b0       ??9?$_List_unchecked_const_iterator@V?$_List_val@U?$_List_simple_types@V?$basic_string@DU?$char_traits@D@std@@V?$allocator@D@2@@std@@@std@@@std@@U_Iterator_base0@2@@std@@QEBA_NAEBV01@@Z 00000001400083b0 f i MessageHistory.obj
 0001:000073f0       ??D?$_List_const_iterator@V?$_List_val@U?$_List_simple_types@V?$basic_string@DU?$char_traits@D@std@@V?$allocator@D@2@@std@@@std@@@std@@@std@@QEBAAEBV?$basic_string@DU?$char_traits@D@std@@V?$allocator@D@2@@1@XZ 00000001400083f0 f i MessageHistory.obj
 0001:00007410       ??E?$_List_const_iterator@V?$_List_val@U?$_List_simple_types@V?$basic_string@DU?$char_traits@D@std@@V?$allocator@D@2@@std@@@std@@@std@@@std@@QEAAAEAV01@XZ 0000000140008410 f i MessageHistory.obj
 0001:00007410       ??E?$_List_unchecked_const_iterator@V?$_List_val@U?$_List_simple_types@V?$basic_string@DU?$char_traits@D@std@@V?$allocator@D@2@@std@@@std@@@std@@U_Iterator_base0@2@@std@@QEAAAEAV01@XZ 0000000140008410 f i MessageHistory.obj
 0001:00007430       ??F?$_List_const_iterator@V?$_List_val@U?$_List_simple_types@V?$basic_string@DU?$char_traits@D@std@@V?$allocator@D@2@@std@@@std@@@std@@@std@@QEAAAEAV01@XZ 0000000140008430 f i MessageHistory.obj
 0001:00007460       ??_G?$basic_string@DU?$char_traits@D@std@@V?$allocator@D@2@@std@@QEAAPEAXI@Z 0000000140008460 f i MessageHistory.obj
 0001:000074a0       ??_Ebad_alloc@std@@UEAAPEAXI@Z 00000001400084a0 f i MessageHistory.obj
 0001:000074a0       ??_Gbad_alloc@std@@UEAAPEAXI@Z 00000001400084a0 f i MessageHistory.obj
 0001:000074e0       ??_Ebad_array_new_length@std@@UEAAPEAXI@Z 00000001400084e0 f i MessageHistory.obj
 0001:000074e0       ??_Gbad_array_new_length@std@@UEAAPEAXI@Z 00000001400084e0 f i MessageHistory.obj
 0001:00007520       ??_Eexception@std@@UEAAPEAXI@Z 0000000140008520 f i MessageHistory.obj
 0001:00007520       ??_Gexception@std@@UEAAPEAXI@Z 0000000140008520 f i MessageHistory.obj
 0001:00007560       ?_Adjust_manually_vector_aligned@std@@YAXAEAPEAXAEA_K@Z 0000000140008560 f i MessageHistory.obj
 0001:00007600       ?_Allocate@?$_Alloc_construct_ptr@V?$allocator@U?$_List_node@V?$basic_string@DU?$char_traits@D@std@@V?$allocator@D@2@@std@@PEAX@std@@@std@@@std@@QEAAXXZ 0000000140008600 f i MessageHistory.obj
 0001:00007640       ?_Allocate@_Default_allocate_traits@std@@SAPEAX_K@Z 0000000140008640 f i MessageHistory.obj
 0001:00007660       ?_Calculate_growth@?$basic_string@DU?$char_traits@D@std@@V?$allocator@D@2@@std@@AEBA_K_K@Z 0000000140008660 f i MessageHistory.obj
 0001:000076a0       ?_Calculate_growth@?$basic_string@DU?$char_traits@D@std@@V?$allocator@D@2@@std@@CA_K_K00@Z 00000001400086a0 f i MessageHistory.obj
 0001:00007740       ?_Getal@?$basic_string@DU?$char_traits@D@std@@V?$allocator@D@2@@std@@AEAAAEAV?$allocator@D@2@XZ 0000000140008740 f i MessageHistory.obj
 0001:00007740       ?_Getal@?$basic_string@DU?$char_traits@D@std@@V?$allocator@D@2@@std@@AEBAAEBV?$allocator@D@2@XZ 0000000140008740 f i MessageHistory.obj
 0001:00007740       ?_Getal@?$list@V?$basic_string@DU?$char_traits@D@std@@V?$allocator@D@2@@std@@V?$allocator@V?$basic_string@DU?$char_traits@D@std@@V?$allocator@D@2@@std@@@2@@std@@AEAAAEAV?$allocator@U?$_List_node@V?$basic_string@DU?$char_traits@D@std@@V?$allocator@D@2@@std@@PEAX@std@@@2@XZ 0000000140008740 f i MessageHistory.obj
 0001:00007740       ?_Getal@?$list@V?$basic_string@DU?$char_traits@D@std@@V?$allocator@D@2@@std@@V?$allocator@V?$basic_string@DU?$char_traits@D@std@@V?$allocator@D@2@@std@@@2@@std@@AEBAAEBV?$allocator@U?$_List_node@V?$basic_string@DU?$char_traits@D@std@@V?$allocator@D@2@@std@@PEAX@std@@@2@XZ 0000000140008740 f i MessageHistory.obj
 0001:00007760       ?_Getcont@_Iterator_base0@std@@QEBAPEBU_Container_base0@2@XZ 0000000140008760 f i MessageHistory.obj
 0001:00007770       ?_Large_string_engaged@?$_String_val@U?$_Simple_types@D@std@@@std@@QEBA_NXZ 0000000140008770 f i MessageHistory.obj
 0001:000077a0       ?_Memcpy_val_from@?$basic_string@DU?$char_traits@D@std@@V?$allocator@D@2@@std@@AEAAXAEBV12@@Z 00000001400087a0 f i MessageHistory.obj
 0001:000077f0       ?_Myptr@?$_String_val@U?$_Simple_types@D@std@@@std@@QEBAPEBDXZ 00000001400087f0 f i MessageHistory.obj
 0001:00007830       ?_Seek_to@?$_List_const_iterator@V?$_List_val@U?$_List_simple_types@V?$basic_string@DU?$char_traits@D@std@@V?$allocator@D@2@@std@@@std@@@std@@@std@@QEAAXV?$_List_unchecked_const_iterator@V?$_List_val@U?$_List_simple_types@V?$basic_string@DU?$char_traits@D@std@@V?$allocator@D@2@@std@@@std@@@std@@U_Iterator_base0@2@@2@@Z 0000000140008830 f i MessageHistory.obj
 0001:00007850       ?_Swap_proxy_and_iterators@?$basic_string@DU?$char_traits@D@std@@V?$allocator@D@2@@std@@AEAAXAEAV12@@Z 0000000140008850 f i MessageHistory.obj
 0001:00007880       ?_Take_contents@?$basic_string@DU?$char_traits@D@std@@V?$allocator@D@2@@std@@AEAAXAEAV12@@Z 0000000140008880 f i MessageHistory.obj
 0001:00007980       ?_Throw_bad_array_new_length@std@@YAXXZ 0000000140008980 f i MessageHistory.obj
 0001:000079b0       ?_Tidy_deallocate@?$basic_string@DU?$char_traits@D@std@@V?$allocator@D@2@@std@@AEAAXXZ 00000001400089b0 f i MessageHistory.obj
 0001:00007a80       ?_Tidy_init@?$basic_string@DU?$char_traits@D@std@@V?$allocator@D@2@@std@@AEAAXXZ 0000000140008a80 f i MessageHistory.obj
 0001:00007af0       ?_Transfer_before@?$_List_node_emplace_op2@V?$allocator@U?$_List_node@V?$basic_string@DU?$char_traits@D@std@@V?$allocator@D@2@@std@@PEAX@std@@@std@@@std@@QEAAPEAU?$_List_node@V?$basic_string@DU?$char_traits@D@std@@V?$allocator@D@2@@std@@PEAX@2@QEAU32@@Z 0000000140008af0 f i MessageHistory.obj
 0001:00007b80       ?_Unchecked_erase@?$list@V?$basic_string@DU?$char_traits@D@std@@V?$allocator@D@2@@std@@V?$allocator@V?$basic_string@DU?$char_traits@D@std@@V?$allocator@D@2@@std@@@2@@std@@AEAAPEAU?$_List_node@V?$basic_string@DU?$char_traits@D@std@@V?$allocator@D@2@@std@@PEAX@2@QEAU32@@Z 0000000140008b80 f i MessageHistory.obj
 0001:00007c10       ?_Unwrapped@?$_List_const_iterator@V?$_List_val@U?$_List_simple_types@V?$basic_string@DU?$char_traits@D@std@@V?$allocator@D@2@@std@@@std@@@std@@@std@@QEBA?AV?$_List_unchecked_const_iterator@V?$_List_val@U?$_List_simple_types@V?$basic_string@DU?$char_traits@D@std@@V?$allocator@D@2@@std@@@std@@@std@@U_Iterator_base0@2@@2@XZ 0000000140008c10 f i MessageHistory.obj
 0001:00007c50       ?_Xlen_string@std@@YAXXZ   0000000140008c50 f i MessageHistory.obj
 0001:00007c70       ?allocate@?$allocator@D@std@@QEAAPEAD_K@Z 0000000140008c70 f i MessageHistory.obj
 0001:00007ca0       ?allocate@?$allocator@U?$_List_node@V?$basic_string@DU?$char_traits@D@std@@V?$allocator@D@2@@std@@PEAX@std@@@std@@QEAAPEAU?$_List_node@V?$basic_string@DU?$char_traits@D@std@@V?$allocator@D@2@@std@@PEAX@2@_K@Z 0000000140008ca0 f i MessageHistory.obj
 0001:00007cd0       ?assign@?$_Narrow_char_traits@DH@std@@SAXAEADAEBD@Z 0000000140008cd0 f i MessageHistory.obj
 0001:00007cf0       ?begin@?$list@V?$basic_string@DU?$char_traits@D@std@@V?$allocator@D@2@@std@@V?$allocator@V?$basic_string@DU?$char_traits@D@std@@V?$allocator@D@2@@std@@@2@@std@@QEAA?AV?$_List_iterator@V?$_List_val@U?$_List_simple_types@V?$basic_string@DU?$char_traits@D@std@@V?$allocator@D@2@@std@@@std@@@std@@@2@XZ 0000000140008cf0 f i MessageHistory.obj
 0001:00007d30       ?c_str@?$basic_string@DU?$char_traits@D@std@@V?$allocator@D@2@@std@@QEBAPEBDXZ 0000000140008d30 f i MessageHistory.obj
 0001:00007d50       ?clear@?$list@V?$basic_string@DU?$char_traits@D@std@@V?$allocator@D@2@@std@@V?$allocator@V?$basic_string@DU?$char_traits@D@std@@V?$allocator@D@2@@std@@@2@@std@@QEAAXXZ 0000000140008d50 f i MessageHistory.obj
 0001:00007dc0       ?copy@?$_Char_traits@DH@std@@SAPEADQEADQEBD_K@Z 0000000140008dc0 f i MessageHistory.obj
 0001:00007e00       ?deallocate@?$_Default_allocator_traits@V?$allocator@U?$_List_node@V?$basic_string@DU?$char_traits@D@std@@V?$allocator@D@2@@std@@PEAX@std@@@std@@@std@@SAXAEAV?$allocator@U?$_List_node@V?$basic_string@DU?$char_traits@D@std@@V?$allocator@D@2@@std@@PEAX@std@@@2@QEAU?$_List_node@V?$basic_string@DU?$char_traits@D@std@@V?$allocator@D@2@@std@@PEAX@2@_K@Z 0000000140008e00 f i MessageHistory.obj
 0001:00007e00       ?deallocate@?$allocator@U?$_List_node@V?$basic_string@DU?$char_traits@D@std@@V?$allocator@D@2@@std@@PEAX@std@@@std@@QEAAXQEAU?$_List_node@V?$basic_string@DU?$char_traits@D@std@@V?$allocator@D@2@@std@@PEAX@2@_K@Z 0000000140008e00 f i MessageHistory.obj
 0001:00007e30       ?deallocate@?$allocator@D@std@@QEAAXQEAD_K@Z 0000000140008e30 f i MessageHistory.obj
 0001:00007e60       ?empty@?$list@V?$basic_string@DU?$char_traits@D@std@@V?$allocator@D@2@@std@@V?$allocator@V?$basic_string@DU?$char_traits@D@std@@V?$allocator@D@2@@std@@@2@@std@@QEBA_NXZ 0000000140008e60 f i MessageHistory.obj
 0001:00007e90       ?end@?$list@V?$basic_string@DU?$char_traits@D@std@@V?$allocator@D@2@@std@@V?$allocator@V?$basic_string@DU?$char_traits@D@std@@V?$allocator@D@2@@std@@@2@@std@@QEAA?AV?$_List_iterator@V?$_List_val@U?$_List_simple_types@V?$basic_string@DU?$char_traits@D@std@@V?$allocator@D@2@@std@@@std@@@std@@@2@XZ 0000000140008e90 f i MessageHistory.obj
 0001:00007ed0       ?length@?$_Narrow_char_traits@DH@std@@SA_KQEBD@Z 0000000140008ed0 f i MessageHistory.obj
 0001:00007ef0       ?max@?$numeric_limits@_J@std@@SA_JXZ 0000000140008ef0 f i MessageHistory.obj
 0001:00007f00       ?max_size@?$_Default_allocator_traits@V?$allocator@D@std@@@std@@SA_KAEBV?$allocator@D@2@@Z 0000000140008f00 f i MessageHistory.obj
 0001:00007f10       ?max_size@?$_Default_allocator_traits@V?$allocator@U?$_List_node@V?$basic_string@DU?$char_traits@D@std@@V?$allocator@D@2@@std@@PEAX@std@@@std@@@std@@SA_KAEBV?$allocator@U?$_List_node@V?$basic_string@DU?$char_traits@D@std@@V?$allocator@D@2@@std@@PEAX@std@@@2@@Z 0000000140008f10 f i MessageHistory.obj
 0001:00007f20       ?max_size@?$basic_string@DU?$char_traits@D@std@@V?$allocator@D@2@@std@@QEBA_KXZ 0000000140008f20 f i MessageHistory.obj
 0001:00007f90       ?max_size@?$list@V?$basic_string@DU?$char_traits@D@std@@V?$allocator@D@2@@std@@V?$allocator@V?$basic_string@DU?$char_traits@D@std@@V?$allocator@D@2@@std@@@2@@std@@QEBA_KXZ 0000000140008f90 f i MessageHistory.obj
 0001:00007fe0       ?pop_front@?$list@V?$basic_string@DU?$char_traits@D@std@@V?$allocator@D@2@@std@@V?$allocator@V?$basic_string@DU?$char_traits@D@std@@V?$allocator@D@2@@std@@@2@@std@@QEAAXXZ 0000000140008fe0 f i MessageHistory.obj
 0001:00008010       ?push_back@?$list@V?$basic_string@DU?$char_traits@D@std@@V?$allocator@D@2@@std@@V?$allocator@V?$basic_string@DU?$char_traits@D@std@@V?$allocator@D@2@@std@@@2@@std@@QEAAX$$QEAV?$basic_string@DU?$char_traits@D@std@@V?$allocator@D@2@@2@@Z 0000000140009010 f i MessageHistory.obj
 0001:00008050       ?size@?$list@V?$basic_string@DU?$char_traits@D@std@@V?$allocator@D@2@@std@@V?$allocator@V?$basic_string@DU?$char_traits@D@std@@V?$allocator@D@2@@std@@@2@@std@@QEBA_KXZ 0000000140009050 f i MessageHistory.obj
 0001:00008060       ?what@exception@std@@UEBAPEBDXZ 0000000140009060 f i MessageHistory.obj
 0001:000080a0       WinMain                    00000001400090a0 f   jaccessinspector.obj
 0001:00008220       ?TimerProc@@YAXPEAUHWND__@@IIK@Z 0000000140009220 f   jaccessinspector.obj
 0001:00008280       ?KeyboardProc@@YA_JH_K_J@Z 0000000140009280 f   jaccessinspector.obj
 0001:00008340       ?MouseProc@@YA_JH_K_J@Z    0000000140009340 f   jaccessinspector.obj
 0001:000083c0       ?InitWindow@@YAHPEAX@Z     00000001400093c0 f   jaccessinspector.obj
 0001:00008490       ?jaccessinspectorDialogProc@@YA_JPEAUHWND__@@I_K_J@Z 0000000140009490 f   jaccessinspector.obj
 0001:0000a100       ?HandleJavaShutdown@@YAXJ@Z 000000014000b100 f   jaccessinspector.obj
 0001:0000a190       ?HandleJavaFocusGained@@YAXJ_J0@Z 000000014000b190 f   jaccessinspector.obj
 0001:0000a240       ?HandleJavaFocusLost@@YAXJ_J0@Z 000000014000b240 f   jaccessinspector.obj
 0001:0000a2f0       ?HandleJavaCaretUpdate@@YAXJ_J0@Z 000000014000b2f0 f   jaccessinspector.obj
 0001:0000a350       ?HandleMouseClicked@@YAXJ_J0@Z 000000014000b350 f   jaccessinspector.obj
 0001:0000a3b0       ?HandleMouseEntered@@YAXJ_J0@Z 000000014000b3b0 f   jaccessinspector.obj
 0001:0000a410       ?HandleMouseExited@@YAXJ_J0@Z 000000014000b410 f   jaccessinspector.obj
 0001:0000a470       ?HandleMousePressed@@YAXJ_J0@Z 000000014000b470 f   jaccessinspector.obj
 0001:0000a4d0       ?HandleMouseReleased@@YAXJ_J0@Z 000000014000b4d0 f   jaccessinspector.obj
 0001:0000a530       ?HandleMenuCanceled@@YAXJ_J0@Z 000000014000b530 f   jaccessinspector.obj
 0001:0000a590       ?HandleMenuDeselected@@YAXJ_J0@Z 000000014000b590 f   jaccessinspector.obj
 0001:0000a5f0       ?HandleMenuSelected@@YAXJ_J0@Z 000000014000b5f0 f   jaccessinspector.obj
 0001:0000a650       ?HandlePopupMenuCanceled@@YAXJ_J0@Z 000000014000b650 f   jaccessinspector.obj
 0001:0000a6b0       ?HandlePopupMenuWillBecomeInvisible@@YAXJ_J0@Z 000000014000b6b0 f   jaccessinspector.obj
 0001:0000a710       ?HandlePopupMenuWillBecomeVisible@@YAXJ_J0@Z 000000014000b710 f   jaccessinspector.obj
 0001:0000a770       ?HandlePropertyNameChange@@YAXJ_J0PEAG1@Z 000000014000b770 f   jaccessinspector.obj
 0001:0000a830       ?HandlePropertyDescriptionChange@@YAXJ_J0PEAG1@Z 000000014000b830 f   jaccessinspector.obj
 0001:0000a8f0       ?HandlePropertyStateChange@@YAXJ_J0PEAG1@Z 000000014000b8f0 f   jaccessinspector.obj
 0001:0000a9b0       ?HandlePropertyValueChange@@YAXJ_J0PEAG1@Z 000000014000b9b0 f   jaccessinspector.obj
 0001:0000aa70       ?HandlePropertySelectionChange@@YAXJ_J0@Z 000000014000ba70 f   jaccessinspector.obj
 0001:0000aad0       ?HandlePropertyTextChange@@YAXJ_J0@Z 000000014000bad0 f   jaccessinspector.obj
 0001:0000ab30       ?HandlePropertyCaretChange@@YAXJ_J0HH@Z 000000014000bb30 f   jaccessinspector.obj
 0001:0000abf0       ?HandlePropertyVisibleDataChange@@YAXJ_J0@Z 000000014000bbf0 f   jaccessinspector.obj
 0001:0000ac50       ?HandlePropertyTableModelChange@@YAXJ_J0PEAG1@Z 000000014000bc50 f   jaccessinspector.obj
 0001:0000ad10       ?SaveActiveEventOptionsToRegistry@@YAHXZ 000000014000bd10 f   jaccessinspector.obj
 0001:0000b4c0       ?ReadActiveEventOptionsFromRegistry@@YAHXZ 000000014000c4c0 f   jaccessinspector.obj
 0001:0000c180       ?ApplyEventOptions@@YAXPEAUHWND__@@@Z 000000014000d180 f   jaccessinspector.obj
 0001:0000c8f0       ?EnableDlgItem@@YAHPEAUHWND__@@HH@Z 000000014000d8f0 f   jaccessinspector.obj
 0001:0000c940       ?EnableMessageNavButtons@@YAXXZ 000000014000d940 f   jaccessinspector.obj
 0001:0000cbd0       ?AddToMessageHistory@@YAXPEBD@Z 000000014000dbd0 f   jaccessinspector.obj
 0001:0000cc00       ?UpdateMessageNumber@@YAHXZ 000000014000dc00 f   jaccessinspector.obj
 0001:0000ccd0       ?GoToMessageDialogProc@@YA_JPEAUHWND__@@I_K_J@Z 000000014000dcd0 f   jaccessinspector.obj
 0001:0000d090       ?InitGoToMessageDialogBox@@YAHPEAX@Z 000000014000e090 f   jaccessinspector.obj
 0001:0000d100       ?ShouldCheckMonitorTheSameEventsAsJAWS@@YAHXZ 000000014000e100 f   jaccessinspector.obj
 0001:0000d230       ?MaybeCheckMonitorTheSameEventsAsJAWS@@YAXPEAUHMENU__@@@Z 000000014000e230 f   jaccessinspector.obj
 0001:0000d280       ?ShouldCheckMonitorAllEvents@@YAHXZ 000000014000e280 f   jaccessinspector.obj
 0001:0000d3b0       ?MaybeCheckMonitorAllEvents@@YAXPEAUHMENU__@@@Z 000000014000e3b0 f   jaccessinspector.obj
 0001:0000d400       ?displayAccessibleInfo@@YAXJ_JHH@Z 000000014000e400 f   jaccessinspector.obj
 0001:0000d4b0       ?displayJavaEvent@@YAXJ_JPEAD@Z 000000014000e4b0 f   jaccessinspector.obj
 0001:0000d590       ?displayAccessiblePropertyChange@@YAXJ_JPEBD@Z 000000014000e590 f   jaccessinspector.obj
 0001:0000d670       ?echoMouseObject@@YAXXZ    000000014000e670 f   jaccessinspector.obj
 0001:0000d730       ?echoMouseHWNDObject@@YAXXZ 000000014000e730 f   jaccessinspector.obj
 0001:0000d7a0       ?displayFocusedObject@@YAXXZ 000000014000e7a0 f   jaccessinspector.obj
 0001:0000d830       ?HandlePropertyChildChange@@YAXJ_J000@Z 000000014000e830 f   jaccessinspector.obj
 0001:0000da30       ?HandlePropertyActiveDescendentChange@@YAXJ_J000@Z 000000014000ea30 f   jaccessinspector.obj
 0001:0000db10       ?exitjaccessinspector@@YAXPEAUHWND__@@@Z 000000014000eb10 f   jaccessinspector.obj
 0001:0000db40       ?reinstallEventListeners@@YAXXZ 000000014000eb40 f   jaccessinspector.obj
 0001:0000dd70       ??$?0$$V@?$_Compressed_pair@V?$allocator@U?$_List_node@V?$basic_string@DU?$char_traits@D@std@@V?$allocator@D@2@@std@@PEAX@std@@@std@@V?$_List_val@U?$_List_simple_types@V?$basic_string@DU?$char_traits@D@std@@V?$allocator@D@2@@std@@@std@@@2@$00@std@@QEAA@U_Zero_then_variadic_args_t@1@@Z 000000014000ed70 f i jaccessinspector.obj
 0001:0000dda0       ??0?$_List_const_iterator@V?$_List_val@U?$_List_simple_types@V?$basic_string@DU?$char_traits@D@std@@V?$allocator@D@2@@std@@@std@@@std@@@std@@QEAA@XZ 000000014000eda0 f i jaccessinspector.obj
 0001:0000ddc0       ??0?$_List_unchecked_const_iterator@V?$_List_val@U?$_List_simple_types@V?$basic_string@DU?$char_traits@D@std@@V?$allocator@D@2@@std@@@std@@@std@@U_Iterator_base0@2@@std@@QEAA@XZ 000000014000edc0 f i jaccessinspector.obj
 0001:0000dde0       ??0?$_List_val@U?$_List_simple_types@V?$basic_string@DU?$char_traits@D@std@@V?$allocator@D@2@@std@@@std@@@std@@QEAA@XZ 000000014000ede0 f i jaccessinspector.obj
 0001:0000de10       ??0?$list@V?$basic_string@DU?$char_traits@D@std@@V?$allocator@D@2@@std@@V?$allocator@V?$basic_string@DU?$char_traits@D@std@@V?$allocator@D@2@@std@@@2@@std@@QEAA@XZ 000000014000ee10 f i jaccessinspector.obj
 0001:0000de40       ??0MessageHistory@@QEAA@XZ 000000014000ee40 f i jaccessinspector.obj
 0001:0000de80       ??1?$list@V?$basic_string@DU?$char_traits@D@std@@V?$allocator@D@2@@std@@V?$allocator@V?$basic_string@DU?$char_traits@D@std@@V?$allocator@D@2@@std@@@2@@std@@QEAA@XZ 000000014000ee80 f i jaccessinspector.obj
 0001:0000dea0       ??1MessageHistory@@QEAA@XZ 000000014000eea0 f i jaccessinspector.obj
 0001:0000dec0       ?_Alloc_sentinel_and_proxy@?$list@V?$basic_string@DU?$char_traits@D@std@@V?$allocator@D@2@@std@@V?$allocator@V?$basic_string@DU?$char_traits@D@std@@V?$allocator@D@2@@std@@@2@@std@@AEAAXXZ 000000014000eec0 f i jaccessinspector.obj
 0001:0000df60       ?_Tidy@?$list@V?$basic_string@DU?$char_traits@D@std@@V?$allocator@D@2@@std@@V?$allocator@V?$basic_string@DU?$char_traits@D@std@@V?$allocator@D@2@@std@@@2@@std@@AEAAXXZ 000000014000ef60 f i jaccessinspector.obj
 0001:0000dfc0       _snprintf                  000000014000efc0 f i jaccessinspector.obj
 0001:0000e020       _vsnprintf                 000000014000f020 f i jaccessinspector.obj
 0001:0000e060       _vsnprintf_l               000000014000f060 f i jaccessinspector.obj
 0001:0000e0d8       ??_U@YAPEAX_K@Z            000000014000f0d8 f   MSVCRT:new_array.obj
 0001:0000e0e0       ??3@YAXPEAX_K@Z            000000014000f0e0 f   MSVCRT:delete_scalar_size.obj
 0001:0000e0e0       ??_V@YAXPEAX@Z             000000014000f0e0 f   MSVCRT:delete_array.obj
 0001:0000e0e8       __raise_securityfailure    000000014000f0e8 f   MSVCRT:gs_report.obj
 0001:0000e11c       __report_gsfailure         000000014000f11c f   MSVCRT:gs_report.obj
 0001:0000e1f0       __report_rangecheckfailure 000000014000f1f0 f   MSVCRT:gs_report.obj
 0001:0000e204       __report_securityfailure   000000014000f204 f   MSVCRT:gs_report.obj
 0001:0000e384       __GSHandlerCheck           000000014000f384 f   MSVCRT:gshandler.obj
 0001:0000e3a4       __GSHandlerCheckCommon     000000014000f3a4 f   MSVCRT:gshandler.obj
 0001:0000e410       __chkstk                   000000014000f410 f   MSVCRT:chkstk.obj
 0001:0000e410       _alloca_probe              000000014000f410 f   MSVCRT:chkstk.obj
 0001:0000e470       __security_check_cookie    000000014000f470 f   MSVCRT:amdsecgs.obj
 0001:0000e490       ??2@YAPEAX_K@Z             000000014000f490 f   MSVCRT:new_scalar.obj
 0001:0000e4cc       __GSHandlerCheck_EH4       000000014000f4cc f   MSVCRT:gshandlereh4.obj
 0001:0000e54c       ??_Etype_info@@UEAAPEAXI@Z 000000014000f54c f i MSVCRT:std_type_info_static.obj
 0001:0000e54c       ??_Gtype_info@@UEAAPEAXI@Z 000000014000f54c f i MSVCRT:std_type_info_static.obj
 0001:0000e578       __scrt_acquire_startup_lock 000000014000f578 f   MSVCRT:utility.obj
 0001:0000e5b4       __scrt_initialize_crt      000000014000f5b4 f   MSVCRT:utility.obj
 0001:0000e600       __scrt_initialize_onexit_tables 000000014000f600 f   MSVCRT:utility.obj
 0001:0000e68c       __scrt_is_nonwritable_in_current_image 000000014000f68c f   MSVCRT:utility.obj
 0001:0000e724       __scrt_release_startup_lock 000000014000f724 f   MSVCRT:utility.obj
 0001:0000e748       __scrt_uninitialize_crt    000000014000f748 f   MSVCRT:utility.obj
 0001:0000e774       _onexit                    000000014000f774 f   MSVCRT:utility.obj
 0001:0000e7b0       atexit                     000000014000f7b0 f   MSVCRT:utility.obj
 0001:0000e7c8       _Init_thread_footer        000000014000f7c8 f   MSVCRT:thread_safe_statics.obj
 0001:0000e834       _Init_thread_header        000000014000f834 f   MSVCRT:thread_safe_statics.obj
 0001:0000eb04       WinMainCRTStartup          000000014000fb04 f   MSVCRT:exe_winmain.obj
 0001:0000eb18       ??3@YAXPEAX@Z              000000014000fb18 f   MSVCRT:delete_scalar.obj
 0001:0000eb20       ??0bad_alloc@std@@QEAA@XZ  000000014000fb20 f i MSVCRT:throw_bad_alloc.obj
 0001:0000eb40       ?__scrt_throw_std_bad_alloc@@YAXXZ 000000014000fb40 f   MSVCRT:throw_bad_alloc.obj
 0001:0000eb60       ?__scrt_throw_std_bad_array_new_length@@YAXXZ 000000014000fb60 f   MSVCRT:throw_bad_alloc.obj
 0001:0000eb80       __isa_available_init       000000014000fb80 f   MSVCRT:cpu_disp.obj
 0001:0000ed2c       _get_startup_argv_mode     000000014000fd2c f   MSVCRT:argv_mode.obj
 0001:0000ed34       __scrt_is_ucrt_dll_in_use  000000014000fd34 f   MSVCRT:ucrt_detection.obj
 0001:0000ed40       __crt_debugger_hook        000000014000fd40 f   MSVCRT:utility_desktop.obj
 0001:0000ed48       __scrt_fastfail            000000014000fd48 f   MSVCRT:utility_desktop.obj
 0001:0000ee94       __scrt_get_show_window_mode 000000014000fe94 f   MSVCRT:utility_desktop.obj
 0001:0000eed0       __scrt_initialize_mta      000000014000fed0 f   MSVCRT:utility_desktop.obj
 0001:0000eed8       __scrt_exe_initialize_mta  000000014000fed8 f   MSVCRT:utility_desktop.obj
 0001:0000eed8       __scrt_initialize_winrt    000000014000fed8 f   MSVCRT:utility_desktop.obj
 0001:0000eed8       __scrt_stub_for_initialize_mta 000000014000fed8 f   MSVCRT:utility_desktop.obj
 0001:0000eed8       _get_startup_commit_mode   000000014000fed8 f   MSVCRT:commit_mode.obj
 0001:0000eed8       _get_startup_new_mode      000000014000fed8 f   MSVCRT:new_mode.obj
 0001:0000eed8       _get_startup_thread_locale_mode 000000014000fed8 f   MSVCRT:thread_locale.obj
 0001:0000eed8       _matherr                   000000014000fed8 f   MSVCRT:matherr.obj
 0001:0000eedc       __scrt_is_managed_app      000000014000fedc f   MSVCRT:utility_desktop.obj
 0001:0000ef30       __scrt_set_unhandled_exception_filter 000000014000ff30 f   MSVCRT:utility_desktop.obj
 0001:0000ef40       __scrt_unhandled_exception_filter 000000014000ff40 f   MSVCRT:utility_desktop.obj
 0001:0000ef9c       _guard_check_icall_nop     000000014000ff9c f i MSVCRT:guard_support.obj
 0001:0000ef9c       _initialize_denormal_control 000000014000ff9c f i MSVCRT:denormal_control.obj
 0001:0000ef9c       _initialize_invalid_parameter_handler 000000014000ff9c f i MSVCRT:invalid_parameter_handler.obj
 0001:0000efa0       __security_init_cookie     000000014000ffa0 f   MSVCRT:gs_support.obj
 0001:0000f04c       _get_startup_file_mode     000000014001004c f   MSVCRT:file_mode.obj
 0001:0000f054       ?__scrt_initialize_type_info@@YAXXZ 0000000140010054 f   MSVCRT:tncleanup.obj
 0001:0000f064       __acrt_initialize          0000000140010064 f   MSVCRT:ucrt_stubs.obj
 0001:0000f064       __acrt_uninitialize        0000000140010064 f   MSVCRT:ucrt_stubs.obj
 0001:0000f064       __scrt_stub_for_acrt_initialize 0000000140010064 f   MSVCRT:ucrt_stubs.obj
 0001:0000f064       __scrt_stub_for_acrt_uninitialize 0000000140010064 f   MSVCRT:ucrt_stubs.obj
 0001:0000f064       __vcrt_initialize          0000000140010064 f   MSVCRT:ucrt_stubs.obj
 0001:0000f064       __vcrt_uninitialize        0000000140010064 f   MSVCRT:ucrt_stubs.obj
 0001:0000f064       _should_initialize_environment 0000000140010064 f   MSVCRT:env_mode.obj
 0001:0000f068       __local_stdio_scanf_options 0000000140010068 f i MSVCRT:default_local_stdio_options.obj
 0001:0000f070       __scrt_initialize_default_local_stdio_options 0000000140010070 f   MSVCRT:default_local_stdio_options.obj
 0001:0000f08c       __scrt_is_user_matherr_present 000000014001008c f   MSVCRT:matherr_detection.obj
 0001:0000f098       __scrt_get_dyn_tls_init_callback 0000000140010098 f   MSVCRT:dyn_tls_init.obj
 0001:0000f0a0       __scrt_get_dyn_tls_dtor_callback 00000001400100a0 f   MSVCRT:dyn_tls_dtor.obj
 0001:0000f0a8       _RTC_Initialize            00000001400100a8 f   MSVCRT:initsect.obj
 0001:0000f0e4       _RTC_Terminate             00000001400100e4 f   MSVCRT:initsect.obj
 0001:0000f120       ?_Xlength_error@std@@YAXPEBD@Z 0000000140010120 f   msvcprt:MSVCP140.dll
 0001:0000f126       memcpy                     0000000140010126 f   vcruntime:VCRUNTIME140.dll
 0001:0000f12c       memset                     000000014001012c f   vcruntime:VCRUNTIME140.dll
 0001:0000f132       __std_exception_copy       0000000140010132 f   vcruntime:VCRUNTIME140.dll
 0001:0000f138       __std_exception_destroy    0000000140010138 f   vcruntime:VCRUNTIME140.dll
 0001:0000f13e       _CxxThrowException         000000014001013e f   vcruntime:VCRUNTIME140.dll
 0001:0000f144       __CxxFrameHandler4         0000000140010144 f   vcruntime:VCRUNTIME140_1.dll
 0001:0000f14a       __C_specific_handler       000000014001014a f   vcruntime:VCRUNTIME140.dll
 0001:0000f150       __current_exception        0000000140010150 f   vcruntime:VCRUNTIME140.dll
 0001:0000f156       __current_exception_context 0000000140010156 f   vcruntime:VCRUNTIME140.dll
 0001:0000f15c       strlen                     000000014001015c f   ucrt:api-ms-win-crt-string-l1-1-0.dll
 0001:0000f162       strcpy                     0000000140010162 f   ucrt:api-ms-win-crt-string-l1-1-0.dll
 0001:0000f168       _callnewh                  0000000140010168 f   ucrt:api-ms-win-crt-heap-l1-1-0.dll
 0001:0000f16e       malloc                     000000014001016e f   ucrt:api-ms-win-crt-heap-l1-1-0.dll
 0001:0000f174       _configure_narrow_argv     0000000140010174 f   ucrt:api-ms-win-crt-runtime-l1-1-0.dll
 0001:0000f17a       _initialize_narrow_environment 000000014001017a f   ucrt:api-ms-win-crt-runtime-l1-1-0.dll
 0001:0000f180       _initialize_onexit_table   0000000140010180 f   ucrt:api-ms-win-crt-runtime-l1-1-0.dll
 0001:0000f186       _register_onexit_function  0000000140010186 f   ucrt:api-ms-win-crt-runtime-l1-1-0.dll
 0001:0000f18c       _crt_atexit                000000014001018c f   ucrt:api-ms-win-crt-runtime-l1-1-0.dll
 0001:0000f192       _cexit                     0000000140010192 f   ucrt:api-ms-win-crt-runtime-l1-1-0.dll
 0001:0000f198       _seh_filter_exe            0000000140010198 f   ucrt:api-ms-win-crt-runtime-l1-1-0.dll
 0001:0000f19e       _set_app_type              000000014001019e f   ucrt:api-ms-win-crt-runtime-l1-1-0.dll
 0001:0000f1a4       __setusermatherr           00000001400101a4 f   ucrt:api-ms-win-crt-math-l1-1-0.dll
 0001:0000f1aa       _get_narrow_winmain_command_line 00000001400101aa f   ucrt:api-ms-win-crt-runtime-l1-1-0.dll
 0001:0000f1b0       _initterm                  00000001400101b0 f   ucrt:api-ms-win-crt-runtime-l1-1-0.dll
 0001:0000f1b6       _initterm_e                00000001400101b6 f   ucrt:api-ms-win-crt-runtime-l1-1-0.dll
 0001:0000f1bc       exit                       00000001400101bc f   ucrt:api-ms-win-crt-runtime-l1-1-0.dll
 0001:0000f1c2       _exit                      00000001400101c2 f   ucrt:api-ms-win-crt-runtime-l1-1-0.dll
 0001:0000f1c8       _set_fmode                 00000001400101c8 f   ucrt:api-ms-win-crt-stdio-l1-1-0.dll
 0001:0000f1ce       _c_exit                    00000001400101ce f   ucrt:api-ms-win-crt-runtime-l1-1-0.dll
 0001:0000f1d4       _register_thread_local_exe_atexit_callback 00000001400101d4 f   ucrt:api-ms-win-crt-runtime-l1-1-0.dll
 0001:0000f1da       _configthreadlocale        00000001400101da f   ucrt:api-ms-win-crt-locale-l1-1-0.dll
 0001:0000f1e0       _set_new_mode              00000001400101e0 f   ucrt:api-ms-win-crt-heap-l1-1-0.dll
 0001:0000f1e6       __p__commode               00000001400101e6 f   ucrt:api-ms-win-crt-stdio-l1-1-0.dll
 0001:0000f1ec       free                       00000001400101ec f   ucrt:api-ms-win-crt-heap-l1-1-0.dll
 0001:0000f1f2       terminate                  00000001400101f2 f   ucrt:api-ms-win-crt-runtime-l1-1-0.dll
 0001:0000f210       _guard_dispatch_icall_nop  0000000140010210 f   MSVCRT:guard_dispatch.obj
 0001:0000f230       _guard_xfg_dispatch_icall_nop 0000000140010230 f   MSVCRT:guard_xfg_dispatch.obj
 0002:00000000       __imp_RegCreateKeyExA      0000000140011000     advapi32:ADVAPI32.dll
 0002:00000008       __imp_RegFlushKey          0000000140011008     advapi32:ADVAPI32.dll
 0002:00000010       __imp_RegOpenKeyExA        0000000140011010     advapi32:ADVAPI32.dll
 0002:00000018       __imp_RegQueryValueExA     0000000140011018     advapi32:ADVAPI32.dll
 0002:00000020       __imp_RegSetValueExA       0000000140011020     advapi32:ADVAPI32.dll
 0002:00000028       __imp_RegCloseKey          0000000140011028     advapi32:ADVAPI32.dll
 0002:00000030       \177ADVAPI32_NULL_THUNK_DATA 0000000140011030     advapi32:ADVAPI32.dll
 0002:00000038       __imp_InitializeSListHead  0000000140011038     kernel32:KERNEL32.dll
 0002:00000040       __imp_GetCurrentProcessId  0000000140011040     kernel32:KERNEL32.dll
 0002:00000048       __imp_QueryPerformanceCounter 0000000140011048     kernel32:KERNEL32.dll
 0002:00000050       __imp_GetModuleHandleW     0000000140011050     kernel32:KERNEL32.dll
 0002:00000058       __imp_GetStartupInfoW      0000000140011058     kernel32:KERNEL32.dll
 0002:00000060       __imp_IsDebuggerPresent    0000000140011060     kernel32:KERNEL32.dll
 0002:00000068       __imp_SleepConditionVariableSRW 0000000140011068     kernel32:KERNEL32.dll
 0002:00000070       __imp_WakeAllConditionVariable 0000000140011070     kernel32:KERNEL32.dll
 0002:00000078       __imp_AcquireSRWLockExclusive 0000000140011078     kernel32:KERNEL32.dll
 0002:00000080       __imp_ReleaseSRWLockExclusive 0000000140011080     kernel32:KERNEL32.dll
 0002:00000088       __imp_IsProcessorFeaturePresent 0000000140011088     kernel32:KERNEL32.dll
 0002:00000090       __imp_TerminateProcess     0000000140011090     kernel32:KERNEL32.dll
 0002:00000098       __imp_GetCurrentProcess    0000000140011098     kernel32:KERNEL32.dll
 0002:000000a0       __imp_SetUnhandledExceptionFilter 00000001400110a0     kernel32:KERNEL32.dll
 0002:000000a8       __imp_UnhandledExceptionFilter 00000001400110a8     kernel32:KERNEL32.dll
 0002:000000b0       __imp_RtlVirtualUnwind     00000001400110b0     kernel32:KERNEL32.dll
 0002:000000b8       __imp_RtlLookupFunctionEntry 00000001400110b8     kernel32:KERNEL32.dll
 0002:000000c0       __imp_RtlCaptureContext    00000001400110c0     kernel32:KERNEL32.dll
 0002:000000c8       __imp_GetCurrentThreadId   00000001400110c8     kernel32:KERNEL32.dll
 0002:000000d0       __imp_FormatMessageA       00000001400110d0     kernel32:KERNEL32.dll
 0002:000000d8       __imp_LocalFree            00000001400110d8     kernel32:KERNEL32.dll
 0002:000000e0       __imp_GetSystemTimeAsFileTime 00000001400110e0     kernel32:KERNEL32.dll
 0002:000000e8       __imp_LoadLibraryA         00000001400110e8     kernel32:KERNEL32.dll
 0002:000000f0       __imp_GetProcAddress       00000001400110f0     kernel32:KERNEL32.dll
 0002:000000f8       __imp_FreeLibrary          00000001400110f8     kernel32:KERNEL32.dll
 0002:00000100       __imp_GetLastError         0000000140011100     kernel32:KERNEL32.dll
 0002:00000108       \177KERNEL32_NULL_THUNK_DATA 0000000140011108     kernel32:KERNEL32.dll
 0002:00000110       __imp_?_Xlength_error@std@@YAXPEBD@Z 0000000140011110     msvcprt:MSVCP140.dll
 0002:00000118       \177MSVCP140_NULL_THUNK_DATA 0000000140011118     msvcprt:MSVCP140.dll
 0002:00000120       __imp_WindowFromPoint      0000000140011120     user32:USER32.dll
 0002:00000128       __imp_CopyRect             0000000140011128     user32:USER32.dll
 0002:00000130       __imp_OffsetRect           0000000140011130     user32:USER32.dll
 0002:00000138       __imp_GetDesktopWindow     0000000140011138     user32:USER32.dll
 0002:00000140       __imp_GetParent            0000000140011140     user32:USER32.dll
 0002:00000148       __imp_GetCursorPos         0000000140011148     user32:USER32.dll
 0002:00000150       __imp_GetWindow            0000000140011150     user32:USER32.dll
 0002:00000158       __imp_SetWindowsHookExA    0000000140011158     user32:USER32.dll
 0002:00000160       __imp_UnhookWindowsHookEx  0000000140011160     user32:USER32.dll
 0002:00000168       __imp_CallNextHookEx       0000000140011168     user32:USER32.dll
 0002:00000170       __imp_IsDialogMessageA     0000000140011170     user32:USER32.dll
 0002:00000178       __imp_RegisterWindowMessageA 0000000140011178     user32:USER32.dll
 0002:00000180       __imp_GetWindowRect        0000000140011180     user32:USER32.dll
 0002:00000188       __imp_GetTopWindow         0000000140011188     user32:USER32.dll
 0002:00000190       __imp_UpdateWindow         0000000140011190     user32:USER32.dll
 0002:00000198       __imp_CheckMenuItem        0000000140011198     user32:USER32.dll
 0002:000001a0       __imp_GetMenu              00000001400111a0     user32:USER32.dll
 0002:000001a8       __imp_GetSystemMetrics     00000001400111a8     user32:USER32.dll
 0002:000001b0       __imp_TranslateAcceleratorA 00000001400111b0     user32:USER32.dll
 0002:000001b8       __imp_LoadAcceleratorsA    00000001400111b8     user32:USER32.dll
 0002:000001c0       __imp_EnableWindow         00000001400111c0     user32:USER32.dll
 0002:000001c8       __imp_KillTimer            00000001400111c8     user32:USER32.dll
 0002:000001d0       __imp_SetTimer             00000001400111d0     user32:USER32.dll
 0002:000001d8       __imp_GetFocus             00000001400111d8     user32:USER32.dll
 0002:000001e0       __imp_SetFocus             00000001400111e0     user32:USER32.dll
 0002:000001e8       __imp_GetDlgCtrlID         00000001400111e8     user32:USER32.dll
 0002:000001f0       __imp_GetDlgItemInt        00000001400111f0     user32:USER32.dll
 0002:000001f8       __imp_GetDlgItem           00000001400111f8     user32:USER32.dll
 0002:00000200       __imp_EndDialog            0000000140011200     user32:USER32.dll
 0002:00000208       __imp_CreateDialogParamA   0000000140011208     user32:USER32.dll
 0002:00000210       __imp_SetWindowPos         0000000140011210     user32:USER32.dll
 0002:00000218       __imp_ShowWindow           0000000140011218     user32:USER32.dll
 0002:00000220       __imp_PostQuitMessage      0000000140011220     user32:USER32.dll
 0002:00000228       __imp_PostMessageA         0000000140011228     user32:USER32.dll
 0002:00000230       __imp_DispatchMessageA     0000000140011230     user32:USER32.dll
 0002:00000238       __imp_TranslateMessage     0000000140011238     user32:USER32.dll
 0002:00000240       __imp_GetMessageA          0000000140011240     user32:USER32.dll
 0002:00000248       __imp_wsprintfA            0000000140011248     user32:USER32.dll
 0002:00000250       __imp_SetDlgItemTextA      0000000140011250     user32:USER32.dll
 0002:00000258       __imp_SetWindowTextA       0000000140011258     user32:USER32.dll
 0002:00000260       \177USER32_NULL_THUNK_DATA 0000000140011260     user32:USER32.dll
 0002:00000268       __imp_memcpy               0000000140011268     vcruntime:VCRUNTIME140.dll
 0002:00000270       __imp_memset               0000000140011270     vcruntime:VCRUNTIME140.dll
 0002:00000278       __imp___std_exception_copy 0000000140011278     vcruntime:VCRUNTIME140.dll
 0002:00000280       __imp___std_exception_destroy 0000000140011280     vcruntime:VCRUNTIME140.dll
 0002:00000288       __imp__CxxThrowException   0000000140011288     vcruntime:VCRUNTIME140.dll
 0002:00000290       __imp___C_specific_handler 0000000140011290     vcruntime:VCRUNTIME140.dll
 0002:00000298       __imp___current_exception  0000000140011298     vcruntime:VCRUNTIME140.dll
 0002:000002a0       __imp___current_exception_context 00000001400112a0     vcruntime:VCRUNTIME140.dll
 0002:000002a8       \177VCRUNTIME140_NULL_THUNK_DATA 00000001400112a8     vcruntime:VCRUNTIME140.dll
 0002:000002b0       __imp___CxxFrameHandler4   00000001400112b0     vcruntime:VCRUNTIME140_1.dll
 0002:000002b8       \177VCRUNTIME140_1_NULL_THUNK_DATA 00000001400112b8     vcruntime:VCRUNTIME140_1.dll
 0002:000002c0       __imp_getenv               00000001400112c0     ucrt:api-ms-win-crt-environment-l1-1-0.dll
 0002:000002c8       \177api-ms-win-crt-environment-l1-1-0_NULL_THUNK_DATA 00000001400112c8     ucrt:api-ms-win-crt-environment-l1-1-0.dll
 0002:000002d0       __imp_malloc               00000001400112d0     ucrt:api-ms-win-crt-heap-l1-1-0.dll
 0002:000002d8       __imp__callnewh            00000001400112d8     ucrt:api-ms-win-crt-heap-l1-1-0.dll
 0002:000002e0       __imp__set_new_mode        00000001400112e0     ucrt:api-ms-win-crt-heap-l1-1-0.dll
 0002:000002e8       __imp_free                 00000001400112e8     ucrt:api-ms-win-crt-heap-l1-1-0.dll
 0002:000002f0       \177api-ms-win-crt-heap-l1-1-0_NULL_THUNK_DATA 00000001400112f0     ucrt:api-ms-win-crt-heap-l1-1-0.dll
 0002:000002f8       __imp__configthreadlocale  00000001400112f8     ucrt:api-ms-win-crt-locale-l1-1-0.dll
 0002:00000300       \177api-ms-win-crt-locale-l1-1-0_NULL_THUNK_DATA 0000000140011300     ucrt:api-ms-win-crt-locale-l1-1-0.dll
 0002:00000308       __imp___setusermatherr     0000000140011308     ucrt:api-ms-win-crt-math-l1-1-0.dll
 0002:00000310       \177api-ms-win-crt-math-l1-1-0_NULL_THUNK_DATA 0000000140011310     ucrt:api-ms-win-crt-math-l1-1-0.dll
 0002:00000318       __imp_terminate            0000000140011318     ucrt:api-ms-win-crt-runtime-l1-1-0.dll
 0002:00000320       __imp__register_thread_local_exe_atexit_callback 0000000140011320     ucrt:api-ms-win-crt-runtime-l1-1-0.dll
 0002:00000328       __imp__c_exit              0000000140011328     ucrt:api-ms-win-crt-runtime-l1-1-0.dll
 0002:00000330       __imp__exit                0000000140011330     ucrt:api-ms-win-crt-runtime-l1-1-0.dll
 0002:00000338       __imp__invalid_parameter_noinfo_noreturn 0000000140011338     ucrt:api-ms-win-crt-runtime-l1-1-0.dll
 0002:00000340       __imp_exit                 0000000140011340     ucrt:api-ms-win-crt-runtime-l1-1-0.dll
 0002:00000348       __imp__initterm_e          0000000140011348     ucrt:api-ms-win-crt-runtime-l1-1-0.dll
 0002:00000350       __imp__configure_narrow_argv 0000000140011350     ucrt:api-ms-win-crt-runtime-l1-1-0.dll
 0002:00000358       __imp__initialize_narrow_environment 0000000140011358     ucrt:api-ms-win-crt-runtime-l1-1-0.dll
 0002:00000360       __imp__initialize_onexit_table 0000000140011360     ucrt:api-ms-win-crt-runtime-l1-1-0.dll
 0002:00000368       __imp__register_onexit_function 0000000140011368     ucrt:api-ms-win-crt-runtime-l1-1-0.dll
 0002:00000370       __imp__initterm            0000000140011370     ucrt:api-ms-win-crt-runtime-l1-1-0.dll
 0002:00000378       __imp__cexit               0000000140011378     ucrt:api-ms-win-crt-runtime-l1-1-0.dll
 0002:00000380       __imp__seh_filter_exe      0000000140011380     ucrt:api-ms-win-crt-runtime-l1-1-0.dll
 0002:00000388       __imp__set_app_type        0000000140011388     ucrt:api-ms-win-crt-runtime-l1-1-0.dll
 0002:00000390       __imp__get_narrow_winmain_command_line 0000000140011390     ucrt:api-ms-win-crt-runtime-l1-1-0.dll
 0002:00000398       __imp__crt_atexit          0000000140011398     ucrt:api-ms-win-crt-runtime-l1-1-0.dll
 0002:000003a0       \177api-ms-win-crt-runtime-l1-1-0_NULL_THUNK_DATA 00000001400113a0     ucrt:api-ms-win-crt-runtime-l1-1-0.dll
 0002:000003a8       __imp___stdio_common_vfprintf 00000001400113a8     ucrt:api-ms-win-crt-stdio-l1-1-0.dll
 0002:000003b0       __imp_fflush               00000001400113b0     ucrt:api-ms-win-crt-stdio-l1-1-0.dll
 0002:000003b8       __imp__set_fmode           00000001400113b8     ucrt:api-ms-win-crt-stdio-l1-1-0.dll
 0002:000003c0       __imp___stdio_common_vsprintf 00000001400113c0     ucrt:api-ms-win-crt-stdio-l1-1-0.dll
 0002:000003c8       __imp_fopen                00000001400113c8     ucrt:api-ms-win-crt-stdio-l1-1-0.dll
 0002:000003d0       __imp_fclose               00000001400113d0     ucrt:api-ms-win-crt-stdio-l1-1-0.dll
 0002:000003d8       __imp___stdio_common_vfwprintf 00000001400113d8     ucrt:api-ms-win-crt-stdio-l1-1-0.dll
 0002:000003e0       __imp___acrt_iob_func      00000001400113e0     ucrt:api-ms-win-crt-stdio-l1-1-0.dll
 0002:000003e8       __imp___p__commode         00000001400113e8     ucrt:api-ms-win-crt-stdio-l1-1-0.dll
 0002:000003f0       \177api-ms-win-crt-stdio-l1-1-0_NULL_THUNK_DATA 00000001400113f0     ucrt:api-ms-win-crt-stdio-l1-1-0.dll
 0002:000003f8       __imp_strncat              00000001400113f8     ucrt:api-ms-win-crt-string-l1-1-0.dll
 0002:00000400       __imp_strlen               0000000140011400     ucrt:api-ms-win-crt-string-l1-1-0.dll
 0002:00000408       __imp_strncpy              0000000140011408     ucrt:api-ms-win-crt-string-l1-1-0.dll
 0002:00000410       __imp_strcpy               0000000140011410     ucrt:api-ms-win-crt-string-l1-1-0.dll
 0002:00000418       \177api-ms-win-crt-string-l1-1-0_NULL_THUNK_DATA 0000000140011418     ucrt:api-ms-win-crt-string-l1-1-0.dll
 0002:00000420       __imp__localtime64         0000000140011420     ucrt:api-ms-win-crt-time-l1-1-0.dll
 0002:00000428       __imp__time64              0000000140011428     ucrt:api-ms-win-crt-time-l1-1-0.dll
 0002:00000430       __imp_asctime              0000000140011430     ucrt:api-ms-win-crt-time-l1-1-0.dll
 0002:00000438       \177api-ms-win-crt-time-l1-1-0_NULL_THUNK_DATA 0000000140011438     ucrt:api-ms-win-crt-time-l1-1-0.dll
 0002:00000440       __guard_check_icall_fptr   0000000140011440     MSVCRT:guard_support.obj
 0002:00000448       __guard_xfg_check_icall_fptr 0000000140011448     MSVCRT:guard_support.obj
 0002:00000450       __guard_dispatch_icall_fptr 0000000140011450     MSVCRT:guard_support.obj
 0002:00000458       __guard_xfg_dispatch_icall_fptr 0000000140011458     MSVCRT:guard_support.obj
 0002:00000460       __guard_xfg_table_dispatch_icall_fptr 0000000140011460     MSVCRT:guard_support.obj
 0002:00000468       __castguard_check_failure_os_handled_fptr 0000000140011468     MSVCRT:guard_support.obj
 0002:00000470       __guard_memcpy_fptr        0000000140011470     vcruntime:softmemtag.obj
 0002:00000478       __xc_a                     0000000140011478     MSVCRT:initializers.obj
 0002:00000490       __xc_z                     0000000140011490     MSVCRT:initializers.obj
 0002:00000498       __xi_a                     0000000140011498     MSVCRT:initializers.obj
 0002:000004b0       __xi_z                     00000001400114b0     MSVCRT:initializers.obj
 0002:000004b8       __xl_a                     00000001400114b8     MSVCRT:tlssup.obj
 0002:000004c0       __xl_z                     00000001400114c0     MSVCRT:tlssup.obj
 0002:000004c8       __xp_a                     00000001400114c8     MSVCRT:initializers.obj
 0002:000004d0       __xp_z                     00000001400114d0     MSVCRT:initializers.obj
 0002:000004d8       __xt_a                     00000001400114d8     MSVCRT:initializers.obj
 0002:000004e0       __xt_z                     00000001400114e0     MSVCRT:initializers.obj
 0002:00001dc8       ??_7exception@std@@6B@     0000000140012dc8     MessageHistory.obj
 0002:00001dd8       ??_C@_0BC@EOODALEL@Unknown?5exception@ 0000000140012dd8     MessageHistory.obj
 0002:00001df8       ??_7bad_alloc@std@@6B@     0000000140012df8     MessageHistory.obj
 0002:00001e10       ??_7bad_array_new_length@std@@6B@ 0000000140012e10     MessageHistory.obj
 0002:00001e20       ??_C@_0BF@KINCDENJ@bad?5array?5new?5length@ 0000000140012e20     MessageHistory.obj
 0002:00001e38       ??_C@_0BA@JFNIOLAK@string?5too?5long@ 0000000140012e38     MessageHistory.obj
 0002:00001e48       ??_C@_0O@NKNMEGII@list?5too?5long@ 0000000140012e48     MessageHistory.obj
 0002:00002700       ??_7type_info@@6B@         0000000140013700     MSVCRT:std_type_info_static.obj
 0002:00002710       __xmm@ffffffffffffffffffffffffffffffff 0000000140013710     MSVCRT:utility.obj
 0002:00002720       ??_C@_0P@GHFPNOJB@bad?5allocation@ 0000000140013720     MSVCRT:throw_bad_alloc.obj
 0002:00002730       _load_config_used          0000000140013730     MSVCRT:loadcfg.obj
 0002:00002900       _tls_used                  0000000140013900     MSVCRT:tlssup.obj
 0002:00002928       ??_R4exception@std@@6B@    0000000140013928     MessageHistory.obj
 0002:00002950       ??_R3exception@std@@8      0000000140013950     MessageHistory.obj
 0002:00002968       ??_R2exception@std@@8      0000000140013968     MessageHistory.obj
 0002:00002978       ??_R1A@?0A@EA@exception@std@@8 0000000140013978     MessageHistory.obj
 0002:000029a0       ??_R4bad_alloc@std@@6B@    00000001400139a0     MessageHistory.obj
 0002:000029c8       ??_R3bad_alloc@std@@8      00000001400139c8     MessageHistory.obj
 0002:000029e0       ??_R2bad_alloc@std@@8      00000001400139e0     MessageHistory.obj
 0002:000029f8       ??_R1A@?0A@EA@bad_alloc@std@@8 00000001400139f8     MessageHistory.obj
 0002:00002a20       ??_R4bad_array_new_length@std@@6B@ 0000000140013a20     MessageHistory.obj
 0002:00002a48       ??_R3bad_array_new_length@std@@8 0000000140013a48     MessageHistory.obj
 0002:00002a60       ??_R2bad_array_new_length@std@@8 0000000140013a60     MessageHistory.obj
 0002:00002a80       ??_R1A@?0A@EA@bad_array_new_length@std@@8 0000000140013a80     MessageHistory.obj
 0002:00002aa8       ??_R4type_info@@6B@        0000000140013aa8     MSVCRT:std_type_info_static.obj
 0002:00002ad0       ??_R3type_info@@8          0000000140013ad0     MSVCRT:std_type_info_static.obj
 0002:00002ae8       ??_R2type_info@@8          0000000140013ae8     MSVCRT:std_type_info_static.obj
 0002:00002af8       ??_R1A@?0A@EA@type_info@@8 0000000140013af8     MSVCRT:std_type_info_static.obj
 0002:00002b1c       __volatile_metadata        0000000140013b1c     <linker-defined>
 0002:00003018       __rtc_iaa                  0000000140014018     MSVCRT:initsect.obj
 0002:00003020       __rtc_izz                  0000000140014020     MSVCRT:initsect.obj
 0002:00003028       __rtc_taa                  0000000140014028     MSVCRT:initsect.obj
 0002:00003030       __rtc_tzz                  0000000140014030     MSVCRT:initsect.obj
 0002:00003038       _tls_start                 0000000140014038     MSVCRT:tlssup.obj
 0002:0000303c       _Init_thread_epoch         000000014001403c     MSVCRT:thread_safe_statics.obj
 0002:00003040       _tls_end                   0000000140014040     MSVCRT:tlssup.obj
 0002:00003908       _TI3?AVbad_array_new_length@std@@ 0000000140014908     MessageHistory.obj
 0002:00003928       _CTA3?AVbad_array_new_length@std@@ 0000000140014928     MessageHistory.obj
 0002:00003948       _CT??_R0?AVbad_array_new_length@std@@@8??0bad_array_new_length@std@@QEAA@AEBV01@@Z24 0000000140014948     MessageHistory.obj
 0002:00003970       _CT??_R0?AVbad_alloc@std@@@8??0bad_alloc@std@@QEAA@AEBV01@@Z24 0000000140014970     MessageHistory.obj
 0002:00003998       _CT??_R0?AVexception@std@@@8??0exception@std@@QEAA@AEBV01@@Z24 0000000140014998     MessageHistory.obj
 0002:000039c0       _TI2?AVbad_alloc@std@@     00000001400149c0     MSVCRT:throw_bad_alloc.obj
 0002:000039e0       _CTA2?AVbad_alloc@std@@    00000001400149e0     MSVCRT:throw_bad_alloc.obj
 0002:000039f4       __IMPORT_DESCRIPTOR_ADVAPI32 00000001400149f4     advapi32:ADVAPI32.dll
 0002:00003a08       __IMPORT_DESCRIPTOR_USER32 0000000140014a08     user32:USER32.dll
 0002:00003a1c       __IMPORT_DESCRIPTOR_MSVCP140 0000000140014a1c     msvcprt:MSVCP140.dll
 0002:00003a30       __IMPORT_DESCRIPTOR_KERNEL32 0000000140014a30     kernel32:KERNEL32.dll
 0002:00003a44       __IMPORT_DESCRIPTOR_VCRUNTIME140 0000000140014a44     vcruntime:VCRUNTIME140.dll
 0002:00003a58       __IMPORT_DESCRIPTOR_VCRUNTIME140_1 0000000140014a58     vcruntime:VCRUNTIME140_1.dll
 0002:00003a6c       __IMPORT_DESCRIPTOR_api-ms-win-crt-string-l1-1-0 0000000140014a6c     ucrt:api-ms-win-crt-string-l1-1-0.dll
 0002:00003a80       __IMPORT_DESCRIPTOR_api-ms-win-crt-stdio-l1-1-0 0000000140014a80     ucrt:api-ms-win-crt-stdio-l1-1-0.dll
 0002:00003a94       __IMPORT_DESCRIPTOR_api-ms-win-crt-environment-l1-1-0 0000000140014a94     ucrt:api-ms-win-crt-environment-l1-1-0.dll
 0002:00003aa8       __IMPORT_DESCRIPTOR_api-ms-win-crt-time-l1-1-0 0000000140014aa8     ucrt:api-ms-win-crt-time-l1-1-0.dll
 0002:00003abc       __IMPORT_DESCRIPTOR_api-ms-win-crt-runtime-l1-1-0 0000000140014abc     ucrt:api-ms-win-crt-runtime-l1-1-0.dll
 0002:00003ad0       __IMPORT_DESCRIPTOR_api-ms-win-crt-heap-l1-1-0 0000000140014ad0     ucrt:api-ms-win-crt-heap-l1-1-0.dll
 0002:00003ae4       __IMPORT_DESCRIPTOR_api-ms-win-crt-math-l1-1-0 0000000140014ae4     ucrt:api-ms-win-crt-math-l1-1-0.dll
 0002:00003af8       __IMPORT_DESCRIPTOR_api-ms-win-crt-locale-l1-1-0 0000000140014af8     ucrt:api-ms-win-crt-locale-l1-1-0.dll
 0002:00003b0c       __NULL_IMPORT_DESCRIPTOR   0000000140014b0c     advapi32:ADVAPI32.dll
 0003:00000b30       ?sm_MaxMessages@MessageHistory@@2_KA 0000000140016b30     MessageHistory.obj
 0003:00000b38       ?szAppName@@3PADA          0000000140016b38     jaccessinspector.obj
 0003:00000b50       __security_cookie_complement 0000000140016b50     MSVCRT:gs_cookie.obj
 0003:00000b58       __security_cookie          0000000140016b58     MSVCRT:gs_cookie.obj
 0003:00000b60       _fltused                   0000000140016b60     MSVCRT:fltused.obj
 0003:00000b64       __scrt_native_dllmain_reason 0000000140016b64     MSVCRT:utility.obj
 0003:00000b68       _Init_global_epoch         0000000140016b68     MSVCRT:thread_safe_statics.obj
 0003:00000b70       __isa_available            0000000140016b70     MSVCRT:cpu_disp.obj
 0003:00000b74       __isa_enabled              0000000140016b74     MSVCRT:cpu_disp.obj
 0003:00000b78       __memset_fast_string_threshold 0000000140016b78     MSVCRT:cpu_disp.obj
 0003:00000b80       __memset_nt_threshold      0000000140016b80     MSVCRT:cpu_disp.obj
 0003:00000b88       __scrt_default_matherr     0000000140016b88     MSVCRT:matherr.obj
 0003:00000b90       __scrt_ucrt_dll_is_in_use  0000000140016b90     MSVCRT:ucrt_stubs.obj
 0003:00000b98       ??_R0?AVbad_array_new_length@std@@@8 0000000140016b98     MessageHistory.obj
 0003:00000bc8       ??_R0?AVbad_alloc@std@@@8  0000000140016bc8     MessageHistory.obj
 0003:00000bf0       ??_R0?AVexception@std@@@8  0000000140016bf0     MessageHistory.obj
 0003:00000c18       ??_R0?AVtype_info@@@8      0000000140016c18     MSVCRT:std_type_info_static.obj
 0003:00000c40       theAccessBridgeInitializedFlag 0000000140016c40     AccessBridgeCalls.obj
 0003:00000c48       ?_OptionsStorage@?1??__local_stdio_printf_options@@9@4_KA 0000000140016c48     AccessBridgeDebug.obj
 0003:00000d60       ?theFromJavaHelloMsgID@@3IA 0000000140016d60     AccessBridgeMessages.obj
 0003:00000d64       ?theFromWindowsHelloMsgID@@3IA 0000000140016d64     AccessBridgeMessages.obj
 0003:00000d68       ?g_LogStringCallback@@3P6AXPEBD@ZEA 0000000140016d68     AccessInfo.obj
 0003:00000db0       ?theDialogWindow@@3PEAUHWND__@@EA 0000000140016db0     jaccessinspector.obj
 0003:00000db8       ?theGoToDialogWindow@@3PEAUHWND__@@EA 0000000140016db8     jaccessinspector.obj
 0003:00000dc0       ?theInstance@@3PEAUHINSTANCE__@@EA 0000000140016dc0     jaccessinspector.obj
 0003:00000dc8       ?theAccessBridgeLoadedFlag@@3HA 0000000140016dc8     jaccessinspector.obj
 0003:00000dcc       ?updateMouse@@3HA          0000000140016dcc     jaccessinspector.obj
 0003:00000dd0       ?prevKbdHook@@3PEAUHHOOK__@@EA 0000000140016dd0     jaccessinspector.obj
 0003:00000dd8       ?prevMouseHook@@3PEAUHHOOK__@@EA 0000000140016dd8     jaccessinspector.obj
 0003:00000de0       ?updateF1@@3HA             0000000140016de0     jaccessinspector.obj
 0003:00000de4       ?updateF2@@3HA             0000000140016de4     jaccessinspector.obj
 0003:00000de8       ?trackMouse@@3HA           0000000140016de8     jaccessinspector.obj
 0003:00000dec       ?trackMouseExited@@3HA     0000000140016dec     jaccessinspector.obj
 0003:00000df0       ?trackMouseClicked@@3HA    0000000140016df0     jaccessinspector.obj
 0003:00000df4       ?trackMousePressed@@3HA    0000000140016df4     jaccessinspector.obj
 0003:00000df8       ?trackMouseReleased@@3HA   0000000140016df8     jaccessinspector.obj
 0003:00000dfc       ?trackFocus@@3HA           0000000140016dfc     jaccessinspector.obj
 0003:00000e00       ?trackFocusLost@@3HA       0000000140016e00     jaccessinspector.obj
 0003:00000e04       ?trackCaret@@3HA           0000000140016e04     jaccessinspector.obj
 0003:00000e08       ?trackShutdown@@3HA        0000000140016e08     jaccessinspector.obj
 0003:00000e0c       ?trackMenuSelected@@3HA    0000000140016e0c     jaccessinspector.obj
 0003:00000e10       ?trackMenuDeselected@@3HA  0000000140016e10     jaccessinspector.obj
 0003:00000e14       ?trackMenuCanceled@@3HA    0000000140016e14     jaccessinspector.obj
 0003:00000e18       ?trackPopupVisible@@3HA    0000000140016e18     jaccessinspector.obj
 0003:00000e1c       ?trackPopupInvisible@@3HA  0000000140016e1c     jaccessinspector.obj
 0003:00000e20       ?trackPopupCanceled@@3HA   0000000140016e20     jaccessinspector.obj
 0003:00000e24       ?trackPropertyNameChange@@3HA 0000000140016e24     jaccessinspector.obj
 0003:00000e28       ?trackPropertyDescriptionChange@@3HA 0000000140016e28     jaccessinspector.obj
 0003:00000e2c       ?trackPropertyStateChange@@3HA 0000000140016e2c     jaccessinspector.obj
 0003:00000e30       ?trackPropertyValueChange@@3HA 0000000140016e30     jaccessinspector.obj
 0003:00000e34       ?trackPropertySelectionChange@@3HA 0000000140016e34     jaccessinspector.obj
 0003:00000e38       ?trackPropertyTextChange@@3HA 0000000140016e38     jaccessinspector.obj
 0003:00000e3c       ?trackPropertyCaretChange@@3HA 0000000140016e3c     jaccessinspector.obj
 0003:00000e40       ?trackPropertyVisibleDataChange@@3HA 0000000140016e40     jaccessinspector.obj
 0003:00000e44       ?trackPropertyChildChange@@3HA 0000000140016e44     jaccessinspector.obj
 0003:00000e48       ?trackPropertyActiveDescendentChange@@3HA 0000000140016e48     jaccessinspector.obj
 0003:00000e4c       ?trackPropertyTableModelChange@@3HA 0000000140016e4c     jaccessinspector.obj
 0003:00000e50       ?logfile@@3PEAU_iobuf@@EA  0000000140016e50     jaccessinspector.obj
 0003:00000e58       ?g_MessageHistory@@3VMessageHistory@@A 0000000140016e58     jaccessinspector.obj
 0003:00001410       __scrt_current_native_startup_state 0000000140017410     MSVCRT:utility.obj
 0003:00001418       __scrt_native_startup_lock 0000000140017418     MSVCRT:utility.obj
 0003:00001468       _tls_index                 0000000140017468     MSVCRT:tlssup.obj
 0003:0000146c       __favor                    000000014001746c     MSVCRT:cpu_disp.obj
 0003:00001470       __scrt_debugger_hook_flag  0000000140017470     MSVCRT:utility_desktop.obj
 0003:00001480       ?__type_info_root_node@@3U__type_info_node@@A 0000000140017480     MSVCRT:tncleanup.obj
 0003:00001490       ?_OptionsStorage@?1??__local_stdio_scanf_options@@9@4_KA 0000000140017490     MSVCRT:default_local_stdio_options.obj
 0003:000014a0       theAccessBridge            00000001400174a0     <common>
 0003:000017a8       theAccessBridgeInstance    00000001400177a8     <common>
 0003:000017b0       __dyn_tls_dtor_callback    00000001400177b0     <common>
 0003:000017b8       __dyn_tls_init_callback    00000001400177b8     <common>

 entry point at        0001:0000eb04

 Static symbols

 0000:fffe4000       .debug$S                   0000000140000000     msvcprt:MSVCP140.dll
 0000:fffe4000       .debug$S                   0000000140000000     vcruntime:VCRUNTIME140.dll
 0000:fffe4000       .debug$S                   0000000140000000     vcruntime:VCRUNTIME140.dll
 0000:fffe4000       .debug$S                   0000000140000000     vcruntime:VCRUNTIME140.dll
 0000:fffe4000       .debug$S                   0000000140000000     vcruntime:VCRUNTIME140.dll
 0000:fffe4000       .debug$S                   0000000140000000     vcruntime:VCRUNTIME140.dll
 0000:fffe4000       .debug$S                   0000000140000000     vcruntime:VCRUNTIME140.dll
 0000:fffe4000       .debug$S                   0000000140000000     vcruntime:VCRUNTIME140.dll
 0000:fffe4000       .debug$S                   0000000140000000     vcruntime:VCRUNTIME140.dll
 0000:fffe4000       .debug$S                   0000000140000000     vcruntime:VCRUNTIME140.dll
 0000:fffe4000       .debug$S                   0000000140000000     vcruntime:VCRUNTIME140_1.dll
 0000:fffe4000       .debug$S                   0000000140000000     ucrt:api-ms-win-crt-environment-l1-1-0.dll
 0000:fffe4000       .debug$S                   0000000140000000     ucrt:api-ms-win-crt-heap-l1-1-0.dll
 0000:fffe4000       .debug$S                   0000000140000000     ucrt:api-ms-win-crt-heap-l1-1-0.dll
 0000:fffe4000       .debug$S                   0000000140000000     ucrt:api-ms-win-crt-heap-l1-1-0.dll
 0000:fffe4000       .debug$S                   0000000140000000     ucrt:api-ms-win-crt-heap-l1-1-0.dll
 0000:fffe4000       .debug$S                   0000000140000000     ucrt:api-ms-win-crt-locale-l1-1-0.dll
 0000:fffe4000       .debug$S                   0000000140000000     ucrt:api-ms-win-crt-math-l1-1-0.dll
 0000:fffe4000       .debug$S                   0000000140000000     ucrt:api-ms-win-crt-runtime-l1-1-0.dll
 0000:fffe4000       .debug$S                   0000000140000000     ucrt:api-ms-win-crt-runtime-l1-1-0.dll
 0000:fffe4000       .debug$S                   0000000140000000     ucrt:api-ms-win-crt-runtime-l1-1-0.dll
 0000:fffe4000       .debug$S                   0000000140000000     ucrt:api-ms-win-crt-runtime-l1-1-0.dll
 0000:fffe4000       .debug$S                   0000000140000000     ucrt:api-ms-win-crt-runtime-l1-1-0.dll
 0000:fffe4000       .debug$S                   0000000140000000     ucrt:api-ms-win-crt-runtime-l1-1-0.dll
 0000:fffe4000       .debug$S                   0000000140000000     ucrt:api-ms-win-crt-runtime-l1-1-0.dll
 0000:fffe4000       .debug$S                   0000000140000000     ucrt:api-ms-win-crt-runtime-l1-1-0.dll
 0000:fffe4000       .debug$S                   0000000140000000     ucrt:api-ms-win-crt-runtime-l1-1-0.dll
 0000:fffe4000       .debug$S                   0000000140000000     ucrt:api-ms-win-crt-runtime-l1-1-0.dll
 0000:fffe4000       .debug$S                   0000000140000000     ucrt:api-ms-win-crt-runtime-l1-1-0.dll
 0000:fffe4000       .debug$S                   0000000140000000     ucrt:api-ms-win-crt-runtime-l1-1-0.dll
 0000:fffe4000       .debug$S                   0000000140000000     ucrt:api-ms-win-crt-runtime-l1-1-0.dll
 0000:fffe4000       .debug$S                   0000000140000000     ucrt:api-ms-win-crt-runtime-l1-1-0.dll
 0000:fffe4000       .debug$S                   0000000140000000     ucrt:api-ms-win-crt-runtime-l1-1-0.dll
 0000:fffe4000       .debug$S                   0000000140000000     ucrt:api-ms-win-crt-runtime-l1-1-0.dll
 0000:fffe4000       .debug$S                   0000000140000000     ucrt:api-ms-win-crt-runtime-l1-1-0.dll
 0000:fffe4000       .debug$S                   0000000140000000     ucrt:api-ms-win-crt-runtime-l1-1-0.dll
 0000:fffe4000       .debug$S                   0000000140000000     ucrt:api-ms-win-crt-runtime-l1-1-0.dll
 0000:fffe4000       .debug$S                   0000000140000000     ucrt:api-ms-win-crt-runtime-l1-1-0.dll
 0000:fffe4000       .debug$S                   0000000140000000     ucrt:api-ms-win-crt-stdio-l1-1-0.dll
 0000:fffe4000       .debug$S                   0000000140000000     ucrt:api-ms-win-crt-stdio-l1-1-0.dll
 0000:fffe4000       .debug$S                   0000000140000000     ucrt:api-ms-win-crt-stdio-l1-1-0.dll
 0000:fffe4000       .debug$S                   0000000140000000     ucrt:api-ms-win-crt-stdio-l1-1-0.dll
 0000:fffe4000       .debug$S                   0000000140000000     ucrt:api-ms-win-crt-stdio-l1-1-0.dll
 0000:fffe4000       .debug$S                   0000000140000000     ucrt:api-ms-win-crt-stdio-l1-1-0.dll
 0000:fffe4000       .debug$S                   0000000140000000     ucrt:api-ms-win-crt-stdio-l1-1-0.dll
 0000:fffe4000       .debug$S                   0000000140000000     ucrt:api-ms-win-crt-stdio-l1-1-0.dll
 0000:fffe4000       .debug$S                   0000000140000000     ucrt:api-ms-win-crt-stdio-l1-1-0.dll
 0000:fffe4000       .debug$S                   0000000140000000     ucrt:api-ms-win-crt-string-l1-1-0.dll
 0000:fffe4000       .debug$S                   0000000140000000     ucrt:api-ms-win-crt-string-l1-1-0.dll
 0000:fffe4000       .debug$S                   0000000140000000     ucrt:api-ms-win-crt-string-l1-1-0.dll
 0000:fffe4000       .debug$S                   0000000140000000     ucrt:api-ms-win-crt-string-l1-1-0.dll
 0000:fffe4000       .debug$S                   0000000140000000     ucrt:api-ms-win-crt-time-l1-1-0.dll
 0000:fffe4000       .debug$S                   0000000140000000     ucrt:api-ms-win-crt-time-l1-1-0.dll
 0000:fffe4000       .debug$S                   0000000140000000     ucrt:api-ms-win-crt-time-l1-1-0.dll
 0000:fffe4000       .debug$S                   0000000140000000     advapi32:ADVAPI32.dll
 0000:fffe4000       .debug$S                   0000000140000000     advapi32:ADVAPI32.dll
 0000:fffe4000       .debug$S                   0000000140000000     advapi32:ADVAPI32.dll
 0000:fffe4000       .debug$S                   0000000140000000     advapi32:ADVAPI32.dll
 0000:fffe4000       .debug$S                   0000000140000000     advapi32:ADVAPI32.dll
 0000:fffe4000       .debug$S                   0000000140000000     advapi32:ADVAPI32.dll
 0000:fffe4000       .debug$S                   0000000140000000     kernel32:KERNEL32.dll
 0000:fffe4000       .debug$S                   0000000140000000     kernel32:KERNEL32.dll
 0000:fffe4000       .debug$S                   0000000140000000     kernel32:KERNEL32.dll
 0000:fffe4000       .debug$S                   0000000140000000     kernel32:KERNEL32.dll
 0000:fffe4000       .debug$S                   0000000140000000     kernel32:KERNEL32.dll
 0000:fffe4000       .debug$S                   0000000140000000     kernel32:KERNEL32.dll
 0000:fffe4000       .debug$S                   0000000140000000     kernel32:KERNEL32.dll
 0000:fffe4000       .debug$S                   0000000140000000     kernel32:KERNEL32.dll
 0000:fffe4000       .debug$S                   0000000140000000     kernel32:KERNEL32.dll
 0000:fffe4000       .debug$S                   0000000140000000     kernel32:KERNEL32.dll
 0000:fffe4000       .debug$S                   0000000140000000     kernel32:KERNEL32.dll
 0000:fffe4000       .debug$S                   0000000140000000     kernel32:KERNEL32.dll
 0000:fffe4000       .debug$S                   0000000140000000     kernel32:KERNEL32.dll
 0000:fffe4000       .debug$S                   0000000140000000     kernel32:KERNEL32.dll
 0000:fffe4000       .debug$S                   0000000140000000     kernel32:KERNEL32.dll
 0000:fffe4000       .debug$S                   0000000140000000     kernel32:KERNEL32.dll
 0000:fffe4000       .debug$S                   0000000140000000     kernel32:KERNEL32.dll
 0000:fffe4000       .debug$S                   0000000140000000     kernel32:KERNEL32.dll
 0000:fffe4000       .debug$S                   0000000140000000     kernel32:KERNEL32.dll
 0000:fffe4000       .debug$S                   0000000140000000     kernel32:KERNEL32.dll
 0000:fffe4000       .debug$S                   0000000140000000     kernel32:KERNEL32.dll
 0000:fffe4000       .debug$S                   0000000140000000     kernel32:KERNEL32.dll
 0000:fffe4000       .debug$S                   0000000140000000     kernel32:KERNEL32.dll
 0000:fffe4000       .debug$S                   0000000140000000     kernel32:KERNEL32.dll
 0000:fffe4000       .debug$S                   0000000140000000     kernel32:KERNEL32.dll
 0000:fffe4000       .debug$S                   0000000140000000     kernel32:KERNEL32.dll
 0000:fffe4000       .debug$S                   0000000140000000     user32:USER32.dll
 0000:fffe4000       .debug$S                   0000000140000000     user32:USER32.dll
 0000:fffe4000       .debug$S                   0000000140000000     user32:USER32.dll
 0000:fffe4000       .debug$S                   0000000140000000     user32:USER32.dll
 0000:fffe4000       .debug$S                   0000000140000000     user32:USER32.dll
 0000:fffe4000       .debug$S                   0000000140000000     user32:USER32.dll
 0000:fffe4000       .debug$S                   0000000140000000     user32:USER32.dll
 0000:fffe4000       .debug$S                   0000000140000000     user32:USER32.dll
 0000:fffe4000       .debug$S                   0000000140000000     user32:USER32.dll
 0000:fffe4000       .debug$S                   0000000140000000     user32:USER32.dll
 0000:fffe4000       .debug$S                   0000000140000000     user32:USER32.dll
 0000:fffe4000       .debug$S                   0000000140000000     user32:USER32.dll
 0000:fffe4000       .debug$S                   0000000140000000     user32:USER32.dll
 0000:fffe4000       .debug$S                   0000000140000000     user32:USER32.dll
 0000:fffe4000       .debug$S                   0000000140000000     user32:USER32.dll
 0000:fffe4000       .debug$S                   0000000140000000     user32:USER32.dll
 0000:fffe4000       .debug$S                   0000000140000000     user32:USER32.dll
 0000:fffe4000       .debug$S                   0000000140000000     user32:USER32.dll
 0000:fffe4000       .debug$S                   0000000140000000     user32:USER32.dll
 0000:fffe4000       .debug$S                   0000000140000000     user32:USER32.dll
 0000:fffe4000       .debug$S                   0000000140000000     user32:USER32.dll
 0000:fffe4000       .debug$S                   0000000140000000     user32:USER32.dll
 0000:fffe4000       .debug$S                   0000000140000000     user32:USER32.dll
 0000:fffe4000       .debug$S                   0000000140000000     user32:USER32.dll
 0000:fffe4000       .debug$S                   0000000140000000     user32:USER32.dll
 0000:fffe4000       .debug$S                   0000000140000000     user32:USER32.dll
 0000:fffe4000       .debug$S                   0000000140000000     user32:USER32.dll
 0000:fffe4000       .debug$S                   0000000140000000     user32:USER32.dll
 0000:fffe4000       .debug$S                   0000000140000000     user32:USER32.dll
 0000:fffe4000       .debug$S                   0000000140000000     user32:USER32.dll
 0000:fffe4000       .debug$S                   0000000140000000     user32:USER32.dll
 0000:fffe4000       .debug$S                   0000000140000000     user32:USER32.dll
 0000:fffe4000       .debug$S                   0000000140000000     user32:USER32.dll
 0000:fffe4000       .debug$S                   0000000140000000     user32:USER32.dll
 0000:fffe4000       .debug$S                   0000000140000000     user32:USER32.dll
 0000:fffe4000       .debug$S                   0000000140000000     user32:USER32.dll
 0000:fffe4000       .debug$S                   0000000140000000     user32:USER32.dll
 0000:fffe4000       .debug$S                   0000000140000000     user32:USER32.dll
 0000:fffe4000       .debug$S                   0000000140000000     user32:USER32.dll
 0000:fffe4000       .debug$S                   0000000140000000     user32:USER32.dll
 0001:00000000       ??__Eg_MessageHistory@@YAXXZ 0000000140001000 f   jaccessinspector.obj
 0001:00005d50       localtime                  0000000140006d50 f   AccessInfo.obj
 0001:00005d70       time                       0000000140006d70 f   AccessInfo.obj
 0001:00009f9c       $LN133                     000000014000af9c     jaccessinspector.obj
 0001:00009fd4       $LN132                     000000014000afd4     jaccessinspector.obj
 0001:0000a0a0       $LN131                     000000014000b0a0     jaccessinspector.obj
 0001:0000e2a0       capture_current_context    000000014000f2a0 f   MSVCRT:gs_report.obj
 0001:0000e310       capture_previous_context   000000014000f310 f   MSVCRT:gs_report.obj
 0001:0000e400       $$000000                   000000014000f400     MSVCRT:chkstk.obj
 0001:0000e460       $$000000                   000000014000f460     MSVCRT:amdsecgs.obj
 0001:0000e8ac       ?pre_c_initialization@@YAHXZ 000000014000f8ac f   MSVCRT:exe_winmain.obj
 0001:0000e964       ?post_pgo_initialization@@YAHXZ 000000014000f964 f   MSVCRT:exe_winmain.obj
 0001:0000e974       ?pre_cpp_initialization@@YAXXZ 000000014000f974 f   MSVCRT:exe_winmain.obj
 0001:0000e990       ?__scrt_common_main_seh@@YAHXZ 000000014000f990 f   MSVCRT:exe_winmain.obj
 0001:0000f200       $$000000                   0000000140010200     MSVCRT:guard_dispatch.obj
 0001:0000f220       $$000000                   0000000140010220     MSVCRT:guard_xfg_dispatch.obj
 0001:0000f240       ?dtor$0@?0??AddMessage@MessageHistory@@QEAAXPEBD@Z@4HA 0000000140010240 f   MessageHistory.obj
 0001:0000f260       ?dtor$0@?0???$?0V?$basic_string@DU?$char_traits@D@std@@V?$allocator@D@2@@std@@@?$_List_node_emplace_op2@V?$allocator@U?$_List_node@V?$basic_string@DU?$char_traits@D@std@@V?$allocator@D@2@@std@@PEAX@std@@@std@@@std@@QEAA@AEAV?$allocator@U?$_List_node@V?$basic_string@DU?$char_traits@D@std@@V?$allocator@D@2@@std@@PEAX@std@@@1@$$QEAV?$basic_string@DU?$char_traits@D@std@@V?$allocator@D@2@@1@@Z@4HA 0000000140010260 f   MessageHistory.obj
 0001:0000f280       ?dtor$0@?0???0?$basic_string@DU?$char_traits@D@std@@V?$allocator@D@2@@std@@QEAA@QEBD@Z@4HA 0000000140010280 f   MessageHistory.obj
 0001:0000f298       __scrt_is_nonwritable_in_current_image$filt$0 0000000140010298 f   MSVCRT:utility.obj
 0001:0000f2b0       ?filt$0@?0??__scrt_common_main_seh@@YAHXZ@4HA 00000001400102b0 f   MSVCRT:exe_winmain.obj
 0001:0000f2d0       ??__Fg_MessageHistory@@YAXXZ 00000001400102d0 f   jaccessinspector.obj
 0002:00000480       ?pre_cpp_initializer@@3P6AXXZEA 0000000140011480     MSVCRT:exe_winmain.obj
 0002:00000488       ?g_MessageHistory$initializer$@@3P6AXXZEA 0000000140011488     jaccessinspector.obj
 0002:000004a0       ?pre_c_initializer@@3P6AHXZEA 00000001400114a0     MSVCRT:exe_winmain.obj
 0002:000004a8       ?post_pgo_initializer@@3P6AHXZEA 00000001400114a8     MSVCRT:exe_winmain.obj
 0002:000004f0       $SG44959                   00000001400114f0     AccessBridgeDebug.obj
 0002:0000050c       $SG44961                   000000014001150c     AccessBridgeDebug.obj
 0002:00000514       $SG44962                   0000000140011514     AccessBridgeDebug.obj
 0002:00000518       $SG44964                   0000000140011518     AccessBridgeDebug.obj
 0002:00000520       $SG44965                   0000000140011520     AccessBridgeDebug.obj
 0002:00000538       $SG44992                   0000000140011538     AccessBridgeDebug.obj
 0002:00000558       $SG44993                   0000000140011558     AccessBridgeDebug.obj
 0002:00000564       $SG44995                   0000000140011564     AccessBridgeDebug.obj
 0002:00000568       $SG45032                   0000000140011568     AccessBridgeDebug.obj
 0002:00000570       $SG45033                   0000000140011570     AccessBridgeDebug.obj
 0002:00000578       $SG45044                   0000000140011578     AccessBridgeDebug.obj
 0002:00000580       $SG45045                   0000000140011580     AccessBridgeDebug.obj
 0002:00000588       $SG45056                   0000000140011588     AccessBridgeDebug.obj
 0002:00000590       $SG45057                   0000000140011590     AccessBridgeDebug.obj
 0002:00000598       $SG45068                   0000000140011598     AccessBridgeDebug.obj
 0002:000005a0       $SG45069                   00000001400115a0     AccessBridgeDebug.obj
 0002:000005a8       $SG40363                   00000001400115a8     AccessBridgeMessages.obj
 0002:000005c8       $SG40364                   00000001400115c8     AccessBridgeMessages.obj
 0002:000005f0       $SG49170                   00000001400115f0     AccessInfo.obj
 0002:000005f4       $SG49172                   00000001400115f4     AccessInfo.obj
 0002:000005f8       $SG49175                   00000001400115f8     AccessInfo.obj
 0002:00000608       $SG49215                   0000000140011608     AccessInfo.obj
 0002:00000634       $SG49216                   0000000140011634     AccessInfo.obj
 0002:00000638       $SG49217                   0000000140011638     AccessInfo.obj
 0002:0000063c       $SG49256                   000000014001163c     AccessInfo.obj
 0002:00000640       $SG49393                   0000000140011640     AccessInfo.obj
 0002:00000668       $SG49394                   0000000140011668     AccessInfo.obj
 0002:00000680       $SG49395                   0000000140011680     AccessInfo.obj
 0002:000006a8       $SG49396                   00000001400116a8     AccessInfo.obj
 0002:000006d8       $SG49397                   00000001400116d8     AccessInfo.obj
 0002:00000708       $SG49398                   0000000140011708     AccessInfo.obj
 0002:00000738       $SG49402                   0000000140011738     AccessInfo.obj
 0002:00000768       $SG49403                   0000000140011768     AccessInfo.obj
 0002:00000790       $SG49406                   0000000140011790     AccessInfo.obj
 0002:000007ac       $SG49407                   00000001400117ac     AccessInfo.obj
 0002:000007b0       $SG49408                   00000001400117b0     AccessInfo.obj
 0002:000007c8       $SG49411                   00000001400117c8     AccessInfo.obj
 0002:000007f0       $SG49412                   00000001400117f0     AccessInfo.obj
 0002:00000810       $SG49413                   0000000140011810     AccessInfo.obj
 0002:00000828       $SG49414                   0000000140011828     AccessInfo.obj
 0002:00000840       $SG49415                   0000000140011840     AccessInfo.obj
 0002:00000868       $SG49416                   0000000140011868     AccessInfo.obj
 0002:00000880       $SG49417                   0000000140011880     AccessInfo.obj
 0002:000008a8       $SG49418                   00000001400118a8     AccessInfo.obj
 0002:000008c8       $SG49419                   00000001400118c8     AccessInfo.obj
 0002:000008e8       $SG49420                   00000001400118e8     AccessInfo.obj
 0002:00000918       $SG49423                   0000000140011918     AccessInfo.obj
 0002:00000940       $SG49426                   0000000140011940     AccessInfo.obj
 0002:00000980       $SG49429                   0000000140011980     AccessInfo.obj
 0002:000009a8       $SG49430                   00000001400119a8     AccessInfo.obj
 0002:000009d0       $SG49431                   00000001400119d0     AccessInfo.obj
 0002:000009f8       $SG49434                   00000001400119f8     AccessInfo.obj
 0002:00000a08       $SG49437                   0000000140011a08     AccessInfo.obj
 0002:00000a40       $SG49438                   0000000140011a40     AccessInfo.obj
 0002:00000a58       $SG49441                   0000000140011a58     AccessInfo.obj
 0002:00000a80       $SG49442                   0000000140011a80     AccessInfo.obj
 0002:00000aa0       $SG49443                   0000000140011aa0     AccessInfo.obj
 0002:00000ab8       $SG49446                   0000000140011ab8     AccessInfo.obj
 0002:00000ae0       $SG49447                   0000000140011ae0     AccessInfo.obj
 0002:00000b08       $SG49451                   0000000140011b08     AccessInfo.obj
 0002:00000b30       $SG49455                   0000000140011b30     AccessInfo.obj
 0002:00000b58       $SG49456                   0000000140011b58     AccessInfo.obj
 0002:00000b78       $SG49457                   0000000140011b78     AccessInfo.obj
 0002:00000b98       $SG49459                   0000000140011b98     AccessInfo.obj
 0002:00000bc0       $SG49461                   0000000140011bc0     AccessInfo.obj
 0002:00000be0       $SG49464                   0000000140011be0     AccessInfo.obj
 0002:00000c28       $SG49467                   0000000140011c28     AccessInfo.obj
 0002:00000c68       $SG49470                   0000000140011c68     AccessInfo.obj
 0002:00000c90       $SG49471                   0000000140011c90     AccessInfo.obj
 0002:00000cb0       $SG49472                   0000000140011cb0     AccessInfo.obj
 0002:00000cd0       $SG49473                   0000000140011cd0     AccessInfo.obj
 0002:00000d00       $SG49475                   0000000140011d00     AccessInfo.obj
 0002:00000d20       $SG49476                   0000000140011d20     AccessInfo.obj
 0002:00000d48       $SG49477                   0000000140011d48     AccessInfo.obj
 0002:00000d70       $SG49478                   0000000140011d70     AccessInfo.obj
 0002:00000d98       $SG49480                   0000000140011d98     AccessInfo.obj
 0002:00000db8       $SG49481                   0000000140011db8     AccessInfo.obj
 0002:00000dd8       $SG49482                   0000000140011dd8     AccessInfo.obj
 0002:00000df8       $SG49483                   0000000140011df8     AccessInfo.obj
 0002:00000e18       $SG49484                   0000000140011e18     AccessInfo.obj
 0002:00000e30       $SG49486                   0000000140011e30     AccessInfo.obj
 0002:00000e50       $SG49487                   0000000140011e50     AccessInfo.obj
 0002:00000e70       $SG49488                   0000000140011e70     AccessInfo.obj
 0002:00000e90       $SG49491                   0000000140011e90     AccessInfo.obj
 0002:00000eb8       $SG49493                   0000000140011eb8     AccessInfo.obj
 0002:00000ee0       $SG49494                   0000000140011ee0     AccessInfo.obj
 0002:00000f00       $SG49495                   0000000140011f00     AccessInfo.obj
 0002:00000f20       $SG49496                   0000000140011f20     AccessInfo.obj
 0002:00000f48       $SG49499                   0000000140011f48     AccessInfo.obj
 0002:00000f78       $SG49502                   0000000140011f78     AccessInfo.obj
 0002:00000fa0       $SG49503                   0000000140011fa0     AccessInfo.obj
 0002:00000fc0       $SG49504                   0000000140011fc0     AccessInfo.obj
 0002:00000fe0       $SG49506                   0000000140011fe0     AccessInfo.obj
 0002:00001008       $SG49508                   0000000140012008     AccessInfo.obj
 0002:00001028       $SG49510                   0000000140012028     AccessInfo.obj
 0002:00001048       $SG49512                   0000000140012048     AccessInfo.obj
 0002:00001068       $SG49516                   0000000140012068     AccessInfo.obj
 0002:00001090       $SG49517                   0000000140012090     AccessInfo.obj
 0002:000010b0       $SG49518                   00000001400120b0     AccessInfo.obj
 0002:000010d8       $SG49519                   00000001400120d8     AccessInfo.obj
 0002:00001100       $SG49520                   0000000140012100     AccessInfo.obj
 0002:00001128       $SG49521                   0000000140012128     AccessInfo.obj
 0002:00001148       $SG49522                   0000000140012148     AccessInfo.obj
 0002:00001168       $SG49525                   0000000140012168     AccessInfo.obj
 0002:00001198       $SG49526                   0000000140012198     AccessInfo.obj
 0002:000011c8       $SG49527                   00000001400121c8     AccessInfo.obj
 0002:000011e0       $SG49528                   00000001400121e0     AccessInfo.obj
 0002:000011f8       $SG49529                   00000001400121f8     AccessInfo.obj
 0002:00001218       $SG49530                   0000000140012218     AccessInfo.obj
 0002:00001230       $SG49533                   0000000140012230     AccessInfo.obj
 0002:00001278       $SG49536                   0000000140012278     AccessInfo.obj
 0002:000012a0       $SG49537                   00000001400122a0     AccessInfo.obj
 0002:000012b8       $SG49538                   00000001400122b8     AccessInfo.obj
 0002:000012d0       $SG49541                   00000001400122d0     AccessInfo.obj
 0002:00001300       $SG49542                   0000000140012300     AccessInfo.obj
 0002:00001328       $SG49543                   0000000140012328     AccessInfo.obj
 0002:00001350       $SG49544                   0000000140012350     AccessInfo.obj
 0002:00001378       $SG49545                   0000000140012378     AccessInfo.obj
 0002:00001398       $SG49548                   0000000140012398     AccessInfo.obj
 0002:000013d0       $SG49549                   00000001400123d0     AccessInfo.obj
 0002:000013e8       $SG49550                   00000001400123e8     AccessInfo.obj
 0002:000013f0       $SG49553                   00000001400123f0     AccessInfo.obj
 0002:00001420       $SG49554                   0000000140012420     AccessInfo.obj
 0002:00001448       $SG49555                   0000000140012448     AccessInfo.obj
 0002:00001460       $SG49556                   0000000140012460     AccessInfo.obj
 0002:00001478       $SG49557                   0000000140012478     AccessInfo.obj
 0002:00001498       $SG49558                   0000000140012498     AccessInfo.obj
 0002:000014b0       $SG49561                   00000001400124b0     AccessInfo.obj
 0002:000014e0       $SG49564                   00000001400124e0     AccessInfo.obj
 0002:00001508       $SG49565                   0000000140012508     AccessInfo.obj
 0002:00001520       $SG49566                   0000000140012520     AccessInfo.obj
 0002:00001538       $SG49568                   0000000140012538     AccessInfo.obj
 0002:00001560       $SG49570                   0000000140012560     AccessInfo.obj
 0002:00001588       $SG49571                   0000000140012588     AccessInfo.obj
 0002:000015a8       $SG49572                   00000001400125a8     AccessInfo.obj
 0002:000015c0       $SG49574                   00000001400125c0     AccessInfo.obj
 0002:000015e8       $SG49575                   00000001400125e8     AccessInfo.obj
 0002:00001608       $SG49576                   0000000140012608     AccessInfo.obj
 0002:00001628       $SG49577                   0000000140012628     AccessInfo.obj
 0002:00001650       $SG49579                   0000000140012650     AccessInfo.obj
 0002:00001690       $SG49582                   0000000140012690     AccessInfo.obj
 0002:000016b0       $SG49584                   00000001400126b0     AccessInfo.obj
 0002:000016d0       $SG49585                   00000001400126d0     AccessInfo.obj
 0002:000016e8       $SG49586                   00000001400126e8     AccessInfo.obj
 0002:00001704       $SG49588                   0000000140012704     AccessInfo.obj
 0002:00001710       $SG49589                   0000000140012710     AccessInfo.obj
 0002:00001720       $SG49590                   0000000140012720     AccessInfo.obj
 0002:00001740       $SG49591                   0000000140012740     AccessInfo.obj
 0002:00001748       $SG49592                   0000000140012748     AccessInfo.obj
 0002:00001754       $SG49593                   0000000140012754     AccessInfo.obj
 0002:00001760       $SG49594                   0000000140012760     AccessInfo.obj
 0002:00001770       $SG49595                   0000000140012770     AccessInfo.obj
 0002:00001780       $SG49596                   0000000140012780     AccessInfo.obj
 0002:00001788       $SG49597                   0000000140012788     AccessInfo.obj
 0002:00001798       $SG49598                   0000000140012798     AccessInfo.obj
 0002:000017ac       $SG49599                   00000001400127ac     AccessInfo.obj
 0002:000017b8       $SG49600                   00000001400127b8     AccessInfo.obj
 0002:000017c8       $SG49601                   00000001400127c8     AccessInfo.obj
 0002:000017d8       $SG49602                   00000001400127d8     AccessInfo.obj
 0002:000017e0       $SG49603                   00000001400127e0     AccessInfo.obj
 0002:000017f0       $SG49604                   00000001400127f0     AccessInfo.obj
 0002:00001800       $SG49605                   0000000140012800     AccessInfo.obj
 0002:00001808       $SG49606                   0000000140012808     AccessInfo.obj
 0002:00001830       $SG49607                   0000000140012830     AccessInfo.obj
 0002:00001858       $SG49608                   0000000140012858     AccessInfo.obj
 0002:00001878       $SG49609                   0000000140012878     AccessInfo.obj
 0002:00001898       $SG49610                   0000000140012898     AccessInfo.obj
 0002:000018c0       $SG49611                   00000001400128c0     AccessInfo.obj
 0002:000018e0       $SG49612                   00000001400128e0     AccessInfo.obj
 0002:00001900       $SG49613                   0000000140012900     AccessInfo.obj
 0002:00001920       $SG49614                   0000000140012920     AccessInfo.obj
 0002:00001940       $SG49615                   0000000140012940     AccessInfo.obj
 0002:00001960       $SG49616                   0000000140012960     AccessInfo.obj
 0002:00001988       $SG49619                   0000000140012988     AccessInfo.obj
 0002:000019a8       $SG49620                   00000001400129a8     AccessInfo.obj
 0002:000019d8       $SG49621                   00000001400129d8     AccessInfo.obj
 0002:000019f8       $SG49623                   00000001400129f8     AccessInfo.obj
 0002:00001a30       $SG49625                   0000000140012a30     AccessInfo.obj
 0002:00001a70       $SG49628                   0000000140012a70     AccessInfo.obj
 0002:00001a90       $SG49630                   0000000140012a90     AccessInfo.obj
 0002:00001ab0       $SG49631                   0000000140012ab0     AccessInfo.obj
 0002:00001ac8       $SG49632                   0000000140012ac8     AccessInfo.obj
 0002:00001ae4       $SG49634                   0000000140012ae4     AccessInfo.obj
 0002:00001af0       $SG49635                   0000000140012af0     AccessInfo.obj
 0002:00001b00       $SG49636                   0000000140012b00     AccessInfo.obj
 0002:00001b20       $SG49637                   0000000140012b20     AccessInfo.obj
 0002:00001b28       $SG49638                   0000000140012b28     AccessInfo.obj
 0002:00001b34       $SG49639                   0000000140012b34     AccessInfo.obj
 0002:00001b40       $SG49640                   0000000140012b40     AccessInfo.obj
 0002:00001b50       $SG49641                   0000000140012b50     AccessInfo.obj
 0002:00001b60       $SG49642                   0000000140012b60     AccessInfo.obj
 0002:00001b68       $SG49643                   0000000140012b68     AccessInfo.obj
 0002:00001b78       $SG49644                   0000000140012b78     AccessInfo.obj
 0002:00001b8c       $SG49645                   0000000140012b8c     AccessInfo.obj
 0002:00001b98       $SG49646                   0000000140012b98     AccessInfo.obj
 0002:00001ba8       $SG49647                   0000000140012ba8     AccessInfo.obj
 0002:00001bb8       $SG49648                   0000000140012bb8     AccessInfo.obj
 0002:00001bc0       $SG49649                   0000000140012bc0     AccessInfo.obj
 0002:00001bd0       $SG49650                   0000000140012bd0     AccessInfo.obj
 0002:00001be0       $SG49651                   0000000140012be0     AccessInfo.obj
 0002:00001be8       $SG49652                   0000000140012be8     AccessInfo.obj
 0002:00001c10       $SG49653                   0000000140012c10     AccessInfo.obj
 0002:00001c38       $SG49654                   0000000140012c38     AccessInfo.obj
 0002:00001c58       $SG49655                   0000000140012c58     AccessInfo.obj
 0002:00001c78       $SG49656                   0000000140012c78     AccessInfo.obj
 0002:00001ca0       $SG49657                   0000000140012ca0     AccessInfo.obj
 0002:00001cc0       $SG49658                   0000000140012cc0     AccessInfo.obj
 0002:00001ce0       $SG49659                   0000000140012ce0     AccessInfo.obj
 0002:00001d00       $SG49660                   0000000140012d00     AccessInfo.obj
 0002:00001d20       $SG49661                   0000000140012d20     AccessInfo.obj
 0002:00001d40       $SG49662                   0000000140012d40     AccessInfo.obj
 0002:00001d68       $SG49665                   0000000140012d68     AccessInfo.obj
 0002:00001d88       $SG49666                   0000000140012d88     AccessInfo.obj
 0002:00001db1       $SG60570                   0000000140012db1     MessageHistory.obj
 0002:00001db2       $SG60576                   0000000140012db2     MessageHistory.obj
 0002:00001db3       $SG60583                   0000000140012db3     MessageHistory.obj
 0002:00001db4       $SG60590                   0000000140012db4     MessageHistory.obj
 0002:00001db5       $SG60612                   0000000140012db5     MessageHistory.obj
 0002:00001db6       $SG60626                   0000000140012db6     MessageHistory.obj
 0002:00001db7       $SG60628                   0000000140012db7     MessageHistory.obj
 0002:00001db8       ?_Fake_alloc@std@@3U_Fake_allocator@1@B 0000000140012db8     MessageHistory.obj
 0002:00001e60       ?jaccessinspectorOptionsRegistryKey@@3QEBDEB 0000000140012e60     jaccessinspector.obj
 0002:00001e68       $SG49294                   0000000140012e68     jaccessinspector.obj
 0002:00001ea0       $SG66819                   0000000140012ea0     jaccessinspector.obj
 0002:00001ea2       ?_Fake_alloc@std@@3U_Fake_allocator@1@B 0000000140012ea2     jaccessinspector.obj
 0002:00001ea8       $SG66820                   0000000140012ea8     jaccessinspector.obj
 0002:00001ec0       $SG66821                   0000000140012ec0     jaccessinspector.obj
 0002:00001ee8       $SG66822                   0000000140012ee8     jaccessinspector.obj
 0002:00001f00       $SG66888                   0000000140012f00     jaccessinspector.obj
 0002:00001f20       $SG66896                   0000000140012f20     jaccessinspector.obj
 0002:00001f30       $SG66905                   0000000140012f30     jaccessinspector.obj
 0002:00001f40       $SG67000                   0000000140012f40     jaccessinspector.obj
 0002:00001f70       $SG67011                   0000000140012f70     jaccessinspector.obj
 0002:00001fa8       $SG67022                   0000000140012fa8     jaccessinspector.obj
 0002:00001fd8       $SG67033                   0000000140012fd8     jaccessinspector.obj
 0002:00002008       $SG67042                   0000000140013008     jaccessinspector.obj
 0002:00002028       $SG67050                   0000000140013028     jaccessinspector.obj
 0002:00002040       $SG67060                   0000000140013040     jaccessinspector.obj
 0002:00002080       $SG67069                   0000000140013080     jaccessinspector.obj
 0002:000020a0       $SG67085                   00000001400130a0     jaccessinspector.obj
 0002:000020e0       $SG67087                   00000001400130e0     jaccessinspector.obj
 0002:00002100       $SG67088                   0000000140013100     jaccessinspector.obj
 0002:00002108       $SG67090                   0000000140013108     jaccessinspector.obj
 0002:00002128       $SG67091                   0000000140013128     jaccessinspector.obj
 0002:00002130       $SG67103                   0000000140013130     jaccessinspector.obj
 0002:00002178       $SG67114                   0000000140013178     jaccessinspector.obj
 0002:000021a8       $SG67413                   00000001400131a8     jaccessinspector.obj
 0002:000021b8       $SG67415                   00000001400131b8     jaccessinspector.obj
 0002:000021d0       $SG67417                   00000001400131d0     jaccessinspector.obj
 0002:000021e8       $SG67419                   00000001400131e8     jaccessinspector.obj
 0002:00002200       $SG67421                   0000000140013200     jaccessinspector.obj
 0002:00002218       $SG67423                   0000000140013218     jaccessinspector.obj
 0002:00002228       $SG67425                   0000000140013228     jaccessinspector.obj
 0002:00002238       $SG67427                   0000000140013238     jaccessinspector.obj
 0002:00002248       $SG67429                   0000000140013248     jaccessinspector.obj
 0002:00002258       $SG67431                   0000000140013258     jaccessinspector.obj
 0002:00002270       $SG67433                   0000000140013270     jaccessinspector.obj
 0002:00002288       $SG67435                   0000000140013288     jaccessinspector.obj
 0002:000022a0       $SG67437                   00000001400132a0     jaccessinspector.obj
 0002:000022b8       $SG67439                   00000001400132b8     jaccessinspector.obj
 0002:000022d0       $SG67441                   00000001400132d0     jaccessinspector.obj
 0002:000022e8       $SG67443                   00000001400132e8     jaccessinspector.obj
 0002:00002300       $SG67445                   0000000140013300     jaccessinspector.obj
 0002:00002320       $SG67447                   0000000140013320     jaccessinspector.obj
 0002:00002340       $SG67449                   0000000140013340     jaccessinspector.obj
 0002:00002360       $SG67451                   0000000140013360     jaccessinspector.obj
 0002:00002380       $SG67453                   0000000140013380     jaccessinspector.obj
 0002:00002398       $SG67455                   0000000140013398     jaccessinspector.obj
 0002:000023b8       $SG67457                   00000001400133b8     jaccessinspector.obj
 0002:000023d8       $SG67459                   00000001400133d8     jaccessinspector.obj
 0002:000023f8       $SG67461                   00000001400133f8     jaccessinspector.obj
 0002:00002420       $SG67463                   0000000140013420     jaccessinspector.obj
 0002:00002440       $SG67558                   0000000140013440     jaccessinspector.obj
 0002:00002450       $SG67561                   0000000140013450     jaccessinspector.obj
 0002:00002468       $SG67564                   0000000140013468     jaccessinspector.obj
 0002:00002480       $SG67567                   0000000140013480     jaccessinspector.obj
 0002:00002498       $SG67570                   0000000140013498     jaccessinspector.obj
 0002:000024b0       $SG67573                   00000001400134b0     jaccessinspector.obj
 0002:000024c0       $SG67576                   00000001400134c0     jaccessinspector.obj
 0002:000024d0       $SG67579                   00000001400134d0     jaccessinspector.obj
 0002:000024e0       $SG67582                   00000001400134e0     jaccessinspector.obj
 0002:000024f0       $SG67585                   00000001400134f0     jaccessinspector.obj
 0002:00002508       $SG67588                   0000000140013508     jaccessinspector.obj
 0002:00002520       $SG67591                   0000000140013520     jaccessinspector.obj
 0002:00002538       $SG67594                   0000000140013538     jaccessinspector.obj
 0002:00002550       $SG67597                   0000000140013550     jaccessinspector.obj
 0002:00002568       $SG67600                   0000000140013568     jaccessinspector.obj
 0002:00002580       $SG67603                   0000000140013580     jaccessinspector.obj
 0002:00002598       $SG67606                   0000000140013598     jaccessinspector.obj
 0002:000025b8       $SG67609                   00000001400135b8     jaccessinspector.obj
 0002:000025d8       $SG67612                   00000001400135d8     jaccessinspector.obj
 0002:000025f8       $SG67615                   00000001400135f8     jaccessinspector.obj
 0002:00002618       $SG67618                   0000000140013618     jaccessinspector.obj
 0002:00002630       $SG67621                   0000000140013630     jaccessinspector.obj
 0002:00002650       $SG67624                   0000000140013650     jaccessinspector.obj
 0002:00002670       $SG67627                   0000000140013670     jaccessinspector.obj
 0002:00002690       $SG67630                   0000000140013690     jaccessinspector.obj
 0002:000026b8       $SG67633                   00000001400136b8     jaccessinspector.obj
 0002:000026d8       $SG67731                   00000001400136d8     jaccessinspector.obj
 0002:000026e8       GS_ExceptionPointers       00000001400136e8     MSVCRT:gs_report.obj
 0002:00003048       $unwind$initializeAccessBridge 0000000140014048     AccessBridgeCalls.obj
 0002:00003050       $unwind$shutdownAccessBridge 0000000140014050     AccessBridgeCalls.obj
 0002:00003058       $unwind$IsJavaWindow       0000000140014058     AccessBridgeCalls.obj
 0002:00003060       $unwind$GetAccessibleContextFromHWND 0000000140014060     AccessBridgeCalls.obj
 0002:00003068       $unwind$getHWNDFromAccessibleContext 0000000140014068     AccessBridgeCalls.obj
 0002:00003070       $unwind$SetJavaShutdown    0000000140014070     AccessBridgeCalls.obj
 0002:00003078       $unwind$SetFocusGained     0000000140014078     AccessBridgeCalls.obj
 0002:00003080       $unwind$SetFocusLost       0000000140014080     AccessBridgeCalls.obj
 0002:00003088       $unwind$SetCaretUpdate     0000000140014088     AccessBridgeCalls.obj
 0002:00003090       $unwind$SetMouseClicked    0000000140014090     AccessBridgeCalls.obj
 0002:00003098       $unwind$SetMouseEntered    0000000140014098     AccessBridgeCalls.obj
 0002:000030a0       $unwind$SetMouseExited     00000001400140a0     AccessBridgeCalls.obj
 0002:000030a8       $unwind$SetMousePressed    00000001400140a8     AccessBridgeCalls.obj
 0002:000030b0       $unwind$SetMouseReleased   00000001400140b0     AccessBridgeCalls.obj
 0002:000030b8       $unwind$SetMenuCanceled    00000001400140b8     AccessBridgeCalls.obj
 0002:000030c0       $unwind$SetMenuDeselected  00000001400140c0     AccessBridgeCalls.obj
 0002:000030c8       $unwind$SetMenuSelected    00000001400140c8     AccessBridgeCalls.obj
 0002:000030d0       $unwind$SetPopupMenuCanceled 00000001400140d0     AccessBridgeCalls.obj
 0002:000030d8       $unwind$SetPopupMenuWillBecomeInvisible 00000001400140d8     AccessBridgeCalls.obj
 0002:000030e0       $unwind$SetPopupMenuWillBecomeVisible 00000001400140e0     AccessBridgeCalls.obj
 0002:000030e8       $unwind$SetPropertyNameChange 00000001400140e8     AccessBridgeCalls.obj
 0002:000030f0       $unwind$SetPropertyDescriptionChange 00000001400140f0     AccessBridgeCalls.obj
 0002:000030f8       $unwind$SetPropertyStateChange 00000001400140f8     AccessBridgeCalls.obj
 0002:00003100       $unwind$SetPropertyValueChange 0000000140014100     AccessBridgeCalls.obj
 0002:00003108       $unwind$SetPropertySelectionChange 0000000140014108     AccessBridgeCalls.obj
 0002:00003110       $unwind$SetPropertyTextChange 0000000140014110     AccessBridgeCalls.obj
 0002:00003118       $unwind$SetPropertyCaretChange 0000000140014118     AccessBridgeCalls.obj
 0002:00003120       $unwind$SetPropertyVisibleDataChange 0000000140014120     AccessBridgeCalls.obj
 0002:00003128       $unwind$SetPropertyChildChange 0000000140014128     AccessBridgeCalls.obj
 0002:00003130       $unwind$SetPropertyActiveDescendentChange 0000000140014130     AccessBridgeCalls.obj
 0002:00003138       $unwind$SetPropertyTableModelChange 0000000140014138     AccessBridgeCalls.obj
 0002:00003140       $unwind$ReleaseJavaObject  0000000140014140     AccessBridgeCalls.obj
 0002:00003148       $unwind$GetVersionInfo     0000000140014148     AccessBridgeCalls.obj
 0002:00003150       $unwind$GetAccessibleContextAt 0000000140014150     AccessBridgeCalls.obj
 0002:00003158       $unwind$GetAccessibleContextWithFocus 0000000140014158     AccessBridgeCalls.obj
 0002:00003160       $unwind$GetAccessibleContextInfo 0000000140014160     AccessBridgeCalls.obj
 0002:00003168       $unwind$GetAccessibleChildFromContext 0000000140014168     AccessBridgeCalls.obj
 0002:00003170       $unwind$GetAccessibleParentFromContext 0000000140014170     AccessBridgeCalls.obj
 0002:00003178       $unwind$GetAccessibleTextInfo 0000000140014178     AccessBridgeCalls.obj
 0002:00003180       $unwind$GetAccessibleTextItems 0000000140014180     AccessBridgeCalls.obj
 0002:00003188       $unwind$GetAccessibleTextSelectionInfo 0000000140014188     AccessBridgeCalls.obj
 0002:00003190       $unwind$GetAccessibleTextAttributes 0000000140014190     AccessBridgeCalls.obj
 0002:00003198       $unwind$GetAccessibleTextRect 0000000140014198     AccessBridgeCalls.obj
 0002:000031a0       $unwind$GetAccessibleTextLineBounds 00000001400141a0     AccessBridgeCalls.obj
 0002:000031a8       $unwind$GetAccessibleTextRange 00000001400141a8     AccessBridgeCalls.obj
 0002:000031b0       $unwind$getAccessibleTableInfo 00000001400141b0     AccessBridgeCalls.obj
 0002:000031b8       $unwind$getAccessibleTableCellInfo 00000001400141b8     AccessBridgeCalls.obj
 0002:000031c0       $unwind$getAccessibleTableRowHeader 00000001400141c0     AccessBridgeCalls.obj
 0002:000031c8       $unwind$getAccessibleTableColumnHeader 00000001400141c8     AccessBridgeCalls.obj
 0002:000031d0       $unwind$getAccessibleTableRowDescription 00000001400141d0     AccessBridgeCalls.obj
 0002:000031d8       $unwind$getAccessibleTableColumnDescription 00000001400141d8     AccessBridgeCalls.obj
 0002:000031e0       $unwind$getAccessibleTableRowSelectionCount 00000001400141e0     AccessBridgeCalls.obj
 0002:000031e8       $unwind$isAccessibleTableRowSelected 00000001400141e8     AccessBridgeCalls.obj
 0002:000031f0       $unwind$getAccessibleTableRowSelections 00000001400141f0     AccessBridgeCalls.obj
 0002:000031f8       $unwind$getAccessibleTableColumnSelectionCount 00000001400141f8     AccessBridgeCalls.obj
 0002:00003200       $unwind$isAccessibleTableColumnSelected 0000000140014200     AccessBridgeCalls.obj
 0002:00003208       $unwind$getAccessibleTableColumnSelections 0000000140014208     AccessBridgeCalls.obj
 0002:00003210       $unwind$getAccessibleTableRow 0000000140014210     AccessBridgeCalls.obj
 0002:00003218       $unwind$getAccessibleTableColumn 0000000140014218     AccessBridgeCalls.obj
 0002:00003220       $unwind$getAccessibleTableIndex 0000000140014220     AccessBridgeCalls.obj
 0002:00003228       $unwind$getAccessibleRelationSet 0000000140014228     AccessBridgeCalls.obj
 0002:00003230       $unwind$getAccessibleHypertext 0000000140014230     AccessBridgeCalls.obj
 0002:00003238       $unwind$activateAccessibleHyperlink 0000000140014238     AccessBridgeCalls.obj
 0002:00003240       $unwind$getAccessibleHyperlinkCount 0000000140014240     AccessBridgeCalls.obj
 0002:00003248       $unwind$getAccessibleHypertextExt 0000000140014248     AccessBridgeCalls.obj
 0002:00003250       $unwind$getAccessibleHypertextLinkIndex 0000000140014250     AccessBridgeCalls.obj
 0002:00003258       $unwind$getAccessibleHyperlink 0000000140014258     AccessBridgeCalls.obj
 0002:00003260       $unwind$getAccessibleKeyBindings 0000000140014260     AccessBridgeCalls.obj
 0002:00003268       $unwind$getAccessibleIcons 0000000140014268     AccessBridgeCalls.obj
 0002:00003270       $unwind$getAccessibleActions 0000000140014270     AccessBridgeCalls.obj
 0002:00003278       $unwind$doAccessibleActions 0000000140014278     AccessBridgeCalls.obj
 0002:00003280       $unwind$IsSameObject       0000000140014280     AccessBridgeCalls.obj
 0002:00003288       $unwind$setTextContents    0000000140014288     AccessBridgeCalls.obj
 0002:00003290       $unwind$getParentWithRole  0000000140014290     AccessBridgeCalls.obj
 0002:00003298       $unwind$getParentWithRoleElseRoot 0000000140014298     AccessBridgeCalls.obj
 0002:000032a0       $unwind$getTopLevelObject  00000001400142a0     AccessBridgeCalls.obj
 0002:000032a8       $unwind$getObjectDepth     00000001400142a8     AccessBridgeCalls.obj
 0002:000032b0       $unwind$getActiveDescendent 00000001400142b0     AccessBridgeCalls.obj
 0002:000032b8       $unwind$GetCurrentAccessibleValueFromContext 00000001400142b8     AccessBridgeCalls.obj
 0002:000032c0       $unwind$GetMaximumAccessibleValueFromContext 00000001400142c0     AccessBridgeCalls.obj
 0002:000032c8       $unwind$GetMinimumAccessibleValueFromContext 00000001400142c8     AccessBridgeCalls.obj
 0002:000032d0       $unwind$GetAccessibleSelectionFromContext 00000001400142d0     AccessBridgeCalls.obj
 0002:000032d8       $unwind$GetAccessibleSelectionCountFromContext 00000001400142d8     AccessBridgeCalls.obj
 0002:000032e0       $unwind$IsAccessibleChildSelectedFromContext 00000001400142e0     AccessBridgeCalls.obj
 0002:000032e8       $unwind$RemoveAccessibleSelectionFromContext 00000001400142e8     AccessBridgeCalls.obj
 0002:000032f0       $unwind$SelectAllAccessibleSelectionFromContext 00000001400142f0     AccessBridgeCalls.obj
 0002:000032f8       $unwind$getVirtualAccessibleName 00000001400142f8     AccessBridgeCalls.obj
 0002:00003300       $unwind$requestFocus       0000000140014300     AccessBridgeCalls.obj
 0002:00003308       $unwind$selectTextRange    0000000140014308     AccessBridgeCalls.obj
 0002:00003310       $unwind$getTextAttributesInRange 0000000140014310     AccessBridgeCalls.obj
 0002:00003318       $unwind$getVisibleChildrenCount 0000000140014318     AccessBridgeCalls.obj
 0002:00003320       $unwind$getVisibleChildren 0000000140014320     AccessBridgeCalls.obj
 0002:00003328       $unwind$setCaretPosition   0000000140014328     AccessBridgeCalls.obj
 0002:00003330       $unwind$getCaretLocation   0000000140014330     AccessBridgeCalls.obj
 0002:00003338       $unwind$getEventsWaiting   0000000140014338     AccessBridgeCalls.obj
 0002:00003340       $unwind$addAccessibleSelectionFromContext 0000000140014340     AccessBridgeCalls.obj
 0002:00003348       $unwind$clearAccessibleSelectionFromContext 0000000140014348     AccessBridgeCalls.obj
 0002:00003350       $unwind$printError         0000000140014350     AccessBridgeDebug.obj
 0002:00003358       $unwind$PrintDebugString   0000000140014358     AccessBridgeDebug.obj
 0002:00003360       $unwind$wPrintJavaDebugString 0000000140014360     AccessBridgeDebug.obj
 0002:00003368       $unwind$wPrintDebugString  0000000140014368     AccessBridgeDebug.obj
 0002:00003370       $unwind$initializeFileLogger 0000000140014370     AccessBridgeDebug.obj
 0002:00003378       $unwind$finalizeFileLogger 0000000140014378     AccessBridgeDebug.obj
 0002:00003380       $unwind$getTimeStamp       0000000140014380     AccessBridgeDebug.obj
 0002:00003388       $unwind$PrintJavaDebugString2 0000000140014388     AccessBridgeDebug.obj
 0002:00003390       $unwind$_vfprintf_l        0000000140014390     AccessBridgeDebug.obj
 0002:00003390       $unwind$_vfwprintf_l       0000000140014390     AccessBridgeDebug.obj
 0002:00003390       $unwind$fprintf            0000000140014390     AccessBridgeDebug.obj
 0002:00003390       $unwind$printf             0000000140014390     AccessBridgeDebug.obj
 0002:00003390       $unwind$snprintf           0000000140014390     AccessInfo.obj
 0002:00003390       $unwind$_snprintf          0000000140014390     jaccessinspector.obj
 0002:00003390       $unwind$_vsnprintf         0000000140014390     jaccessinspector.obj
 0002:00003398       $unwind$vfprintf           0000000140014398     AccessBridgeDebug.obj
 0002:00003398       $unwind$vfwprintf          0000000140014398     AccessBridgeDebug.obj
 0002:00003398       $unwind$??$_Get_unwrapped_n@V?$_List_const_iterator@V?$_List_val@U?$_List_simple_types@V?$basic_string@DU?$char_traits@D@std@@V?$allocator@D@2@@std@@@std@@@std@@@std@@_K@std@@YA?A_T$$QEAV?$_List_const_iterator@V?$_List_val@U?$_List_simple_types@V?$basic_string@DU?$char_traits@D@std@@V?$allocator@D@2@@std@@@std@@@std@@@0@_K@Z 0000000140014398     MessageHistory.obj
 0002:00003398       $unwind$??0?$_List_const_iterator@V?$_List_val@U?$_List_simple_types@V?$basic_string@DU?$char_traits@D@std@@V?$allocator@D@2@@std@@@std@@@std@@@std@@QEAA@PEAU?$_List_node@V?$basic_string@DU?$char_traits@D@std@@V?$allocator@D@2@@std@@PEAX@1@PEBV?$_List_val@U?$_List_simple_types@V?$basic_string@DU?$char_traits@D@std@@V?$allocator@D@2@@std@@@std@@@1@@Z 0000000140014398     MessageHistory.obj
 0002:00003398       $unwind$??0?$_List_iterator@V?$_List_val@U?$_List_simple_types@V?$basic_string@DU?$char_traits@D@std@@V?$allocator@D@2@@std@@@std@@@std@@@std@@QEAA@PEAU?$_List_node@V?$basic_string@DU?$char_traits@D@std@@V?$allocator@D@2@@std@@PEAX@1@PEBV?$_List_val@U?$_List_simple_types@V?$basic_string@DU?$char_traits@D@std@@V?$allocator@D@2@@std@@@std@@@1@@Z 0000000140014398     MessageHistory.obj
 0002:00003398       $unwind$??0?$_List_unchecked_const_iterator@V?$_List_val@U?$_List_simple_types@V?$basic_string@DU?$char_traits@D@std@@V?$allocator@D@2@@std@@@std@@@std@@U_Iterator_base0@2@@std@@QEAA@PEAU?$_List_node@V?$basic_string@DU?$char_traits@D@std@@V?$allocator@D@2@@std@@PEAX@1@PEBV?$_List_val@U?$_List_simple_types@V?$basic_string@DU?$char_traits@D@std@@V?$allocator@D@2@@std@@@std@@@1@@Z 0000000140014398     MessageHistory.obj
 0002:00003398       $unwind$?copy@?$_Char_traits@DH@std@@SAPEADQEADQEBD_K@Z 0000000140014398     MessageHistory.obj
 0002:00003398       $unwind$?deallocate@?$_Default_allocator_traits@V?$allocator@U?$_List_node@V?$basic_string@DU?$char_traits@D@std@@V?$allocator@D@2@@std@@PEAX@std@@@std@@@std@@SAXAEAV?$allocator@U?$_List_node@V?$basic_string@DU?$char_traits@D@std@@V?$allocator@D@2@@std@@PEAX@std@@@2@QEAU?$_List_node@V?$basic_string@DU?$char_traits@D@std@@V?$allocator@D@2@@std@@PEAX@2@_K@Z 0000000140014398     MessageHistory.obj
 0002:00003398       $unwind$?deallocate@?$allocator@D@std@@QEAAXQEAD_K@Z 0000000140014398     MessageHistory.obj
 0002:00003398       $unwind$?deallocate@?$allocator@U?$_List_node@V?$basic_string@DU?$char_traits@D@std@@V?$allocator@D@2@@std@@PEAX@std@@@std@@QEAAXQEAU?$_List_node@V?$basic_string@DU?$char_traits@D@std@@V?$allocator@D@2@@std@@PEAX@2@_K@Z 0000000140014398     MessageHistory.obj
 0002:000033a0       $unwind$?initBroadcastMessageIDs@@YAHXZ 00000001400143a0     AccessBridgeMessages.obj
 0002:000033a8       $unwind$vsnprintf          00000001400143a8     AccessInfo.obj
 0002:000033a8       $unwind$_vsnprintf_l       00000001400143a8     jaccessinspector.obj
 0002:000033b0       $unwind$?getTimeAndDate@@YAPEADXZ 00000001400143b0     AccessInfo.obj
 0002:000033bc       $unwind$?displayAndLog@@YAXPEAUHWND__@@HPEAU_iobuf@@PEADZZ 00000001400143bc     AccessInfo.obj
 0002:000033cc       $unwind$?logString@@YAXPEAU_iobuf@@PEBDZZ 00000001400143cc     AccessInfo.obj
 0002:000033dc       $unwind$?getAccessibleInfo@@YAPEADJ_JPEADH@Z 00000001400143dc     AccessInfo.obj
 0002:000033e4       $unwind$?getAccessibleInfo@@YAPEADJ_JHHPEADH@Z 00000001400143e4     AccessInfo.obj
 0002:000033f8       $unwind$localtime          00000001400143f8     AccessInfo.obj
 0002:00003400       $unwind$time               0000000140014400     AccessInfo.obj
 0002:00003408       $unwind$?appendToBuffer@@YAHPEAD_KPEBDZZ 0000000140014408     AccessInfo.obj
 0002:00003418       $unwind$??0exception@std@@QEAA@QEBDH@Z 0000000140014418     MessageHistory.obj
 0002:00003420       $unwind$??0exception@std@@QEAA@AEBV01@@Z 0000000140014420     MessageHistory.obj
 0002:00003428       $unwind$??$_Allocate@$0BA@U_Default_allocate_traits@std@@$0A@@std@@YAPEAX_K@Z 0000000140014428     MessageHistory.obj
 0002:00003428       $unwind$??0?$_String_val@U?$_Simple_types@D@std@@@std@@QEAA@XZ 0000000140014428     MessageHistory.obj
 0002:00003428       $unwind$??0bad_array_new_length@std@@QEAA@XZ 0000000140014428     MessageHistory.obj
 0002:00003428       $unwind$??1?$_Compressed_pair@V?$allocator@D@std@@V?$_String_val@U?$_Simple_types@D@std@@@2@$00@std@@QEAA@XZ 0000000140014428     MessageHistory.obj
 0002:00003428       $unwind$??1?$_String_val@U?$_Simple_types@D@std@@@std@@QEAA@XZ 0000000140014428     MessageHistory.obj
 0002:00003428       $unwind$??1?$basic_string@DU?$char_traits@D@std@@V?$allocator@D@2@@std@@QEAA@XZ 0000000140014428     MessageHistory.obj
 0002:00003428       $unwind$??1bad_alloc@std@@UEAA@XZ 0000000140014428     MessageHistory.obj
 0002:00003428       $unwind$??1bad_array_new_length@std@@UEAA@XZ 0000000140014428     MessageHistory.obj
 0002:00003428       $unwind$??1exception@std@@UEAA@XZ 0000000140014428     MessageHistory.obj
 0002:00003428       $unwind$?_Allocate@?$_Alloc_construct_ptr@V?$allocator@U?$_List_node@V?$basic_string@DU?$char_traits@D@std@@V?$allocator@D@2@@std@@PEAX@std@@@std@@@std@@QEAAXXZ 0000000140014428     MessageHistory.obj
 0002:00003428       $unwind$?_Allocate@_Default_allocate_traits@std@@SAPEAX_K@Z 0000000140014428     MessageHistory.obj
 0002:00003428       $unwind$?_Getal@?$basic_string@DU?$char_traits@D@std@@V?$allocator@D@2@@std@@AEAAAEAV?$allocator@D@2@XZ 0000000140014428     MessageHistory.obj
 0002:00003428       $unwind$?_Getal@?$basic_string@DU?$char_traits@D@std@@V?$allocator@D@2@@std@@AEBAAEBV?$allocator@D@2@XZ 0000000140014428     MessageHistory.obj
 0002:00003428       $unwind$?_Getal@?$list@V?$basic_string@DU?$char_traits@D@std@@V?$allocator@D@2@@std@@V?$allocator@V?$basic_string@DU?$char_traits@D@std@@V?$allocator@D@2@@std@@@2@@std@@AEAAAEAV?$allocator@U?$_List_node@V?$basic_string@DU?$char_traits@D@std@@V?$allocator@D@2@@std@@PEAX@std@@@2@XZ 0000000140014428     MessageHistory.obj
 0002:00003428       $unwind$?_Getal@?$list@V?$basic_string@DU?$char_traits@D@std@@V?$allocator@D@2@@std@@V?$allocator@V?$basic_string@DU?$char_traits@D@std@@V?$allocator@D@2@@std@@@2@@std@@AEBAAEBV?$allocator@U?$_List_node@V?$basic_string@DU?$char_traits@D@std@@V?$allocator@D@2@@std@@PEAX@std@@@2@XZ 0000000140014428     MessageHistory.obj
 0002:00003428       $unwind$?c_str@?$basic_string@DU?$char_traits@D@std@@V?$allocator@D@2@@std@@QEBAPEBDXZ 0000000140014428     MessageHistory.obj
 0002:00003428       $unwind$?length@?$_Narrow_char_traits@DH@std@@SA_KQEBD@Z 0000000140014428     MessageHistory.obj
 0002:00003428       $unwind$?pop_front@?$list@V?$basic_string@DU?$char_traits@D@std@@V?$allocator@D@2@@std@@V?$allocator@V?$basic_string@DU?$char_traits@D@std@@V?$allocator@D@2@@std@@@2@@std@@QEAAXXZ 0000000140014428     MessageHistory.obj
 0002:00003428       $unwind$??0?$_List_const_iterator@V?$_List_val@U?$_List_simple_types@V?$basic_string@DU?$char_traits@D@std@@V?$allocator@D@2@@std@@@std@@@std@@@std@@QEAA@XZ 0000000140014428     jaccessinspector.obj
 0002:00003428       $unwind$??0MessageHistory@@QEAA@XZ 0000000140014428     jaccessinspector.obj
 0002:00003428       $unwind$??1?$list@V?$basic_string@DU?$char_traits@D@std@@V?$allocator@D@2@@std@@V?$allocator@V?$basic_string@DU?$char_traits@D@std@@V?$allocator@D@2@@std@@@2@@std@@QEAA@XZ 0000000140014428     jaccessinspector.obj
 0002:00003428       $unwind$??1MessageHistory@@QEAA@XZ 0000000140014428     jaccessinspector.obj
 0002:00003430       $unwind$??$_Get_size_of_n@$00@std@@YA_K_K@Z 0000000140014430     MessageHistory.obj
 0002:00003430       $unwind$??F?$_List_const_iterator@V?$_List_val@U?$_List_simple_types@V?$basic_string@DU?$char_traits@D@std@@V?$allocator@D@2@@std@@@std@@@std@@@std@@QEAAAEAV01@XZ 0000000140014430     MessageHistory.obj
 0002:00003430       $unwind$?_Large_string_engaged@?$_String_val@U?$_Simple_types@D@std@@@std@@QEBA_NXZ 0000000140014430     MessageHistory.obj
 0002:00003430       $unwind$?empty@?$list@V?$basic_string@DU?$char_traits@D@std@@V?$allocator@D@2@@std@@V?$allocator@V?$basic_string@DU?$char_traits@D@std@@V?$allocator@D@2@@std@@@2@@std@@QEBA_NXZ 0000000140014430     MessageHistory.obj
 0002:00003430       $unwind$?what@exception@std@@UEBAPEBDXZ 0000000140014430     MessageHistory.obj
 0002:00003438       $unwind$??$?0$$V@?$_Compressed_pair@V?$allocator@D@std@@V?$_String_val@U?$_Simple_types@D@std@@@2@$00@std@@QEAA@U_Zero_then_variadic_args_t@1@@Z 0000000140014438     MessageHistory.obj
 0002:00003438       $unwind$??_G?$basic_string@DU?$char_traits@D@std@@V?$allocator@D@2@@std@@QEAAPEAXI@Z 0000000140014438     MessageHistory.obj
 0002:00003438       $unwind$??_Gbad_alloc@std@@UEAAPEAXI@Z 0000000140014438     MessageHistory.obj
 0002:00003438       $unwind$??_Gbad_array_new_length@std@@UEAAPEAXI@Z 0000000140014438     MessageHistory.obj
 0002:00003438       $unwind$??_Gexception@std@@UEAAPEAXI@Z 0000000140014438     MessageHistory.obj
 0002:00003438       $unwind$??$?0$$V@?$_Compressed_pair@V?$allocator@U?$_List_node@V?$basic_string@DU?$char_traits@D@std@@V?$allocator@D@2@@std@@PEAX@std@@@std@@V?$_List_val@U?$_List_simple_types@V?$basic_string@DU?$char_traits@D@std@@V?$allocator@D@2@@std@@@std@@@2@$00@std@@QEAA@U_Zero_then_variadic_args_t@1@@Z 0000000140014438     jaccessinspector.obj
 0002:00003440       $unwind$??$_Get_unwrapped@AEAV?$_List_const_iterator@V?$_List_val@U?$_List_simple_types@V?$basic_string@DU?$char_traits@D@std@@V?$allocator@D@2@@std@@@std@@@std@@@std@@@std@@YA?A_TAEAV?$_List_const_iterator@V?$_List_val@U?$_List_simple_types@V?$basic_string@DU?$char_traits@D@std@@V?$allocator@D@2@@std@@@std@@@std@@@0@@Z 0000000140014440     MessageHistory.obj
 0002:00003440       $unwind$??$_Seek_wrapped@V?$_List_const_iterator@V?$_List_val@U?$_List_simple_types@V?$basic_string@DU?$char_traits@D@std@@V?$allocator@D@2@@std@@@std@@@std@@@std@@V?$_List_unchecked_const_iterator@V?$_List_val@U?$_List_simple_types@V?$basic_string@DU?$char_traits@D@std@@V?$allocator@D@2@@std@@@std@@@std@@U_Iterator_base0@2@@2@@std@@YAXAEAV?$_List_const_iterator@V?$_List_val@U?$_List_simple_types@V?$basic_string@DU?$char_traits@D@std@@V?$allocator@D@2@@std@@@std@@@std@@@0@$$QEAV?$_List_unchecked_const_iterator@V?$_List_val@U?$_List_simple_types@V?$basic_string@DU?$char_traits@D@std@@V?$allocator@D@2@@std@@@std@@@std@@U_Iterator_base0@2@@0@@Z 0000000140014440     MessageHistory.obj
 0002:00003440       $unwind$??$destroy@V?$basic_string@DU?$char_traits@D@std@@V?$allocator@D@2@@std@@@?$_Default_allocator_traits@V?$allocator@U?$_List_node@V?$basic_string@DU?$char_traits@D@std@@V?$allocator@D@2@@std@@PEAX@std@@@std@@@std@@SAXAEAV?$allocator@U?$_List_node@V?$basic_string@DU?$char_traits@D@std@@V?$allocator@D@2@@std@@PEAX@std@@@1@QEAV?$basic_string@DU?$char_traits@D@std@@V?$allocator@D@2@@1@@Z 0000000140014440     MessageHistory.obj
 0002:00003440       $unwind$??0bad_alloc@std@@AEAA@QEBD@Z 0000000140014440     MessageHistory.obj
 0002:00003440       $unwind$??0bad_alloc@std@@QEAA@AEBV01@@Z 0000000140014440     MessageHistory.obj
 0002:00003440       $unwind$??0bad_array_new_length@std@@QEAA@AEBV01@@Z 0000000140014440     MessageHistory.obj
 0002:00003440       $unwind$?_Calculate_growth@?$basic_string@DU?$char_traits@D@std@@V?$allocator@D@2@@std@@AEBA_K_K@Z 0000000140014440     MessageHistory.obj
 0002:00003440       $unwind$?_Swap_proxy_and_iterators@?$basic_string@DU?$char_traits@D@std@@V?$allocator@D@2@@std@@AEAAXAEAV12@@Z 0000000140014440     MessageHistory.obj
 0002:00003440       $unwind$?_Unwrapped@?$_List_const_iterator@V?$_List_val@U?$_List_simple_types@V?$basic_string@DU?$char_traits@D@std@@V?$allocator@D@2@@std@@@std@@@std@@@std@@QEBA?AV?$_List_unchecked_const_iterator@V?$_List_val@U?$_List_simple_types@V?$basic_string@DU?$char_traits@D@std@@V?$allocator@D@2@@std@@@std@@@std@@U_Iterator_base0@2@@2@XZ 0000000140014440     MessageHistory.obj
 0002:00003440       $unwind$?allocate@?$allocator@D@std@@QEAAPEAD_K@Z 0000000140014440     MessageHistory.obj
 0002:00003440       $unwind$?allocate@?$allocator@U?$_List_node@V?$basic_string@DU?$char_traits@D@std@@V?$allocator@D@2@@std@@PEAX@std@@@std@@QEAAPEAU?$_List_node@V?$basic_string@DU?$char_traits@D@std@@V?$allocator@D@2@@std@@PEAX@2@_K@Z 0000000140014440     MessageHistory.obj
 0002:00003440       $unwind$?begin@?$list@V?$basic_string@DU?$char_traits@D@std@@V?$allocator@D@2@@std@@V?$allocator@V?$basic_string@DU?$char_traits@D@std@@V?$allocator@D@2@@std@@@2@@std@@QEAA?AV?$_List_iterator@V?$_List_val@U?$_List_simple_types@V?$basic_string@DU?$char_traits@D@std@@V?$allocator@D@2@@std@@@std@@@std@@@2@XZ 0000000140014440     MessageHistory.obj
 0002:00003440       $unwind$?end@?$list@V?$basic_string@DU?$char_traits@D@std@@V?$allocator@D@2@@std@@V?$allocator@V?$basic_string@DU?$char_traits@D@std@@V?$allocator@D@2@@std@@@2@@std@@QEAA?AV?$_List_iterator@V?$_List_val@U?$_List_simple_types@V?$basic_string@DU?$char_traits@D@std@@V?$allocator@D@2@@std@@@std@@@std@@@2@XZ 0000000140014440     MessageHistory.obj
 0002:00003440       $unwind$?push_back@?$list@V?$basic_string@DU?$char_traits@D@std@@V?$allocator@D@2@@std@@V?$allocator@V?$basic_string@DU?$char_traits@D@std@@V?$allocator@D@2@@std@@@2@@std@@QEAAX$$QEAV?$basic_string@DU?$char_traits@D@std@@V?$allocator@D@2@@2@@Z 0000000140014440     MessageHistory.obj
 0002:00003448       $unwind$?_Throw_bad_array_new_length@std@@YAXXZ 0000000140014448     MessageHistory.obj
 0002:00003448       $unwind$?__scrt_throw_std_bad_alloc@@YAXXZ 0000000140014448     MSVCRT:throw_bad_alloc.obj
 0002:00003448       $unwind$?__scrt_throw_std_bad_array_new_length@@YAXXZ 0000000140014448     MSVCRT:throw_bad_alloc.obj
 0002:00003450       $unwind$??$distance@V?$_List_const_iterator@V?$_List_val@U?$_List_simple_types@V?$basic_string@DU?$char_traits@D@std@@V?$allocator@D@2@@std@@@std@@@std@@@std@@@std@@YA_JV?$_List_const_iterator@V?$_List_val@U?$_List_simple_types@V?$basic_string@DU?$char_traits@D@std@@V?$allocator@D@2@@std@@@std@@@std@@@0@0@Z 0000000140014450     MessageHistory.obj
 0002:00003450       $unwind$?_Adjust_manually_vector_aligned@std@@YAXAEAPEAXAEA_K@Z 0000000140014450     MessageHistory.obj
 0002:00003458       $unwind$?_Xlen_string@std@@YAXXZ 0000000140014458     MessageHistory.obj
 0002:00003458       $unwind$??__Eg_MessageHistory@@YAXXZ 0000000140014458     jaccessinspector.obj
 0002:00003458       $unwind$??__Fg_MessageHistory@@YAXXZ 0000000140014458     jaccessinspector.obj
 0002:00003458       $unwind$__scrt_initialize_default_local_stdio_options 0000000140014458     MSVCRT:default_local_stdio_options.obj
 0002:00003458       $unwind$?post_pgo_initialization@@YAHXZ 0000000140014458     MSVCRT:exe_winmain.obj
 0002:00003458       $unwind$?pre_cpp_initialization@@YAXXZ 0000000140014458     MSVCRT:exe_winmain.obj
 0002:00003458       $unwind$WinMainCRTStartup  0000000140014458     MSVCRT:exe_winmain.obj
 0002:00003458       $unwind$__report_rangecheckfailure 0000000140014458     MSVCRT:gs_report.obj
 0002:00003458       $unwind$__GSHandlerCheck   0000000140014458     MSVCRT:gshandler.obj
 0002:00003458       $unwind$__scrt_acquire_startup_lock 0000000140014458     MSVCRT:utility.obj
 0002:00003458       $unwind$atexit             0000000140014458     MSVCRT:utility.obj
 0002:00003458       $unwind$__scrt_is_managed_app 0000000140014458     MSVCRT:utility_desktop.obj
 0002:00003460       $unwind$??$_Get_size_of_n@$0DA@@std@@YA_K_K@Z 0000000140014460     MessageHistory.obj
 0002:00003460       $unwind$?_Myptr@?$_String_val@U?$_Simple_types@D@std@@@std@@QEBAPEBDXZ 0000000140014460     MessageHistory.obj
 0002:00003460       $unwind$?_Tidy_init@?$basic_string@DU?$char_traits@D@std@@V?$allocator@D@2@@std@@AEAAXXZ 0000000140014460     MessageHistory.obj
 0002:00003460       $unwind$?clear@?$list@V?$basic_string@DU?$char_traits@D@std@@V?$allocator@D@2@@std@@V?$allocator@V?$basic_string@DU?$char_traits@D@std@@V?$allocator@D@2@@std@@@2@@std@@QEAAXXZ 0000000140014460     MessageHistory.obj
 0002:00003460       $unwind$?max_size@?$list@V?$basic_string@DU?$char_traits@D@std@@V?$allocator@D@2@@std@@V?$allocator@V?$basic_string@DU?$char_traits@D@std@@V?$allocator@D@2@@std@@@2@@std@@QEBA_KXZ 0000000140014460     MessageHistory.obj
 0002:00003460       $unwind$??0?$list@V?$basic_string@DU?$char_traits@D@std@@V?$allocator@D@2@@std@@V?$allocator@V?$basic_string@DU?$char_traits@D@std@@V?$allocator@D@2@@std@@@2@@std@@QEAA@XZ 0000000140014460     jaccessinspector.obj
 0002:00003460       $unwind$?_Tidy@?$list@V?$basic_string@DU?$char_traits@D@std@@V?$allocator@D@2@@std@@V?$allocator@V?$basic_string@DU?$char_traits@D@std@@V?$allocator@D@2@@std@@@2@@std@@AEAAXXZ 0000000140014460     jaccessinspector.obj
 0002:00003460       $unwind$__report_gsfailure 0000000140014460     MSVCRT:gs_report.obj
 0002:00003468       $unwind$??0_Bxty@?$_String_val@U?$_Simple_types@D@std@@@std@@QEAA@XZ 0000000140014468     MessageHistory.obj
 0002:00003470       $unwind$??0?$basic_string@DU?$char_traits@D@std@@V?$allocator@D@2@@std@@QEAA@QEBD@Z 0000000140014470     MessageHistory.obj
 0002:00003480       $cppxdata$??0?$basic_string@DU?$char_traits@D@std@@V?$allocator@D@2@@std@@QEAA@QEBD@Z 0000000140014480     MessageHistory.obj
 0002:00003489       $stateUnwindMap$??0?$basic_string@DU?$char_traits@D@std@@V?$allocator@D@2@@std@@QEAA@QEBD@Z 0000000140014489     MessageHistory.obj
 0002:0000348f       $ip2state$??0?$basic_string@DU?$char_traits@D@std@@V?$allocator@D@2@@std@@QEAA@QEBD@Z 000000014001448f     MessageHistory.obj
 0002:00003498       $unwind$?dtor$0@?0???$?0V?$basic_string@DU?$char_traits@D@std@@V?$allocator@D@2@@std@@@?$_List_node_emplace_op2@V?$allocator@U?$_List_node@V?$basic_string@DU?$char_traits@D@std@@V?$allocator@D@2@@std@@PEAX@std@@@std@@@std@@QEAA@AEAV?$allocator@U?$_List_node@V?$basic_string@DU?$char_traits@D@std@@V?$allocator@D@2@@std@@PEAX@std@@@1@$$QEAV?$basic_string@DU?$char_traits@D@std@@V?$allocator@D@2@@1@@Z@4HA 0000000140014498     MessageHistory.obj
 0002:00003498       $unwind$?dtor$0@?0???0?$basic_string@DU?$char_traits@D@std@@V?$allocator@D@2@@std@@QEAA@QEBD@Z@4HA 0000000140014498     MessageHistory.obj
 0002:00003498       $unwind$?filt$0@?0??__scrt_common_main_seh@@YAHXZ@4HA 0000000140014498     MSVCRT:exe_winmain.obj
 0002:000034a0       $unwind$??$_Construct_in_place@PEADAEAPEAD@std@@YAXAEAPEAD0@Z 00000001400144a0     MessageHistory.obj
 0002:000034a0       $unwind$??$_Construct_in_place@PEADAEBQEAD@std@@YAXAEAPEADAEBQEAD@Z 00000001400144a0     MessageHistory.obj
 0002:000034a0       $unwind$??$_Construct_in_place@PEAU?$_List_node@V?$basic_string@DU?$char_traits@D@std@@V?$allocator@D@2@@std@@PEAX@std@@AEBQEAU12@@std@@YAXAEAPEAU?$_List_node@V?$basic_string@DU?$char_traits@D@std@@V?$allocator@D@2@@std@@PEAX@0@AEBQEAU10@@Z 00000001400144a0     MessageHistory.obj
 0002:000034a0       $unwind$??$_Free_non_head@V?$allocator@U?$_List_node@V?$basic_string@DU?$char_traits@D@std@@V?$allocator@D@2@@std@@PEAX@std@@@std@@@?$_List_node@V?$basic_string@DU?$char_traits@D@std@@V?$allocator@D@2@@std@@PEAX@std@@SAXAEAV?$allocator@U?$_List_node@V?$basic_string@DU?$char_traits@D@std@@V?$allocator@D@2@@std@@PEAX@std@@@1@PEAU01@@Z 00000001400144a0     MessageHistory.obj
 0002:000034a0       $unwind$??$advance@V?$_List_const_iterator@V?$_List_val@U?$_List_simple_types@V?$basic_string@DU?$char_traits@D@std@@V?$allocator@D@2@@std@@@std@@@std@@@std@@_K@std@@YAXAEAV?$_List_const_iterator@V?$_List_val@U?$_List_simple_types@V?$basic_string@DU?$char_traits@D@std@@V?$allocator@D@2@@std@@@std@@@std@@@0@_K@Z 00000001400144a0     MessageHistory.obj
 0002:000034a0       $unwind$??0?$basic_string@DU?$char_traits@D@std@@V?$allocator@D@2@@std@@QEAA@$$QEAV01@@Z 00000001400144a0     MessageHistory.obj
 0002:000034a0       $unwind$??9?$_List_const_iterator@V?$_List_val@U?$_List_simple_types@V?$basic_string@DU?$char_traits@D@std@@V?$allocator@D@2@@std@@@std@@@std@@@std@@QEBA_NAEBV01@@Z 00000001400144a0     MessageHistory.obj
 0002:000034a0       $unwind$??9?$_List_unchecked_const_iterator@V?$_List_val@U?$_List_simple_types@V?$basic_string@DU?$char_traits@D@std@@V?$allocator@D@2@@std@@@std@@@std@@U_Iterator_base0@2@@std@@QEBA_NAEBV01@@Z 00000001400144a0     MessageHistory.obj
 0002:000034a0       $unwind$?_Memcpy_val_from@?$basic_string@DU?$char_traits@D@std@@V?$allocator@D@2@@std@@AEAAXAEBV12@@Z 00000001400144a0     MessageHistory.obj
 0002:000034a0       $unwind$?_Transfer_before@?$_List_node_emplace_op2@V?$allocator@U?$_List_node@V?$basic_string@DU?$char_traits@D@std@@V?$allocator@D@2@@std@@PEAX@std@@@std@@@std@@QEAAPEAU?$_List_node@V?$basic_string@DU?$char_traits@D@std@@V?$allocator@D@2@@std@@PEAX@2@QEAU32@@Z 00000001400144a0     MessageHistory.obj
 0002:000034a0       $unwind$?_Unchecked_erase@?$list@V?$basic_string@DU?$char_traits@D@std@@V?$allocator@D@2@@std@@V?$allocator@V?$basic_string@DU?$char_traits@D@std@@V?$allocator@D@2@@std@@@2@@std@@AEAAPEAU?$_List_node@V?$basic_string@DU?$char_traits@D@std@@V?$allocator@D@2@@std@@PEAX@2@QEAU32@@Z 00000001400144a0     MessageHistory.obj
 0002:000034a0       $unwind$??$_Construct_in_place@PEAU?$_List_node@V?$basic_string@DU?$char_traits@D@std@@V?$allocator@D@2@@std@@PEAX@std@@AEAPEAU12@@std@@YAXAEAPEAU?$_List_node@V?$basic_string@DU?$char_traits@D@std@@V?$allocator@D@2@@std@@PEAX@0@0@Z 00000001400144a0     jaccessinspector.obj
 0002:000034a8       $unwind$?_Take_contents@?$basic_string@DU?$char_traits@D@std@@V?$allocator@D@2@@std@@AEAAXAEAV12@@Z 00000001400144a8     MessageHistory.obj
 0002:000034b8       $cppxdata$??$_Deallocate@$0BA@$0A@@std@@YAXPEAX_K@Z 00000001400144b8     MessageHistory.obj
 0002:000034b8       $cppxdata$??$_Freenode0@V?$allocator@U?$_List_node@V?$basic_string@DU?$char_traits@D@std@@V?$allocator@D@2@@std@@PEAX@std@@@std@@@?$_List_node@V?$basic_string@DU?$char_traits@D@std@@V?$allocator@D@2@@std@@PEAX@std@@SAXAEAV?$allocator@U?$_List_node@V?$basic_string@DU?$char_traits@D@std@@V?$allocator@D@2@@std@@PEAX@std@@@1@PEAU01@@Z 00000001400144b8     MessageHistory.obj
 0002:000034b8       $cppxdata$??$_Freenode@V?$allocator@U?$_List_node@V?$basic_string@DU?$char_traits@D@std@@V?$allocator@D@2@@std@@PEAX@std@@@std@@@?$_List_node@V?$basic_string@DU?$char_traits@D@std@@V?$allocator@D@2@@std@@PEAX@std@@SAXAEAV?$allocator@U?$_List_node@V?$basic_string@DU?$char_traits@D@std@@V?$allocator@D@2@@std@@PEAX@std@@@1@PEAU01@@Z 00000001400144b8     MessageHistory.obj
 0002:000034b8       $cppxdata$??1?$_Alloc_construct_ptr@V?$allocator@U?$_List_node@V?$basic_string@DU?$char_traits@D@std@@V?$allocator@D@2@@std@@PEAX@std@@@std@@@std@@QEAA@XZ 00000001400144b8     MessageHistory.obj
 0002:000034b8       $cppxdata$??1?$_List_node_emplace_op2@V?$allocator@U?$_List_node@V?$basic_string@DU?$char_traits@D@std@@V?$allocator@D@2@@std@@PEAX@std@@@std@@@std@@QEAA@XZ 00000001400144b8     MessageHistory.obj
 0002:000034b8       $cppxdata$?_Take_contents@?$basic_string@DU?$char_traits@D@std@@V?$allocator@D@2@@std@@AEAAXAEAV12@@Z 00000001400144b8     MessageHistory.obj
 0002:000034b8       $cppxdata$?_Tidy_deallocate@?$basic_string@DU?$char_traits@D@std@@V?$allocator@D@2@@std@@AEAAXXZ 00000001400144b8     MessageHistory.obj
 0002:000034bd       $ip2state$??$_Deallocate@$0BA@$0A@@std@@YAXPEAX_K@Z 00000001400144bd     MessageHistory.obj
 0002:000034bd       $ip2state$??$_Freenode0@V?$allocator@U?$_List_node@V?$basic_string@DU?$char_traits@D@std@@V?$allocator@D@2@@std@@PEAX@std@@@std@@@?$_List_node@V?$basic_string@DU?$char_traits@D@std@@V?$allocator@D@2@@std@@PEAX@std@@SAXAEAV?$allocator@U?$_List_node@V?$basic_string@DU?$char_traits@D@std@@V?$allocator@D@2@@std@@PEAX@std@@@1@PEAU01@@Z 00000001400144bd     MessageHistory.obj
 0002:000034bd       $ip2state$??$_Freenode@V?$allocator@U?$_List_node@V?$basic_string@DU?$char_traits@D@std@@V?$allocator@D@2@@std@@PEAX@std@@@std@@@?$_List_node@V?$basic_string@DU?$char_traits@D@std@@V?$allocator@D@2@@std@@PEAX@std@@SAXAEAV?$allocator@U?$_List_node@V?$basic_string@DU?$char_traits@D@std@@V?$allocator@D@2@@std@@PEAX@std@@@1@PEAU01@@Z 00000001400144bd     MessageHistory.obj
 0002:000034bd       $ip2state$??1?$_Alloc_construct_ptr@V?$allocator@U?$_List_node@V?$basic_string@DU?$char_traits@D@std@@V?$allocator@D@2@@std@@PEAX@std@@@std@@@std@@QEAA@XZ 00000001400144bd     MessageHistory.obj
 0002:000034bd       $ip2state$??1?$_List_node_emplace_op2@V?$allocator@U?$_List_node@V?$basic_string@DU?$char_traits@D@std@@V?$allocator@D@2@@std@@PEAX@std@@@std@@@std@@QEAA@XZ 00000001400144bd     MessageHistory.obj
 0002:000034bd       $ip2state$?_Take_contents@?$basic_string@DU?$char_traits@D@std@@V?$allocator@D@2@@std@@AEAAXAEAV12@@Z 00000001400144bd     MessageHistory.obj
 0002:000034bd       $ip2state$?_Tidy_deallocate@?$basic_string@DU?$char_traits@D@std@@V?$allocator@D@2@@std@@AEAAXXZ 00000001400144bd     MessageHistory.obj
 0002:000034c0       $unwind$?max_size@?$basic_string@DU?$char_traits@D@std@@V?$allocator@D@2@@std@@QEBA_KXZ 00000001400144c0     MessageHistory.obj
 0002:000034c8       $unwind$??$construct@V?$basic_string@DU?$char_traits@D@std@@V?$allocator@D@2@@std@@V12@@?$_Default_allocator_traits@V?$allocator@U?$_List_node@V?$basic_string@DU?$char_traits@D@std@@V?$allocator@D@2@@std@@PEAX@std@@@std@@@std@@SAXAEAV?$allocator@U?$_List_node@V?$basic_string@DU?$char_traits@D@std@@V?$allocator@D@2@@std@@PEAX@std@@@1@QEAV?$basic_string@DU?$char_traits@D@std@@V?$allocator@D@2@@1@$$QEAV31@@Z 00000001400144c8     MessageHistory.obj
 0002:000034c8       $unwind$?_Calculate_growth@?$basic_string@DU?$char_traits@D@std@@V?$allocator@D@2@@std@@CA_K_K00@Z 00000001400144c8     MessageHistory.obj
 0002:000034d0       $unwind$?_Tidy_deallocate@?$basic_string@DU?$char_traits@D@std@@V?$allocator@D@2@@std@@AEAAXXZ 00000001400144d0     MessageHistory.obj
 0002:000034e0       $unwind$??$max@_K@std@@YAAEB_KAEB_K0@Z 00000001400144e0     MessageHistory.obj
 0002:000034e0       $unwind$??$min@_K@std@@YAAEB_KAEB_K0@Z 00000001400144e0     MessageHistory.obj
 0002:000034e0       $unwind$??8?$_List_const_iterator@V?$_List_val@U?$_List_simple_types@V?$basic_string@DU?$char_traits@D@std@@V?$allocator@D@2@@std@@@std@@@std@@@std@@QEBA_NAEBV01@@Z 00000001400144e0     MessageHistory.obj
 0002:000034e0       $unwind$??8?$_List_unchecked_const_iterator@V?$_List_val@U?$_List_simple_types@V?$basic_string@DU?$char_traits@D@std@@V?$allocator@D@2@@std@@@std@@@std@@U_Iterator_base0@2@@std@@QEBA_NAEBV01@@Z 00000001400144e0     MessageHistory.obj
 0002:000034e8       $unwind$?AddMessage@MessageHistory@@QEAAXPEBD@Z 00000001400144e8     MessageHistory.obj
 0002:000034fc       $cppxdata$?AddMessage@MessageHistory@@QEAAXPEBD@Z 00000001400144fc     MessageHistory.obj
 0002:00003505       $stateUnwindMap$?AddMessage@MessageHistory@@QEAAXPEBD@Z 0000000140014505     MessageHistory.obj
 0002:0000350b       $ip2state$?AddMessage@MessageHistory@@QEAAXPEBD@Z 000000014001450b     MessageHistory.obj
 0002:00003514       $unwind$?dtor$0@?0??AddMessage@MessageHistory@@QEAAXPEBD@Z@4HA 0000000140014514     MessageHistory.obj
 0002:0000351c       $unwind$?GetFirstMessage@MessageHistory@@QEAAPEBDXZ 000000014001451c     MessageHistory.obj
 0002:00003524       $unwind$?GetPreviousMessage@MessageHistory@@QEAAPEBDXZ 0000000140014524     MessageHistory.obj
 0002:0000352c       $unwind$?GetNextMessage@MessageHistory@@QEAAPEBDXZ 000000014001452c     MessageHistory.obj
 0002:00003534       $unwind$?GetLastMessage@MessageHistory@@QEAAPEBDXZ 0000000140014534     MessageHistory.obj
 0002:0000353c       $unwind$?GetCurrentMessage@MessageHistory@@QEAAPEBDXZ 000000014001453c     MessageHistory.obj
 0002:00003544       $unwind$?GetMessageA@MessageHistory@@QEAAPEBD_K@Z 0000000140014544     MessageHistory.obj
 0002:0000354c       $unwind$?GetCurrentMessageIndex@MessageHistory@@QEAA_KXZ 000000014001454c     MessageHistory.obj
 0002:00003554       $unwind$?IsFirstMessage@MessageHistory@@QEAAHXZ 0000000140014554     MessageHistory.obj
 0002:0000355c       $unwind$?IsLastMessage@MessageHistory@@QEAAHXZ 000000014001455c     MessageHistory.obj
 0002:00003564       $unwind$?GetMessageCount@MessageHistory@@QEAA_KXZ 0000000140014564     MessageHistory.obj
 0002:0000356c       $unwind$?clear@MessageHistory@@QEAAXXZ 000000014001456c     MessageHistory.obj
 0002:00003574       $unwind$??$_Emplace@V?$basic_string@DU?$char_traits@D@std@@V?$allocator@D@2@@std@@@?$list@V?$basic_string@DU?$char_traits@D@std@@V?$allocator@D@2@@std@@V?$allocator@V?$basic_string@DU?$char_traits@D@std@@V?$allocator@D@2@@std@@@2@@std@@QEAAPEAU?$_List_node@V?$basic_string@DU?$char_traits@D@std@@V?$allocator@D@2@@std@@PEAX@1@QEAU21@$$QEAV?$basic_string@DU?$char_traits@D@std@@V?$allocator@D@2@@1@@Z 0000000140014574     MessageHistory.obj
 0002:0000357c       $unwind$??$?0V?$allocator@D@std@@$$V@?$_Compressed_pair@V?$allocator@D@std@@V?$_String_val@U?$_Simple_types@D@std@@@2@$00@std@@QEAA@U_One_then_variadic_args_t@1@$$QEAV?$allocator@D@1@@Z 000000014001457c     MessageHistory.obj
 0002:00003584       $unwind$??$_Construct@$00PEBD@?$basic_string@DU?$char_traits@D@std@@V?$allocator@D@2@@std@@AEAAXQEBD_K@Z 0000000140014584     MessageHistory.obj
 0002:0000358c       $unwind$??$_Deallocate@$0BA@$0A@@std@@YAXPEAX_K@Z 000000014001458c     MessageHistory.obj
 0002:0000358c       $unwind$??$_Freenode0@V?$allocator@U?$_List_node@V?$basic_string@DU?$char_traits@D@std@@V?$allocator@D@2@@std@@PEAX@std@@@std@@@?$_List_node@V?$basic_string@DU?$char_traits@D@std@@V?$allocator@D@2@@std@@PEAX@std@@SAXAEAV?$allocator@U?$_List_node@V?$basic_string@DU?$char_traits@D@std@@V?$allocator@D@2@@std@@PEAX@std@@@1@PEAU01@@Z 000000014001458c     MessageHistory.obj
 0002:0000358c       $unwind$??$_Freenode@V?$allocator@U?$_List_node@V?$basic_string@DU?$char_traits@D@std@@V?$allocator@D@2@@std@@PEAX@std@@@std@@@?$_List_node@V?$basic_string@DU?$char_traits@D@std@@V?$allocator@D@2@@std@@PEAX@std@@SAXAEAV?$allocator@U?$_List_node@V?$basic_string@DU?$char_traits@D@std@@V?$allocator@D@2@@std@@PEAX@std@@@1@PEAU01@@Z 000000014001458c     MessageHistory.obj
 0002:0000359c       $unwind$??1?$_Alloc_construct_ptr@V?$allocator@U?$_List_node@V?$basic_string@DU?$char_traits@D@std@@V?$allocator@D@2@@std@@PEAX@std@@@std@@@std@@QEAA@XZ 000000014001459c     MessageHistory.obj
 0002:0000359c       $unwind$??1?$_List_node_emplace_op2@V?$allocator@U?$_List_node@V?$basic_string@DU?$char_traits@D@std@@V?$allocator@D@2@@std@@PEAX@std@@@std@@@std@@QEAA@XZ 000000014001459c     MessageHistory.obj
 0002:000035ac       $unwind$??$?0V?$basic_string@DU?$char_traits@D@std@@V?$allocator@D@2@@std@@@?$_List_node_emplace_op2@V?$allocator@U?$_List_node@V?$basic_string@DU?$char_traits@D@std@@V?$allocator@D@2@@std@@PEAX@std@@@std@@@std@@QEAA@AEAV?$allocator@U?$_List_node@V?$basic_string@DU?$char_traits@D@std@@V?$allocator@D@2@@std@@PEAX@std@@@1@$$QEAV?$basic_string@DU?$char_traits@D@std@@V?$allocator@D@2@@1@@Z 00000001400145ac     MessageHistory.obj
 0002:000035bc       $cppxdata$??$?0V?$basic_string@DU?$char_traits@D@std@@V?$allocator@D@2@@std@@@?$_List_node_emplace_op2@V?$allocator@U?$_List_node@V?$basic_string@DU?$char_traits@D@std@@V?$allocator@D@2@@std@@PEAX@std@@@std@@@std@@QEAA@AEAV?$allocator@U?$_List_node@V?$basic_string@DU?$char_traits@D@std@@V?$allocator@D@2@@std@@PEAX@std@@@1@$$QEAV?$basic_string@DU?$char_traits@D@std@@V?$allocator@D@2@@1@@Z 00000001400145bc     MessageHistory.obj
 0002:000035c5       $stateUnwindMap$??$?0V?$basic_string@DU?$char_traits@D@std@@V?$allocator@D@2@@std@@@?$_List_node_emplace_op2@V?$allocator@U?$_List_node@V?$basic_string@DU?$char_traits@D@std@@V?$allocator@D@2@@std@@PEAX@std@@@std@@@std@@QEAA@AEAV?$allocator@U?$_List_node@V?$basic_string@DU?$char_traits@D@std@@V?$allocator@D@2@@std@@PEAX@std@@@1@$$QEAV?$basic_string@DU?$char_traits@D@std@@V?$allocator@D@2@@1@@Z 00000001400145c5     MessageHistory.obj
 0002:000035cb       $ip2state$??$?0V?$basic_string@DU?$char_traits@D@std@@V?$allocator@D@2@@std@@@?$_List_node_emplace_op2@V?$allocator@U?$_List_node@V?$basic_string@DU?$char_traits@D@std@@V?$allocator@D@2@@std@@PEAX@std@@@std@@@std@@QEAA@AEAV?$allocator@U?$_List_node@V?$basic_string@DU?$char_traits@D@std@@V?$allocator@D@2@@std@@PEAX@std@@@1@$$QEAV?$basic_string@DU?$char_traits@D@std@@V?$allocator@D@2@@1@@Z 00000001400145cb     MessageHistory.obj
 0002:000035d4       $unwind$??$_Allocate_manually_vector_aligned@U_Default_allocate_traits@std@@@std@@YAPEAX_K@Z 00000001400145d4     MessageHistory.obj
 0002:000035d4       $unwind$?_Alloc_sentinel_and_proxy@?$list@V?$basic_string@DU?$char_traits@D@std@@V?$allocator@D@2@@std@@V?$allocator@V?$basic_string@DU?$char_traits@D@std@@V?$allocator@D@2@@std@@@2@@std@@AEAAXXZ 00000001400145d4     jaccessinspector.obj
 0002:000035dc       $unwind$WinMain            00000001400145dc     jaccessinspector.obj
 0002:000035e4       $unwind$?TimerProc@@YAXPEAUHWND__@@IIK@Z 00000001400145e4     jaccessinspector.obj
 0002:000035ec       $unwind$?KeyboardProc@@YA_JH_K_J@Z 00000001400145ec     jaccessinspector.obj
 0002:000035f4       $unwind$?MouseProc@@YA_JH_K_J@Z 00000001400145f4     jaccessinspector.obj
 0002:000035fc       $unwind$?InitWindow@@YAHPEAX@Z 00000001400145fc     jaccessinspector.obj
 0002:00003604       $unwind$?jaccessinspectorDialogProc@@YA_JPEAUHWND__@@I_K_J@Z 0000000140014604     jaccessinspector.obj
 0002:00003614       $unwind$?HandleJavaShutdown@@YAXJ@Z 0000000140014614     jaccessinspector.obj
 0002:00003624       $unwind$?HandleJavaFocusGained@@YAXJ_J0@Z 0000000140014624     jaccessinspector.obj
 0002:00003634       $unwind$?HandleJavaFocusLost@@YAXJ_J0@Z 0000000140014634     jaccessinspector.obj
 0002:00003644       $unwind$?HandleJavaCaretUpdate@@YAXJ_J0@Z 0000000140014644     jaccessinspector.obj
 0002:0000364c       $unwind$?HandleMouseClicked@@YAXJ_J0@Z 000000014001464c     jaccessinspector.obj
 0002:00003654       $unwind$?HandleMouseEntered@@YAXJ_J0@Z 0000000140014654     jaccessinspector.obj
 0002:0000365c       $unwind$?HandleMouseExited@@YAXJ_J0@Z 000000014001465c     jaccessinspector.obj
 0002:00003664       $unwind$?HandleMousePressed@@YAXJ_J0@Z 0000000140014664     jaccessinspector.obj
 0002:0000366c       $unwind$?HandleMouseReleased@@YAXJ_J0@Z 000000014001466c     jaccessinspector.obj
 0002:00003674       $unwind$?HandleMenuCanceled@@YAXJ_J0@Z 0000000140014674     jaccessinspector.obj
 0002:0000367c       $unwind$?HandleMenuDeselected@@YAXJ_J0@Z 000000014001467c     jaccessinspector.obj
 0002:00003684       $unwind$?HandleMenuSelected@@YAXJ_J0@Z 0000000140014684     jaccessinspector.obj
 0002:0000368c       $unwind$?HandlePopupMenuCanceled@@YAXJ_J0@Z 000000014001468c     jaccessinspector.obj
 0002:00003694       $unwind$?HandlePopupMenuWillBecomeInvisible@@YAXJ_J0@Z 0000000140014694     jaccessinspector.obj
 0002:0000369c       $unwind$?HandlePopupMenuWillBecomeVisible@@YAXJ_J0@Z 000000014001469c     jaccessinspector.obj
 0002:000036a4       $unwind$?HandlePropertyNameChange@@YAXJ_J0PEAG1@Z 00000001400146a4     jaccessinspector.obj
 0002:000036b4       $unwind$?HandlePropertyDescriptionChange@@YAXJ_J0PEAG1@Z 00000001400146b4     jaccessinspector.obj
 0002:000036c4       $unwind$?HandlePropertyStateChange@@YAXJ_J0PEAG1@Z 00000001400146c4     jaccessinspector.obj
 0002:000036d4       $unwind$?HandlePropertyValueChange@@YAXJ_J0PEAG1@Z 00000001400146d4     jaccessinspector.obj
 0002:000036e4       $unwind$?HandlePropertySelectionChange@@YAXJ_J0@Z 00000001400146e4     jaccessinspector.obj
 0002:000036ec       $unwind$?HandlePropertyTextChange@@YAXJ_J0@Z 00000001400146ec     jaccessinspector.obj
 0002:000036f4       $unwind$?HandlePropertyCaretChange@@YAXJ_J0HH@Z 00000001400146f4     jaccessinspector.obj
 0002:00003704       $unwind$?HandlePropertyVisibleDataChange@@YAXJ_J0@Z 0000000140014704     jaccessinspector.obj
 0002:0000370c       $unwind$?HandlePropertyTableModelChange@@YAXJ_J0PEAG1@Z 000000014001470c     jaccessinspector.obj
 0002:0000371c       $unwind$?SaveActiveEventOptionsToRegistry@@YAHXZ 000000014001471c     jaccessinspector.obj
 0002:00003724       $unwind$?ReadActiveEventOptionsFromRegistry@@YAHXZ 0000000140014724     jaccessinspector.obj
 0002:0000372c       $unwind$?ApplyEventOptions@@YAXPEAUHWND__@@@Z 000000014001472c     jaccessinspector.obj
 0002:00003734       $unwind$?EnableDlgItem@@YAHPEAUHWND__@@HH@Z 0000000140014734     jaccessinspector.obj
 0002:0000373c       $unwind$?EnableMessageNavButtons@@YAXXZ 000000014001473c     jaccessinspector.obj
 0002:00003744       $unwind$?AddToMessageHistory@@YAXPEBD@Z 0000000140014744     jaccessinspector.obj
 0002:0000374c       $unwind$?UpdateMessageNumber@@YAHXZ 000000014001474c     jaccessinspector.obj
 0002:0000375c       $unwind$?GoToMessageDialogProc@@YA_JPEAUHWND__@@I_K_J@Z 000000014001475c     jaccessinspector.obj
 0002:0000376c       $unwind$?InitGoToMessageDialogBox@@YAHPEAX@Z 000000014001476c     jaccessinspector.obj
 0002:00003774       $unwind$?MaybeCheckMonitorTheSameEventsAsJAWS@@YAXPEAUHMENU__@@@Z 0000000140014774     jaccessinspector.obj
 0002:0000377c       $unwind$?MaybeCheckMonitorAllEvents@@YAXPEAUHMENU__@@@Z 000000014001477c     jaccessinspector.obj
 0002:00003784       $unwind$?displayAccessibleInfo@@YAXJ_JHH@Z 0000000140014784     jaccessinspector.obj
 0002:00003794       $unwind$?displayJavaEvent@@YAXJ_JPEAD@Z 0000000140014794     jaccessinspector.obj
 0002:000037a4       $unwind$?displayAccessiblePropertyChange@@YAXJ_JPEBD@Z 00000001400147a4     jaccessinspector.obj
 0002:000037b4       $unwind$?echoMouseObject@@YAXXZ 00000001400147b4     jaccessinspector.obj
 0002:000037c4       $unwind$?echoMouseHWNDObject@@YAXXZ 00000001400147c4     jaccessinspector.obj
 0002:000037cc       $unwind$?displayFocusedObject@@YAXXZ 00000001400147cc     jaccessinspector.obj
 0002:000037d4       $unwind$?HandlePropertyChildChange@@YAXJ_J000@Z 00000001400147d4     jaccessinspector.obj
 0002:000037e4       $unwind$?HandlePropertyActiveDescendentChange@@YAXJ_J000@Z 00000001400147e4     jaccessinspector.obj
 0002:000037f4       $unwind$?exitjaccessinspector@@YAXPEAUHWND__@@@Z 00000001400147f4     jaccessinspector.obj
 0002:000037fc       $unwind$?reinstallEventListeners@@YAXXZ 00000001400147fc     jaccessinspector.obj
 0002:00003804       $unwind$__report_securityfailure 0000000140014804     MSVCRT:gs_report.obj
 0002:0000380c       $unwind$capture_current_context 000000014001480c     MSVCRT:gs_report.obj
 0002:00003818       $unwind$capture_previous_context 0000000140014818     MSVCRT:gs_report.obj
 0002:00003824       $unwind$?pre_c_initialization@@YAHXZ 0000000140014824     MSVCRT:exe_winmain.obj
 0002:00003824       $unwind$__raise_securityfailure 0000000140014824     MSVCRT:gs_report.obj
 0002:00003824       $unwind$??2@YAPEAX_K@Z     0000000140014824     MSVCRT:new_scalar.obj
 0002:00003824       $unwind$??_Gtype_info@@UEAAPEAXI@Z 0000000140014824     MSVCRT:std_type_info_static.obj
 0002:00003824       $unwind$_Init_thread_footer 0000000140014824     MSVCRT:thread_safe_statics.obj
 0002:00003824       $unwind$_Init_thread_header 0000000140014824     MSVCRT:thread_safe_statics.obj
 0002:00003824       $unwind$__scrt_initialize_crt 0000000140014824     MSVCRT:utility.obj
 0002:00003824       $unwind$__scrt_initialize_onexit_tables 0000000140014824     MSVCRT:utility.obj
 0002:00003824       $unwind$__scrt_release_startup_lock 0000000140014824     MSVCRT:utility.obj
 0002:00003824       $unwind$__scrt_uninitialize_crt 0000000140014824     MSVCRT:utility.obj
 0002:00003824       $unwind$_onexit            0000000140014824     MSVCRT:utility.obj
 0002:0000382c       $unwind$__GSHandlerCheckCommon 000000014001482c     MSVCRT:gshandler.obj
 0002:00003838       $xdatasym                  0000000140014838     MSVCRT:chkstk.obj
 0002:00003840       $xdatasym                  0000000140014840     MSVCRT:amdsecgs.obj
 0002:00003844       $unwind$__GSHandlerCheck_EH4 0000000140014844     MSVCRT:gshandlereh4.obj
 0002:0000385c       $unwind$__scrt_is_nonwritable_in_current_image 000000014001485c     MSVCRT:utility.obj
 0002:0000387c       $unwind$__scrt_is_nonwritable_in_current_image$filt$0 000000014001487c     MSVCRT:utility.obj
 0002:00003884       $unwind$?__scrt_common_main_seh@@YAHXZ 0000000140014884     MSVCRT:exe_winmain.obj
 0002:000038b8       $unwind$__isa_available_init 00000001400148b8     MSVCRT:cpu_disp.obj
 0002:000038c8       $unwind$__scrt_get_show_window_mode 00000001400148c8     MSVCRT:utility_desktop.obj
 0002:000038d0       $unwind$__scrt_fastfail    00000001400148d0     MSVCRT:utility_desktop.obj
 0002:000038e0       $unwind$_RTC_Initialize    00000001400148e0     MSVCRT:initsect.obj
 0002:000038e0       $unwind$_RTC_Terminate     00000001400148e0     MSVCRT:initsect.obj
 0002:000038e0       $unwind$__scrt_unhandled_exception_filter 00000001400148e0     MSVCRT:utility_desktop.obj
 0002:000038ec       $unwind$__security_init_cookie 00000001400148ec     MSVCRT:gs_support.obj
 0002:000038f8       $xdatasym                  00000001400148f8     MSVCRT:guard_dispatch.obj
 0002:00003900       $xdatasym                  0000000140014900     MSVCRT:guard_xfg_dispatch.obj
 0002:00003fc4       .idata$6                   0000000140014fc4     advapi32:ADVAPI32.dll
 0002:00004264       .idata$6                   0000000140015264     user32:USER32.dll
 0002:00004292       .idata$6                   0000000140015292     msvcprt:MSVCP140.dll
 0002:000044da       .idata$6                   00000001400154da     kernel32:KERNEL32.dll
 0002:000045a6       .idata$6                   00000001400155a6     vcruntime:VCRUNTIME140.dll
 0002:000045b8       .idata$6                   00000001400155b8     vcruntime:VCRUNTIME140_1.dll
 0002:0000487c       .idata$6                   000000014001587c     ucrt:api-ms-win-crt-string-l1-1-0.dll
 0002:0000489e       .idata$6                   000000014001589e     ucrt:api-ms-win-crt-stdio-l1-1-0.dll
 0002:000048be       .idata$6                   00000001400158be     ucrt:api-ms-win-crt-environment-l1-1-0.dll
 0002:000048e4       .idata$6                   00000001400158e4     ucrt:api-ms-win-crt-time-l1-1-0.dll
 0002:00004904       .idata$6                   0000000140015904     ucrt:api-ms-win-crt-runtime-l1-1-0.dll
 0002:00004926       .idata$6                   0000000140015926     ucrt:api-ms-win-crt-heap-l1-1-0.dll
 0002:00004946       .idata$6                   0000000140015946     ucrt:api-ms-win-crt-math-l1-1-0.dll
 0002:00004966       .idata$6                   0000000140015966     ucrt:api-ms-win-crt-locale-l1-1-0.dll
 0003:00000000       $SG37387                   0000000140016000     AccessBridgeCalls.obj
 0003:00000018       $SG37391                   0000000140016018     AccessBridgeCalls.obj
 0003:00000028       $SG37393                   0000000140016028     AccessBridgeCalls.obj
 0003:00000040       $SG37395                   0000000140016040     AccessBridgeCalls.obj
 0003:00000058       $SG37397                   0000000140016058     AccessBridgeCalls.obj
 0003:00000068       $SG37399                   0000000140016068     AccessBridgeCalls.obj
 0003:00000080       $SG37401                   0000000140016080     AccessBridgeCalls.obj
 0003:00000098       $SG37403                   0000000140016098     AccessBridgeCalls.obj
 0003:000000b0       $SG37405                   00000001400160b0     AccessBridgeCalls.obj
 0003:000000c8       $SG37407                   00000001400160c8     AccessBridgeCalls.obj
 0003:000000e0       $SG37409                   00000001400160e0     AccessBridgeCalls.obj
 0003:000000f8       $SG37411                   00000001400160f8     AccessBridgeCalls.obj
 0003:00000110       $SG37413                   0000000140016110     AccessBridgeCalls.obj
 0003:00000128       $SG37415                   0000000140016128     AccessBridgeCalls.obj
 0003:00000140       $SG37417                   0000000140016140     AccessBridgeCalls.obj
 0003:00000158       $SG37419                   0000000140016158     AccessBridgeCalls.obj
 0003:00000180       $SG37421                   0000000140016180     AccessBridgeCalls.obj
 0003:000001a0       $SG37423                   00000001400161a0     AccessBridgeCalls.obj
 0003:000001b8       $SG37425                   00000001400161b8     AccessBridgeCalls.obj
 0003:000001d8       $SG37427                   00000001400161d8     AccessBridgeCalls.obj
 0003:000001f8       $SG37429                   00000001400161f8     AccessBridgeCalls.obj
 0003:00000218       $SG37431                   0000000140016218     AccessBridgeCalls.obj
 0003:00000238       $SG37433                   0000000140016238     AccessBridgeCalls.obj
 0003:00000250       $SG37435                   0000000140016250     AccessBridgeCalls.obj
 0003:00000270       $SG37437                   0000000140016270     AccessBridgeCalls.obj
 0003:00000290       $SG37439                   0000000140016290     AccessBridgeCalls.obj
 0003:000002b0       $SG37441                   00000001400162b0     AccessBridgeCalls.obj
 0003:000002d8       $SG37443                   00000001400162d8     AccessBridgeCalls.obj
 0003:000002f8       $SG37445                   00000001400162f8     AccessBridgeCalls.obj
 0003:00000310       $SG37447                   0000000140016310     AccessBridgeCalls.obj
 0003:00000320       $SG37449                   0000000140016320     AccessBridgeCalls.obj
 0003:00000330       $SG37451                   0000000140016330     AccessBridgeCalls.obj
 0003:00000340       $SG37453                   0000000140016340     AccessBridgeCalls.obj
 0003:00000360       $SG37455                   0000000140016360     AccessBridgeCalls.obj
 0003:00000380       $SG37457                   0000000140016380     AccessBridgeCalls.obj
 0003:00000398       $SG37459                   0000000140016398     AccessBridgeCalls.obj
 0003:000003b8       $SG37461                   00000001400163b8     AccessBridgeCalls.obj
 0003:000003d8       $SG37463                   00000001400163d8     AccessBridgeCalls.obj
 0003:000003f8       $SG37465                   00000001400163f8     AccessBridgeCalls.obj
 0003:00000418       $SG37467                   0000000140016418     AccessBridgeCalls.obj
 0003:00000430       $SG37469                   0000000140016430     AccessBridgeCalls.obj
 0003:00000450       $SG37471                   0000000140016450     AccessBridgeCalls.obj
 0003:00000470       $SG37473                   0000000140016470     AccessBridgeCalls.obj
 0003:00000490       $SG37475                   0000000140016490     AccessBridgeCalls.obj
 0003:000004b8       $SG37477                   00000001400164b8     AccessBridgeCalls.obj
 0003:000004e0       $SG37479                   00000001400164e0     AccessBridgeCalls.obj
 0003:00000508       $SG37481                   0000000140016508     AccessBridgeCalls.obj
 0003:00000528       $SG37483                   0000000140016528     AccessBridgeCalls.obj
 0003:00000548       $SG37485                   0000000140016548     AccessBridgeCalls.obj
 0003:00000570       $SG37487                   0000000140016570     AccessBridgeCalls.obj
 0003:00000590       $SG37489                   0000000140016590     AccessBridgeCalls.obj
 0003:000005b8       $SG37491                   00000001400165b8     AccessBridgeCalls.obj
 0003:000005d0       $SG37493                   00000001400165d0     AccessBridgeCalls.obj
 0003:000005f0       $SG37495                   00000001400165f0     AccessBridgeCalls.obj
 0003:00000608       $SG37497                   0000000140016608     AccessBridgeCalls.obj
 0003:00000628       $SG37499                   0000000140016628     AccessBridgeCalls.obj
 0003:00000640       $SG37501                   0000000140016640     AccessBridgeCalls.obj
 0003:00000660       $SG37503                   0000000140016660     AccessBridgeCalls.obj
 0003:00000680       $SG37505                   0000000140016680     AccessBridgeCalls.obj
 0003:000006a0       $SG37507                   00000001400166a0     AccessBridgeCalls.obj
 0003:000006c0       $SG37509                   00000001400166c0     AccessBridgeCalls.obj
 0003:000006d8       $SG37511                   00000001400166d8     AccessBridgeCalls.obj
 0003:000006f8       $SG37513                   00000001400166f8     AccessBridgeCalls.obj
 0003:00000710       $SG37515                   0000000140016710     AccessBridgeCalls.obj
 0003:00000728       $SG37517                   0000000140016728     AccessBridgeCalls.obj
 0003:00000740       $SG37519                   0000000140016740     AccessBridgeCalls.obj
 0003:00000758       $SG37521                   0000000140016758     AccessBridgeCalls.obj
 0003:00000770       $SG37523                   0000000140016770     AccessBridgeCalls.obj
 0003:00000790       $SG37525                   0000000140016790     AccessBridgeCalls.obj
 0003:000007b0       $SG37527                   00000001400167b0     AccessBridgeCalls.obj
 0003:000007c8       $SG37529                   00000001400167c8     AccessBridgeCalls.obj
 0003:000007e8       $SG37531                   00000001400167e8     AccessBridgeCalls.obj
 0003:00000800       $SG37533                   0000000140016800     AccessBridgeCalls.obj
 0003:00000828       $SG37535                   0000000140016828     AccessBridgeCalls.obj
 0003:00000850       $SG37537                   0000000140016850     AccessBridgeCalls.obj
 0003:00000878       $SG37539                   0000000140016878     AccessBridgeCalls.obj
 0003:000008a0       $SG37541                   00000001400168a0     AccessBridgeCalls.obj
 0003:000008c8       $SG37543                   00000001400168c8     AccessBridgeCalls.obj
 0003:000008f0       $SG37545                   00000001400168f0     AccessBridgeCalls.obj
 0003:00000918       $SG37547                   0000000140016918     AccessBridgeCalls.obj
 0003:00000940       $SG37549                   0000000140016940     AccessBridgeCalls.obj
 0003:00000968       $SG37551                   0000000140016968     AccessBridgeCalls.obj
 0003:00000990       $SG37553                   0000000140016990     AccessBridgeCalls.obj
 0003:000009a0       $SG37555                   00000001400169a0     AccessBridgeCalls.obj
 0003:000009b8       $SG37557                   00000001400169b8     AccessBridgeCalls.obj
 0003:000009d0       $SG37559                   00000001400169d0     AccessBridgeCalls.obj
 0003:000009f0       $SG37561                   00000001400169f0     AccessBridgeCalls.obj
 0003:00000a00       $SG37563                   0000000140016a00     AccessBridgeCalls.obj
 0003:00000a18       $SG37565                   0000000140016a18     AccessBridgeCalls.obj
 0003:00000a38       $SG37567                   0000000140016a38     AccessBridgeCalls.obj
 0003:00000a48       $SG37569                   0000000140016a48     AccessBridgeCalls.obj
 0003:00000a58       $SG37571                   0000000140016a58     AccessBridgeCalls.obj
 0003:00000a78       $SG37573                   0000000140016a78     AccessBridgeCalls.obj
 0003:00000a90       $SG37575                   0000000140016a90     AccessBridgeCalls.obj
 0003:00000aa8       $SG37577                   0000000140016aa8     AccessBridgeCalls.obj
 0003:00000ac0       $SG37579                   0000000140016ac0     AccessBridgeCalls.obj
 0003:00000ad8       $SG37581                   0000000140016ad8     AccessBridgeCalls.obj
 0003:00000af0       ?warning@?1??appendToBuffer@@YAHPEAD_KPEBDZZ@4PADA 0000000140016af0     AccessInfo.obj
 0003:00000c50       logFP                      0000000140016c50     AccessBridgeDebug.obj
 0003:00000c60       ?retbuf@?1??printError@@9@4PADA 0000000140016c60     AccessBridgeDebug.obj
 0003:00000d70       ?datebuf@?1??getTimeAndDate@@YAPEADXZ@4PADA 0000000140016d70     AccessInfo.obj
 0003:00000e70       ?titleBarHeight@?1??jaccessinspectorDialogProc@@YA_JPEAUHWND__@@I_K_J@Z@4HA 0000000140016e70     jaccessinspector.obj
 0003:00000e74       ?$TSS0@?1??jaccessinspectorDialogProc@@YA_JPEAUHWND__@@I_K_J@Z@4HA 0000000140016e74     jaccessinspector.obj
 0003:00000e78       ?menuBarHeight@?1??jaccessinspectorDialogProc@@YA_JPEAUHWND__@@I_K_J@Z@4HA 0000000140016e78     jaccessinspector.obj
 0003:00000e7c       ?$TSS1@?1??jaccessinspectorDialogProc@@YA_JPEAUHWND__@@I_K_J@Z@4HA 0000000140016e7c     jaccessinspector.obj
 0003:00000e80       ?borderHeight@?1??jaccessinspectorDialogProc@@YA_JPEAUHWND__@@I_K_J@Z@4HA 0000000140016e80     jaccessinspector.obj
 0003:00000e84       ?$TSS2@?1??jaccessinspectorDialogProc@@YA_JPEAUHWND__@@I_K_J@Z@4HA 0000000140016e84     jaccessinspector.obj
 0003:00000e88       ?borderWidth@?1??jaccessinspectorDialogProc@@YA_JPEAUHWND__@@I_K_J@Z@4HA 0000000140016e88     jaccessinspector.obj
 0003:00000e8c       ?$TSS3@?1??jaccessinspectorDialogProc@@YA_JPEAUHWND__@@I_K_J@Z@4HA 0000000140016e8c     jaccessinspector.obj
 0003:00000e90       ?verticalScrollBarWidth@?1??jaccessinspectorDialogProc@@YA_JPEAUHWND__@@I_K_J@Z@4HA 0000000140016e90     jaccessinspector.obj
 0003:00000e94       ?$TSS4@?1??jaccessinspectorDialogProc@@YA_JPEAUHWND__@@I_K_J@Z@4HA 0000000140016e94     jaccessinspector.obj
 0003:00000ea0       GS_ExceptionRecord         0000000140016ea0     MSVCRT:gs_report.obj
 0003:00000f40       GS_ContextRecord           0000000140016f40     MSVCRT:gs_report.obj
 0003:00001420       ?is_initialized_as_dll@@3_NA 0000000140017420     MSVCRT:utility.obj
 0003:00001421       ?module_local_atexit_table_initialized@@3_NA 0000000140017421     MSVCRT:utility.obj
 0003:00001428       ?module_local_atexit_table@@3U_onexit_table_t@@A 0000000140017428     MSVCRT:utility.obj
 0003:00001440       ?module_local_at_quick_exit_table@@3U_onexit_table_t@@A 0000000140017440     MSVCRT:utility.obj
 0003:00001458       ?g_tss_cv@@3U_RTL_CONDITION_VARIABLE@@A 0000000140017458     MSVCRT:thread_safe_statics.obj
 0003:00001460       ?g_tss_srw@@3U_RTL_SRWLOCK@@A 0000000140017460     MSVCRT:thread_safe_statics.obj
 0005:000001c0       $R000000                   00000001400191c0     jaccessinspector.exe.res
 0005:00000510       $R000350                   0000000140019510     jaccessinspector.exe.res
 0005:000006a8       $R0004E8                   00000001400196a8     jaccessinspector.exe.res
 0005:000007b8       $R0005F8                   00000001400197b8     jaccessinspector.exe.res
 0005:00001060       $R000EA0                   000000014001a060     jaccessinspector.exe.res
